:020000040800F2
:1000000000A0002009340108A57400083D2401085F
:10001000A3740008A17400089F7400080000000089
:100020000000000000000000000000009D740008B7
:100030009B7400080000000099740008AF060108D6
:1000400071340108713401087134010871340108F8
:1000500071340108713401087134010871340108E8
:1000600071340108713401087134010871340108D8
:1000700071340108154B0008EDD7000871340108F0
:1000800071340108713401087134010871340108B8
:10009000D56C00087134010871340108713401080D
:1000A000E1740008F1D50008CF74000815D60008E7
:1000B000E5D50008D5D50008117500087134010890
:1000C0007134010871340108713401087134010878
:1000D00071340108E5D70008DDD700087134010844
:1000E000BD06010871340108C56C000871340108AF
:1000F000F1740008713401080175000871340108B9
:100100000000000000000000000000007134010841
:100110007134010871340108713401087134010827
:100120007134010871340108713401087134010817
:100130007134010871340108000000000000000063
:1001400071340108713401087134010800000000A5
:10015000000000000000000000000000000000009F
:100160000000000000000000713401087134010833
:1001700071340108000000000000000000000000D1
:080180000000000071340108C9
:100188002DE9F04F2DED068B754D764B2B60AFB0FA
:1001980000236B6010F034FD18B910F053FD0CF01B
:1001A800BDFE0CF079FF704B704C1A7842F00102DA
:1001B8001A706F4A4FF47001C2F888100022099231
:1001C8000A92226842F4803222600493236803F47E
:1001D80000330A93099B013309930A9B1BB9099BB6
:1001E800B3F5A04FF2D1236813F4003318BF0123ED
:1001F8000A930A9B012B00F089805D4F5D4BFB60E1
:10020800636AAB60636ADFF8A4B1DFF8A481DFF842
:10021800A49143F080736362636943F4FC032EAED8
:10022800636103238DF86A3041F6FF7326F8503D69
:100238004FF09040314604F05FFD4FF6FF734E4893
:10024800ADF86830314604F057FD4C48314604F0AB
:1002580053FD4B48314604F04FFD5846314604F0F3
:100268004BFD3146474804F047FD304608F078FD1D
:100278001A9B454AB3FBF2F3444A1360444B454A80
:100288004FF0000AC3F800A0434B5A60F02287F8E9
:1002980023200722C3F808A0404F1A60D8F8083076
:1002A8003B6099E80F0086E80F0063691A9843F4E9
:1002B80000136361636943F4001363614FF4885367
:1002C800ABF828304FF48843ABF828301BA904F06A
:1002D80013FD1DA91C9804F00FFD642010F0D9F936
:1002E8004FF4A0722E48514615F057F9E3692D4A8C
:1002F80043F00703E361A36943F4E523A36163695A
:1003080043F4BC03636102F5907E55E0264B12224C
:100318001A606368636063686360636843F480635A
:100328006360636823F47C136360636843F4E813D1
:100338006360236843F08073236022680B4B92014B
:10034800FBD55A6822F003025A605A6842F002024A
:100358005A60636803F00C03082BFAD14DE700BF1D
:100368007001002023C80008882D002000100240DA
:1003780000ED00E00005FA05000400480008004808
:10038800000C00480014004840420F007C27002061
:10039800802700203F19010010E000E09829002084
:1003A800C8270020408F01080020024000100048A4
:1003B800BC120020406F0108937B506892F80FC070
:1003C80003F00701DB0800EB83038900186A4FF08C
:1003D8000F0A0CFA01FC0AFA01F120EA010119627C
:1003E800196A10324CEA010172451962E4D10022FF
:1003F800B849002353540132122AF9D1DFF814A363
:100408000AF11E02FF2199540133082BF6D1B24A92
:10041800B24B1360DFF800B3B14A039303211170A4
:1004280058460021242215F0B8F814228BF8002031
:10043800AC49039B3F6801228BF8182098F805B057
:1004480081F800B0A3F5F171CAF82810A649A3F500
:1004580091730B60A54B03EBCB035B78CAF82C3088
:10046800BB0648BFCAF82C200023A14A40F2DC5141
:1004780022F813100133082BF7D113A800211C22EE
:1004880015F08BF8BBF10E0F03D00BF0EF03082B20
:1004980002D101238DF85C30022009F099FB18B1D4
:1004A8004088003018BF0120C7F340038DF8523050
:1004B800C7F380138DF85430C7F340338DF84C30B0
:1004C800C7F3C03300F001008DF84F3017F4006314
:1004D8008DF8510007D098F8843103F1FF3EDEF122
:1004E800000343EB0E038DF85030C7F300438DF83B
:1004F8005530EB6AB8F84401ADF86000003318BF16
:1005080001238DF85630C7F300538DF85730B8F8EB
:100518004631ADF85A30B8F85231ADF8583007F0D6
:100528000101C7F38043C7F3C002FF0448BF714805
:100538008DF85330B8F8503144BFB0F84C01ADF8DD
:100548006000B3F5FA7FADF85E3084BF0023ADF8E4
:100558006030694898F8D43185F83030002385F840
:10056800313043709DF85C308DF84D10002B8DF8BC
:100578004E200CBF0023022301B902B1013309EB5D
:1005880083094FF0000AD9F810309A1E22330392DB
:100598000593039A32F8023F03924FF6FF72934293
:1005A80000F05E81DAB2190A9DF8553033B11301B3
:1005B8005248C058524B984200F04D819DF8523035
:1005C80053B14E4B4F4F03EB02135868B84203D157
:1005D8001B89012B00F03F819DF84F3053B1474BE9
:1005E800484F03EB02135868B84203D11B89042B08
:1005F80000F031819DF8503053B1404B414F03EB2F
:1006080002135868B84203D11B89022B00F02381DA
:10061800022902D19DF84C3003E0012904D19DF84C
:100628004D30002B00F01781344F9DF857304FEABA
:1006380002194F4433B19DF85C301BB9043A032AC0
:1006480040F2F2800129CBB268D1FF2385F87830D7
:1006580085F87930294BC5F8887003EB09024FF00B
:100668000008517B50688DF86A1002F1080B128956
:10067800ADF868201AA9022285F87C8006938DF8C7
:100688006B2085F83480C5F83880C5F83C80C5F8FB
:100698004080C5F8748085F87A8085F87B8004F0FE
:1006A8002BFB069B9BF8021053F80900424604F006
:1006B80077F9384610F096FE134B1449C5F88C307C
:1006C800134BC5F89030C5F8948038460A1D0DF0D4
:1006D80027F8C0E07C010020C81D0020AE140020CF
:1006E80091120020100A0020842900200C9501088E
:1006F80000120020BC120020A1010020408F010838
:1007080000440140000800483D470008FC01002063
:100718001D48000870010020CC1D0020022B49D183
:100728005FFA8AF21C2101FB02FC9D4ACDF81CC02D
:1007380002EB0C089B4A88F87DA0012188F87C1000
:1007480002EB09014FF0000B91F80DE0486888F8BA
:100758007EB001F108020989ADF8681088F886B002
:100768001AA9C8F888708DF86AE006928DF86B307F
:1007780004F0C2FA8B4B069A53F8090091785A464E
:1007880004F00EF9384610F02DFE854BDDF81CC03C
:10079800854AC8F88C2003EB0C01844AC8F89020DD
:1007A8008C31C8F894B038460A1D0CF0B9FF0AF12C
:1007B800010A50E0032B35D19DF85330DFF8E08172
:1007C800DFF820923BB198F832B0384608214FF64E
:1007D800FF7200231AE0BDF85E2098F832B0BDF829
:1007E8006030B2F5FA7F0BD97149B1FBF2F23846A5
:1007F800082192B204F0A9FA6E4B49F82B000AE0DE
:100808006D49B1FBF2F23846012192B204F09DFA2B
:100818006A4B49F82B00C36098F83230013388F8E6
:10082800323018E0042B16D195F83180BDF85820E5
:10083800614B93FBF2F23846BDF85A30012192B26F
:1008480004F083FA95F8313005EB88080133C8F8CD
:100858005C0185F83130039B059A93427FF499AE89
:1008680095F8312085F87C21554A564B92F800E0DE
:10087800AEF117020027022A1F709C461AD8AB6AED
:100888003B44D3ED007AF5EE407AF1EE10FA02D14E
:10089800EB6A63BB26E04C4A07EB02080FCB88E8FB
:1008A8000F009CF8003010370133C02F8CF800304F
:1008B800E5D1EDE7454B13F83E908CF8009003EB3B
:1008C800CE03D3F804A0BAF1000FE1D04F45DFDA28
:1008D8003D4A3B0103EB020853440FCB013788E83C
:1008E8000F00F3E73A4D2B68D80424D41DE0394BA8
:1008F800394A13F83E00107003EBCE035D68002DF3
:10090800F0D000238342EDDAC3EBC3016A18DFF8A5
:10091800D880D2F8009041F8089001EB0807918838
:10092800B9809279BA710133ECE70EF0EF03082B26
:100938002A4B20D122E09CF80020012AF5D9284B27
:1009480003EB0212103210339342EED053ED047AC7
:10095800B6EE007A67EE877A43ED047A53ED057AAE
:1009680067EE877A43ED057A53ED037A67EE877A67
:1009780043ED037AE7E7BEF10E0F09D11A7842F08A
:1009880010021A70BEF1180F30D110F0F7F82DE0F0
:100998001A7822F010021A70BEF1190FF4E700BF9E
:1009A80070010020408F0108A54A0008154700087B
:1009B80000127A003D48000840420F002D48000808
:1009C800100A0020C42700204C0900200C950108BB
:1009D80098290020107D010810290020A41A002061
:1009E80054090020942700201129002010F0AAF8AB
:1009F8002B68BD48DFF82CB359035EBFBB4B0122FF
:100A08001A70049B049A1B7843F0040313706269FC
:100A18004FF408534FF002094FF0010A42F4001254
:100A2800ADF8683031468DF86AA08DF86B90626138
:100A380004F062F9AE4AAF49116000200FF042FE9F
:100A4800A26942F48052A261E26842F48052E260F4
:100A580062694FF0904542F4003262612A6A22F4DA
:100A680070022A622A6A42F4A0022A622A6A22F0E2
:100A780070622A622A6A42F0A0622A622A6A22F016
:100A880070422A622A6A42F0A0422A622A6A22F442
:100A980070222A622A6A42F4A02200272A624FF0B2
:100AA8000308E022284631461A928DF86D808DF8A9
:100AB8006C908DF86E708DF86F7008F0C7FA102280
:100AC800284631461A9205928DF86D808DF86CA0F3
:100AD8008DF86E708DF86F7008F0B8FAE168864D81
:100AE80041F48051E160E16821F48051E16083497B
:100AF800888820F480500004000C8880888880B2A0
:100B080040F480508880088800F4415040F44570D3
:100B180040EA08000880888820F470600004000C0F
:100B280040F4E0608880888B20F40060000407238C
:100B3800000C88830B82088880B240F0400008804F
:100B48006F490D60616941F480216161E16941F497
:100B58000011E161216B21F010012163216B41F04B
:100B680010012163DBF8201021F07061CBF8201010
:100B7800DBF8201041F08061CBF82010DBF8201062
:100B880021F07041CBF82010DBF8201041F08041B3
:100B9800CBF82010402158461A9131468DF86D80C7
:100BA8008DF86E708DF86F708DF86C9008F04EFAB5
:100BB800802158461A91314608F048FA2968514B65
:100BC800514E059A21F00101296028684F490140DA
:100BD80029604F492961296841EA0A012960AF6003
:100BE800EF60AF60A96841F40041A96029682960F5
:100BF800696821F0784121F400416960296841EA77
:100C08000A0129601D680493304605F400633946DB
:100C1800039314F0C2FC049B8DF83C8005F4004B50
:100C280015EA09058DF83D908DF83E708DF83F70F6
:100C380098460DD03748CDF838A00EA908F006FA26
:100C48000622072332707770F37086F802A05546A3
:100C5800BBF1000F0ED004232E480E930EA908F006
:100C6800F5F9082333710723F371012375711D44C6
:100C7800B371EDB2039B6BB1022326480E930EA904
:100C880008F0E4F907233373F373012375731D44E4
:100C9800B373EDB20EA908231E480E9308F0D6F9D7
:100CA8000923337207237572F3720123B3721D444B
:100CB800E36A194823F4F873E362E36A43F4D873E8
:100CC800E362636943F0805343F00103636107F013
:100CD80090FF1AA807F062FF104B1A93EDB2104B61
:100CE8001B93012D20E000BF00100048780E002063
:100CF8009C2D0020F90401080054004000300140F8
:100D0800CC11002098290020201E0020FFE0CF00F1
:100D18007A25E00000080048080002404000005022
:100D2800301E0020000400484FF000030CBF1A4694
:100D380080221F924FF48072BB4C20924FF4806245
:100D480021922022204622921AA94FF400521C9385
:100D58001E9323922493ADF8745007F02CFF236858
:100D680043F0010323604FF0A0440A20A36823F056
:100D78004053A360A36843F08053A3600FF089FC3D
:100D8800A36823F08043A360A368A360A36843F02B
:100D98000043A3604FF0A0418B68002BFADB8B68FF
:100DA800A24A23F040538B608B6843F000538B605A
:100DB80090689F4B034043F468339360CA689D4B27
:100DC800134043F40053CB600A6B013D22F00F023D
:100DD80015430D63002401233219917800296CD042
:100DE8005D1C042B375DD078EDB24FF0A04E0ED8C5
:100DF80003EB43035A00DEF830101F23934021EA27
:100E0800030107FA02F30B43CEF8303031E0092B27
:100E18000ED8053B06225A43DEF834101F239340B0
:100E280021EA030107FA02F30B43CEF8343020E03D
:100E38000E2B4FF006010ED8A3F10A024A43DEF842
:100E480038C01F2393402CEA030107FA02F30B432F
:100E5800CEF838300DE00F3B01FB03F2DEF83CC062
:100E68001F2393402CEA030107FA02F30B43CEF841
:100E78003C30092F4FF0A0420FD99369A7F10A031C
:100E880003EB430397690721994027EA0101916120
:100E980091699840084390610EE053697B1E03EB0B
:100EA800430357693821994027EA01015161516983
:100EB80003339840084350612B460434102C8BD1DF
:100EC8004FF0A042936843F0010393604FF0A043B2
:100ED8001A68D207FAD5DA68574C22F00202DA60AB
:100EE800DA6842F00202DA60DA6842F00102DA6097
:100EF8009A6842F004029A60B4F85831002B40F026
:100F08003187B4F95A21002A40F02C87B4F95C21C2
:100F1800002A40F02787494B494E1B684948B3F8D7
:100F28005630039300210C2294F85FB194F869912C
:100F380094F86A71DFF83CA1434D14F02EFB30465B
:100F48000021142214F029FB00238AF80030C5F888
:100F5800803107F0E5FA002800F0DC863B4B33606F
:100F68003B4B73603B4BF3603B4A3C4B3361012383
:100F780013708AF800300223394A3A4913700B6813
:100F880043F001030B609246374A0023BBF1090F77
:100F9800137001D99B46F7E7012202FA0BF340F2DE
:100FA800B2311940002940F08A8013F0450F0AD168
:100FB8001B0740F184800023C5F8803107F0B0FAA0
:100FC80000287CD00DE0192027211AAB03F0AAFFD6
:100FD8000028F0D01B4B254A1A60254A5A60062380
:100FE80073E0062168200A460DEB000303F09AFF20
:100FF8009DF86D1001F001029DF86B1001F00101E0
:101008004B0043EA82019DF8692002F001030B437B
:1010180032D05BB2012B01D1002302E0022B36D182
:10102800012385F8843139E00800024000030050AC
:10103800E010FCFF07C0FFFDBC12002010120020CA
:10104800E825002048270020700100207D7B00084B
:10105800897A0008E17800080000002090C1793DF5
:10106800FC000020A01A0020BA2D00207B6B00088D
:10107800256B0008340800200EAB68200C210122E3
:1010880003F050FF9DF8383013F00F0303D103200D
:101098000FF06CFB02E0042BC2D1BDE79C4B9D4ACC
:1010A8001A609D4A5A6095F88421002A0CBF6F2265
:1010B8006E221A72994B01221A70032305E0BBF1C4
:1010C800010F09D94FF0000B5EE7954A8AF8013005
:1010D800136843F002031360042F00F2A080DFE8D6
:1010E80007F003A7680368000A200FF0D2FA7720F8
:1010F800A02101220EAB03F015FF002859D01E21B4
:101108000122772003F08AFF4FF42F600FF0B6FA20
:101118004FF0000BABF160010027C9B202221AABF5
:1011280077208DF868708DF8697003F0FBFE9DF8E4
:1011380069309DF8682043EA02227A4B03F5C371AF
:101148002BF801200BF1020BBBF1100FE2D1B3F821
:10115800942102F47F4EA3F894E102F00F010120DC
:101168003B4627F001022A44B2F88621002A18BF1C
:10117800002017F0010F03D0D2B25340082202E03A
:1011880083EA1223FAE713F4004F18BF83F4C0531D
:10119800013A4FEA4303F6D10137102FE1D14EEA65
:1011A8000102A5F8942120B9C3F30333994200F052
:1011B800BD8595F896B15B4FBBF1000F40F0C8852F
:1011C80014200FF066FA07F297137620D021012237
:1011D80003F0A8FE97F89731582B29D107F5CC735F
:1011E80088211822762003F09DFE31227620F421F2
:1011F80003F014FF012387F896314B4B4B4A9A6052
:101208004B4A5A6045F6D8125A804A4ADA604A4A26
:101218001A614A4AA3F800B05A6100F099BD012F3B
:1012280006D03F4A8AF80270136843F0040313603B
:101238003B4F3B68990702D5354B1B6898470023FD
:1012480085F8B4313E4B4FF47A721A603368984788
:101258003C4A002313709346B9F1000F04D0A9F15A
:101268000202012A00F277854FF0000C0C2061463B
:1012780001221AAB8DF868C0CDF810C003F052FEF9
:10128800B0B19DF86830DDF810C0482B40F0D98522
:101298002D4B2E4A1A602E4A5A6006238BF80030CE
:1012A80003238AF803303B6843F008033B6002E0FD
:1012B800844600F0C6BD94F854310BB1254A13702A
:1012C80094F855310BB1154A137094F856310BB197
:1012D8008BF800303B681A0740D5BDF90C10DFEDDC
:1012E8001E6A642291FBF2F302FB131212B207EE9C
:1012F800902AB8EEE77A07EE903AF8EEE77AE7EE4A
:10130800267AB2EE047A67EE877AC5ED6E7A28E01F
:1013180048270020E57B0008CB7A0008BA2D00207A
:10132800A01A002070010020DC0600201D770008AC
:101338001F77000845790008F7790008217500082B
:10134800B01F0020B42D0020B80600200D7B000837
:1013580063790008340800208988883C0023C5F890
:10136800B831B84B1A7842F002021A70B64A4FF4F4
:10137800884191614FF4885111854FF00A0A9946C6
:10138800B14DAB8A9BB283F48843AB82AB8A9BB2E4
:1013980083F48853AB8219200FF07BF901200FF0FA
:1013A80091F919200FF075F90AF1FF3A00200FF0B2
:1013B80089F91AF0FF0AE3D14FF488532B853B686B
:1013C8004FF4884A1B07A5F828A009D59F4BC5F8F4
:1013D80018A01B6898479E4BA5F828A001221A70F0
:1013E8009C4B9FED9D8A1D68DFED9C8A2B7B00EE50
:1013F800103AB8EEC00A20EE080A0BF035FD984BFB
:1014080083ED000A974B1B8807EE903AF8EEE77ACF
:10141800B7EE007AC7EE277A934BB0EE680AC3EDB1
:10142800007AD6ED047A914B67EE887A0026C3EDF0
:10143800007A2B788E4D07EE903AF8EEE77A8D4BCE
:10144800C7EE277AC3ED007A77EE677A8A4BC3ED49
:10145800007A8A4B83ED027AC3ED008AC3ED018AD4
:10146800874B83ED027AC3ED008AC3ED018A0BF046
:10147800FBFCB0EE408AB0EE680A0BF095FC20EE5B
:10148800006A68EE086A66EE007A7E4BE6EE887AB5
:101498002846FF2120EE087AC3ED007A67EE007A2D
:1014A8001B22F0EE675AD7EE085AE7EE087A28EEC4
:1014B800468AC3ED015AA6EE808AC3ED027A83ED0F
:1014C800038A714B1E7014F068F83B686F4A2E70DF
:1014D800012113F0020F18BF697011701FBF03219B
:1014E80011700221A9705E0748BF1178284641BFD4
:1014F8004D1C15700325455413F00A0F0CD01378B2
:101508000421C154591CC9B205254554D91C0233BC
:10151800DBB211700621C154D8F800108D0641BF06
:1015280013785D1C1570072548BFC5540B0608D5F0
:1015380013780925C5549D1C0133DBB215700A25A3
:10154800C5546579082D01D00E2D04D113785E1C81
:1015580016700B26C65413780C27C754CF0303F113
:10156800010644BF494F0233F6B2167041BF3B70C3
:101578003F4B0E279F554B0741BF13785E1C1670D3
:10158800102648BFC654137812275E1CF6B2C754FB
:101598004F05167008D594F80C722FB13B4F0233E3
:1015A8003B70334B13279F5513781427C7548F0567
:1015B80048BF364F03F10106F6B248BF0233167032
:1015C80041BF3B702A4B15279F55182D0BD1137817
:1015D8001626C6545E1CF6B217278755DE1C023342
:1015E800DBB21670C5540E0341BF13785D1C15702D
:1015F800192548BFC554CD0541BF1378591C117032
:101608001A2248BFC25400219822214813F0C5FF6E
:1016180007F031F81F4B204A1A60204BB4F84E11DE
:1016280019801F4900230B808B701E490A60B4F88B
:10163800962190B21C4921F813000133122BF9D1DD
:1016480034E000BF882D002000100048B8060020B4
:10165800D0060020C820002035FA8E3C000000008B
:10166800C4200020040000207C20002080200020CE
:10167800D9110020DC200020CC200020E020002010
:10168800D0200020B42000203B200020D8110020CA
:10169800241D0020AC0F002044140020B00F0020AF
:1016A800582D00204C2D0020782C00208F4E3368B8
:1016B800D8045EBF8E48B0F89C0108801B0740F133
:1016C800C5808B4B93F89031062B00F2B980DFE888
:1016D80003F004070E3D5877770045F2F05201E019
:1016E80042F6F822834B1A8007F07BF8A7E007EE52
:1016F800902ADFED816A7F4BB8EEE77ADFED7F7ADB
:10170800E7EE267A42F6F82119800023FCEEE77A04
:101718007B4A17EE901A42F823100133122BF7D1A7
:10172800784A79491160794A4020137008F038FBEB
:10173800002800F0858001234FF0070C90F9000085
:10174800734A8DE808104021724B73E0694B42F6EA
:10175800F8221A806B4B704A1A606C4B102240209A
:101768001A7008F01DFB00286AD001234FF0000E04
:1017780090F90000694A8DE8084040214FF4E133B0
:1017880058E05C4B42F6F8221A805E4B644A1A60B5
:101798005E4B082240201A7008F002FB00284FD048
:1017A8000123002790F900005E4A8DE88800402157
:1017B8004FF4E13308F0D0F85B4BC3F8BC013BE0D1
:1017C8004C4ADFF8A0C1DFF8A0E1584F584D594CFA
:1017D800594842F6F82111804C490C22062B0A7010
:1017E8000DD000238CF800308EF800303B701B239E
:1017F8002B700523227003704FF4E1340AE00021B6
:101808008CF800108EF800103970227021214B4C92
:10181800297003703B4B4A4A1A60402008F0C0FA0E
:1018280070B101230025474A90F9000040218DE856
:101838002800234608F090F8003018BF012028B986
:1018480008200BF039FB2F4B3F4A1A6033682F4AA8
:1018580013F4804F1FBF082111702A493B4818BF55
:10186800086042F20101194003F0010003F400543A
:1018780079B1204944F620650D8024B10821117002
:101888002049334C0C6020B10C2111701D4931489E
:101898000860117804395170190640F19E80224879
:1018A800DFF8C8802C4FC0F8C071002421461522EB
:1018B80000F5E270294D88F80140C8F80440C8F8DE
:1018C8000840053F13F069FE20462F6006F09AFC99
:1018D800234B02201B68C8F80C3008F061FA002876
:1018E80046D180200BF0E8FA6FE000BF982900206D
:1018F800BC120020BA080020CDCCCC3F0000B0C4F8
:10190800302C002008000020311D0108C01D0020D7
:10191800B11F0108A08601001D1D0108051F01084F
:10192800051D0108B91E010870010020BC2C00200B
:10193800BE2C0020BD2B0020BF2C002090D003001F
:101948002D1C0108991D0108951D0108651D010838
:10195800851D0108751D0108AE14002030080020FF
:10196800BC290020BE2B0020BD2C00201008002020
:10197800447998F80130C3490C2202FB03125278CB
:10198800A24204D00133DBB2042BF4D9002388F837
:1019980001302B6898F801201B7890F90000002B83
:1019A8004FF00C0303FB021314BF0324012400228D
:1019B8005B7800940192022107F0CEFFB24B1860C9
:1019C80000288ED0012006F01DFCB04B1868B04BE3
:1019D80000F5C5721A6006F0C3FCAE4AAE4B136040
:1019E800AE4AAF4D8033136033680024DA032C709D
:1019F80040F1A8800DF0B4FADFF810C3DFF81083C7
:101A0800CDF810C040F22A3B0127604621465A46CD
:101A18002F7013F0C2FDD8F81430A248A24D43F439
:101A28008023C8F81430436A23F00F034362436AE3
:101A38003B434362022203234FF4807A0CA98DF8BA
:101A4800342003928DF835308DF83640CDF830A02B
:101A58008DF8377007F0FAFAD8F81830039A43F47B
:101A68000033C8F818302B8823F440731B041B0C70
:101A78002B801D23EB620EA92A8560232C8628461D
:101A88006F610E93ADF83E401094ADF84440ADF848
:101A98004640ADF84840ADF84A40ADF83C7007F014
:101AA80021F9AB6943F00803AB616B6C43F4004365
:101AB8006B64D8F814303B43C8F81430A8F57D6837
:101AC800404607F096F81AA807F068F8774B1A937B
:101AD80010231C938023DDF810C01F931AA94FF41C
:101AE80000534046CDF86CC02393ADF874B01E94F3
:101AF800CDF880A021942294249407F05CF8EB6838
:101B080043F40073EB60D8F8003043F00203C8F8E0
:101B180000300BA80D238DF82C308DF82D708DF822
:101B28002E408DF82F700FF03FFC2146604B1A684D
:101B3800604B43F8212001312029F7D102F0FEFF44
:101B480002F0FCFF33685B0554D55B4D5B4BD5F861
:101B580004751F60042008F023F90421C5F808055E
:101B680008F0F8F8564B85F80C0508201F6008F0B7
:101B780017F9544B544C1860082108F0EBF8002171
:101B880085F80D052C22204613F007FD8E2363707F
:101B98004FF07C0AE0234FF07D08E37084F800A042
:101BA80084F82B80494C2C220021204613F0F5FCA8
:101BB8008A2363701020A023E37084F800A084F8BF
:101BC8002B80C5F8107508F0EBF81021C5F814053E
:101BD80008F0C0F885F818052020C5F81C7508F02D
:101BE800DFF82021C5F8200508F0B4F885F82405A9
:101BF80010F020FB3368364A13F4002318BF012382
:101C080013700EF01FFD334B1860334B5A79052AB9
:101C1800194602BF314B4FF4C8721A80304B4FF44B
:101C28007A721A802F4BC8221A802F4A137843F0F1
:101C3800080313702D4A137823F0020313703268D7
:101C480040F6020313406BB1294B2A4A1A602A4B0B
:101C580003221A70294B01221A70294A0023138083
:101C6800284A13808B683360274B01221A7099F831
:101C7800003063F07F0389F800302FB0BDEC068B8D
:101C8800BDE8F08FD06F01085C1F00201012002003
:101C980000100020981F0020D8140020941F002056
:101CA800790E0020000400480044014034440140FB
:101CB800606F01087A0E002070010020941A00203D
:101CC800EC1A0020381B0020BC1A0020F11A002052
:101CD800D82900208C080020BC1200204E200020AB
:101CE800AE2D0020AC2D0020A41A0020B62D002017
:101CF8008C1A002036140020F01A0020F40000206E
:101D0800A0100020A2100020780E00204903002017
:101D180000100240504B3360504B7360504B33619E
:101D280004238AF800300523FFF726B94D4B42F209
:101D380010721A805A804C4A5A604C4A9A604C4A2F
:101D4800DA604C4A1A614C4A5A610327FFF769BAAC
:101D58000427FFF766BAB9F1010F7FF6ACAA9946D6
:101D6800FFF776BA1BB208EE103AB4F95A31DFED34
:101D7800437A434A09EE103AB4F95C31B8EEC88A9E
:101D880008EE903A28EE278AB8EEC99AF8EEE88A63
:101D98000021B0EE480A29EE279A68EEA78A11704A
:101DA8000BF062F8F0EE40AAB0EE480A0AF0FCFF29
:101DB800B0EE408AB0EE490A0BF056F8F0EE409AC1
:101DC800B0EE490A0AF0F0FFB0EE40AAB0EE680A99
:101DD8000BF04AF8B0EE409AB0EE680A0AF0E4FF59
:101DE80060EE2A6A68EE097AF0EE665AE7EE8A5AD9
:101DF800244B29EE2A6A28EE007AC3ED035AF0EE46
:101E0800465A29EEC00AE7EE4A5AE6EE8A7AA6EE64
:101E18004A7A29EE299A83ED010A28EE698A29EE81
:101E2800AA0A83ED009A83ED02AAC3ED045A83ED52
:101E3800058A83ED067AC3ED077A83ED080AFFF772
:101E48006AB8B9F1010F7FF636AA4FF000098BF88E
:101E580000C0FFF709BA00BF196C0008BD6B000885
:101E6800295C8F3DDC06002059790008797A000842
:101E78004F790008697A00082177000835FA8E3C06
:101E88006C000020FC1D0020954A2DE9F04F1568D4
:101E9800944C05F59C4320332DED028B2360924B27
:101EA800196889B011F4804F0592984605D110F051
:101EB8000FF910B92379013323718C4B1F78C7B1FF
:101EC8008B4A1268954240F2DF80013F1F70DBE0C9
:101ED800D9F800308748072D98BF595D864B88BFD1
:101EE80029461B689847032D0BD904EB4505013794
:101EF800E880804BDFF81C921E78FDB2AE42E7D82E
:101F080020E0D9F8002005F10E0302EB830399883D
:101F1800DA880028E9D04FF47A73401A5843531AE4
:101F280090FBF3F040F6C90300F57A70984205DC9F
:101F380040F2EE239842B8BF184601E040F6CA00C6
:101F480080B2D2E70F23277984F82A3094F82B300F
:101F58000193032594F82C30B7FBF5F505EB4505FF
:101F68007D1B0393D9F800300293DFF8B0A1EBB2E0
:101F780004930025B54254DA6049019B31F815B045
:101F88004FEA450953B910F0A3F828B1039B002B79
:101F980008BF4FF0000B01E0DDF804B0029B988AFF
:101FA800584502D8D88A58450ED2E8B210F03AF807
:101FB800032D8346DFBF94F82AE00120A8402EEACB
:101FC8000000D8BF84F82A0010F082F818B14C48F5
:101FD80029F800B021E0049B94F876002AF813B0A1
:101FE80028B9022F15D93F49012081F87600BAF89F
:101FF8000210BAF800000844BAF80410084441492D
:1020080080B229F8010000B2032190FBF1F080B200
:1020180000E058463A4929F8010001350AF1060A54
:10202800A8E794F82A203848384BA2F10F014A4211
:102038004A4184F890206AB1354A1268520109D49D
:102048000268D9689A60521AC82A1DD9012283F8F1
:10205800212019E002689868DA605B68121A9A42CF
:1020680088BF2A4B4FF0000184F82B1088BF83F8F3
:1020780021100025B54207DAE8B20FF0D3FF204B54
:1020880023F815000135F5E7D8F80030DF0405D549
:102098001F4B1B68DE0701D40FF090FD059B1968E4
:1020A8001C4B1868837A002B3AD0013B144D027BF5
:1020B80035F813301AB1C3F53B6308339BB21BB232
:1020C800A3F57A73B3F57A7FA8BF4FF47A7323EA3E
:1020D800E37307EE903A9FED107AF8EEE77A58E04E
:1020E800942D0020000F002098290020542D002056
:1020F800502D0020C01D002008000020060F0020E1
:10210800782C0020780F0020BC290020582D0020B2
:10211800D41100204C2D002000007A442E0F0020FE
:10212800D8F80020150440D5D4F89420934E8A1A84
:10213800002A3ADB01F59C422032C6F89420904AE6
:10214800C07A55798F4A32F8152096F8985001359B
:1021580092B292FBF0F205F00F0086F89800304436
:1021680080F899201A468848185C01330244102BDD
:1021780092B2F8D112B292FBF3F31BB2642BA8BF50
:10218800642323EAE37307EE903A9FED807AF8EE32
:10219800E77AC7EE877A7E4A9FED7E7A67EE877A7E
:1021A800FCEEE77A17EE903A1380D8F800307A4FB1
:1021B80013F4807F00F00981784BDFF8E4919942AD
:1021C80005D999F8022012B9012289F8022099F854
:1021D8000220002A00F0F980714A3E7892F82150D6
:1021E8006A1E554255416F4A1168002DC1F380633C
:1021F800C6F380060193924614BF4FF0000B4FF0D0
:10220800030B99F82020052A00F2D980DFE802F0B4
:10221800034D527584A1002E3AD0D4F8AC00B4F81E
:10222800B0100EF0CAF9012809D15F495F4A096860
:102238001268C988642000FB0122C9F81020019B9C
:102248006BB1594A126812794AB10CF0FBFD0322AE
:1022580089F820204FF47A72C9F81C20D1E7002DA4
:1022680040F0AD80514AD9F8101010684C4A8842A5
:102278000AD902920CF0E6FD029A032182F8201096
:1022880040F6B831D161BCE7012182F82010B8E7E7
:10229800019B4FF4806013B10AF0FEFD01E00AF0E3
:1022A800EBFD0022C9F8102089E0002D46D10CF082
:1022B800C9FDA6E725B1052289F82020012000E004
:1022C800284666B1D4F8AC20D189394A11805180AA
:1022D8009180354909684988D1804FF0020B334A0B
:1022E8001168D9F81420914201D8002E64D147F220
:1022F8003052C9F81C20032221E03A7842F0020249
:102308003A700FF05BFC294AD9F81C1012680A448D
:10231800C9F81820042212E0244A9DB11168D9F89E
:10232800182091424BD9234A12781AB9DAF80020BA
:10233800D30744D43A7822F002023A70052289F889
:1023480020205EE71268D9F81C100A44C9F8182042
:1023580035E01549154A09681268C988642000FBE8
:102368000122C9F810204FF48060002289F820204B
:1023780089F803200AF080FD43E700BF000F002022
:10238800201E0020301E0020990F00200000C842A7
:102398003012002000C07F44B62D0020404B4C0076
:1023A800582D0020D411002008260020BC29002028
:1023B800782C00200300002000287FF422AFBBF116
:1023C800000F02D058460EF097F9924D05F5C470EB
:1023D800B5F84E110EF0F1F8834668B90CF024FDFB
:1023E8008D4BC3F800B0C3F804B0C3F808B08B4BEA
:1023F80000221A605A609A603B785E0736D5D8F892
:102408000030D80632D5864B1B78D9062ED4854B9A
:102418001B7893B195F8E031BBF1000F15D17BB172
:10242800814B1A68D4F8B4309B1A002B08DA0FF0E5
:10243800C5FB7E4B83F8B8B018E0BBF1000F0DD197
:1024480010200EF059F901230EE03BB1764A1268CC
:102458004FF47A7101FB0323C4F8B43094F8B83010
:1024680023B10EF035F9002384F8B830002295F82E
:10247800DEA195F8DF11B5F898E1B5F89AC11346D1
:102488006B4E019636F912009B087045C4BF63F085
:102498007F03DBB201326045B8BF43F04003042A32
:1024A800EED194F8B92061489A4205D190F8BA2043
:1024B800F92A04D8013200E0002280F8BA2084F812
:1024C800B930584B5B4E1A789946E2B93368DA0747
:1024D80008D5BBF1000F16D13B78DB0713D50FF0F9
:1024E800D7F910E03B7858070DD5504B93F82B30AF
:1024F8004BB1514BDB7833B911B10FF05FFB02E000
:10250800BBF1000FF9D094F8BA30484ADFF844B16B
:10251800142B40F0B18099F800301AF1000A18BF66
:102528004FF0010A6BB392F8B9305F2B11D13B78A9
:1025380003F0040303F0FF0113B10FF03FFB08E0C1
:102548000B20039102920EF0D7F8029A039982F8B1
:10255800BA10BAF1000F14D094F8B9307D2B10D10D
:102568003B7803F0040303F0FF0213B10FF026FBDE
:1025780007E00B2002920EF0BFF82C4B029A83F86A
:10258800BA203B7803F0040303F0FF01002B73D15A
:1025980094F8B930254A572B16D1284B4FF47A7244
:1025A8001A80D8F80030190601D505F03BFF244BF6
:1025B8001B685A0742BF234A0A21118013F00803F7
:1025C8005AD1214A138057E0D8F80000400716D5A1
:1025D8005A2B14D11D4B187820B119701C4B0122AD
:1025E8001A7049E092F8BB3083F0010382F8BB30DF
:1025F8000BB10C2000E00D200EF07EF83CE05D2BC6
:1026080000F029855B2B00F028855E2B24D1032060
:1026180000F024BDBC120020B41F002010200020B0
:10262800A41A002003000020BC290020000F00206D
:10263800782C0020D4110020582D0020AE2D002029
:10264800A01A0020AC2D0020AC1200207920002018
:102658007A20002010120020562B01D10AF0CCFE5F
:1026680099F80030002B00F00E8594F8B9306F2BE4
:1026780040F003850FF00CF9D8F80030580732D530
:1026880094F8BB30A3B13B78590711D5019BB3F936
:102698000620B5F898319A420ADD336813F0010331
:1026A80001BFAF4A32211180AE4A08BF82F8BB3061
:1026B8003368DA030AD5AC4B1A782AB9AB4A1278D0
:1026C80012B9A74A3221118001220BE0A74A1378D8
:1026D8004BB13B7803F0040303F0FF011BB9A44B93
:1026E800117001221A70DBF800A0002333600AF190
:1026F8007B090AF1CB0B99F8002099F8013019F8F9
:10270800010C9A420BD249460DF020FF38B119F856
:10271800022C012303FA02F233681343336009F1F0
:102728000409D945E7D1934B1B7853B1924B934E8B
:102738001A68DFF860A212F0020F994640F042834F
:1027480039E30AF1CA060AF589793278737816F8F6
:10275800010C9A4225D231460DF0F8FE08B3B37841
:1027680096F804E0864A96F803A07E480C21013BBF
:1027780001FB0E4103EB43031344D1F8C0209A42F6
:102788000FD0C1F8C030002390F8EC20C1F8C43055
:10279800012303FA0EF322EA030381F8BCA080F8B0
:1027A800EC3006364E45D0D1764B1E68764B1B680A
:1027B800039394F82B300493744B029300230193F2
:1027C800029B1B68002B00F0EB8293F800A0BAF183
:1027D800000F00F0E582029A039952688A1A002ACB
:1027E8000CDB01F5FA7202994A60019901228A40CC
:1027F80094F8EC1021EA020284F8EC20049A002AEA
:1028080000F0CE82029A597812F8042C0432D2B21F
:10281800002940F084825E4931F91210B5F89621FA
:1028280002F1C800814202DD93F802B015E0C83A0F
:10283800914203DA9978C1F1000B0EE0019A012365
:10284800934094F8EC2022EA030384F8EC30039BCD
:10285800029A03F5FA735360A2E294F8EC30019AF5
:102868001341DB0700F19C82BBF1000FCCBF0220B3
:1028780001200DF063FF0AF1FF33DFF8E890132B16
:1028880000F28682DFE813F01400250037004B00C1
:1028980064008E00F1005401BB01E90119028402B1
:1028A8004B005A008E00F1005401C30026018B0131
:1028B80096F80090D944B9F1FA0FA8BF4FF0FA0979
:1028C80029EAE979304686F800900DF025FE0120C6
:1028D8000FE096F80190D944B9F1640FA8BF4FF002
:1028E800640929EAE979304686F801900DF014FE6A
:1028F80002204946DEE196F803A0DA44BAF1640FF3
:10290800A8BF4FF0640A2AEAEA7A86F803A030469C
:10291800D9F8F01007F04CFA03205146CAE1717952
:1029280059446429A8BF642121EAE17171710D201D
:102938000DF074FEBAF10D0F00F02A823179594476
:102948006429A8BF642121EAE17131710E20B1E147
:10295800B179594481F30801B1710520AAE100BF9A
:1029680060200020000F002078200020792000201F
:102978007A200020B92D0020D4110020A01A0020B0
:10298800CC73010834120020BC290020C00F00209D
:10299800782C0020681B002000007A440000C84200
:1029A80000000000D9F8F4301A78022A20D107EE86
:1029B80090BAB8EEE70A5FED077A93ED097A80EEF0
:1029C800270A30EE070AB5EEC00AF1EE10FA07D46E
:1029D800B4EE670AF1EE10FAC8BFB0EE670A01E07C
:1029E8001FED110A83ED090A0F200DF001FE0AE020
:1029F80099785944C829A8BFC82121EAE17199707A
:102A08000F200DF00BFEBAF10F0F00F0C181D9F8BD
:102A1800F4301A78022A1ED107EE90BAB8EEE78A87
:102A28005FED227A93ED080A88EE278A38EE000ACD
:102A3800B5EEC00AF1EE10FA07D4B4EE670AF1EE6B
:102A480010FAC8BFB0EE670A01E01FED2B0A83ED4C
:102A5800080A122056E159785944C829A8BFC82144
:102A680021EAE1715970122024E1D9F8F4301A787A
:102A7800022A20D107EE90BAB8EEE70A5FED397A5C
:102A880093ED0C7A80EE270A30EE070AB5EEC00AFD
:102A9800F1EE10FA07D4B4EE670AF1EE10FAC8BFE7
:102AA800B0EE670A01E01FED420A83ED0C0A102020
:102AB8000DF09EFD0AE0197B5944C829A8BFC8211A
:102AC80021EAE171197310200DF0A8FDBAF1100F79
:102AD80000F05E81D9F8F4301A78022A1ED107EE88
:102AE80090BAB8EEE78A5FED537A93ED0B0A88EE59
:102AF800278A38EE000AB5EEC00AF1EE10FA07D4BC
:102B0800B4EE670AF1EE10FAC8BFB0EE670A01E04A
:102B18001FED5D0A83ED0B0A1320F3E0D97A5944BF
:102B2800C829A8BFC82121EAE171D9721320C1E0E0
:102B3800D9F8F4301A78022A22D107EE90BA1FED9C
:102B48006A0AF8EEE77A87EE800AD3ED0F7A30EE5C
:102B5800270AB5EEC00AF1EE10FA09D45FED717AD2
:102B6800B4EE670AF1EE10FAC8BFB0EE670A01E0EA
:102B78001FED750A83ED0F0A11200DF039FD0AE0EB
:102B8800997D5944C829A8BFC82121EAE1719975DE
:102B980011200DF043FDBAF1110F00F0F980D9F8BA
:102BA800F4301A78022A20D107EE90BA1FED860A6F
:102BB800B8EEE78A88EE008A93ED0E0A38EE000A2E
:102BC800B5EEC00AF1EE10FA09D45FED8C7AB4EED6
:102BD800670AF1EE10FAC8BFB0EE670A01E01FED10
:102BE800900A83ED0E0A14208CE0597D5944C829B7
:102BF800A8BFC82121EAE171597514205AE0D9F813
:102C0800F4301A78022A1ED107EE90BAB8EEE78A95
:102C18005FED9E7A93ED0A0A88EE278A38EE000A5D
:102C2800B5EEC00AF1EE10FA07D4B4EE670AF1EE79
:102C380010FAC8BFB0EE670A01E01FEDA70A83EDDE
:102C48000A0A09205EE0D9785944C829A8BFC821D2
:102C580021EAE171D97009202CE0D9F8F4301A780A
:102C6800022A1ED107EE90BAB8EEE78A5FEDB57A70
:102C780093ED0D0A88EE278A38EE000AB5EEC00AF1
:102C8800F1EE10FA07D4B4EE670AF1EE10FAC8BFF5
:102C9800B0EE670A01E01FEDBE0A83ED0D0A0A20B7
:102CA80030E0597B5944C829A8BFC82121EAE171FD
:102CB80059730A200DF0B2FC6AE0D9F8F4301A789A
:102CC800022A22D107EE90BA1FEDCD0AB8EEE78AA4
:102CD80088EE008A93ED100A38EE000AB5EEC00AB5
:102CE800F1EE10FA09D45FEDD37AB4EE670AF1EE8B
:102CF80010FAC8BFB0EE670A01E01FEDD70A83EDEE
:102D0800100A0B200DF074FC42E0D97D5944C82903
:102D1800A8BFC82121EAE171D9750B20CAE70129AA
:102D280036D19878B84B33F91230B3F5617F05DBAB
:102D380040F633029342A8BF134601E04FF4617393
:102D4800BAF10C0F24D14FF4966292FBF0F0AF4A1F
:102D5800A3F5617393FBF0F35FFA83F913784B459E
:102D680016D0B9F1040F34BF4B4602231370A84A9A
:102D78000AFB035303F2A67313600AF069F950467D
:102D880049460DF04BFC09F10100C0B20DF0D6FC2C
:102D9800019A0123934094F8EC20134384F8EC3013
:102DA800019B01330193029B0C330293019B042B7B
:102DB8007FF406ADBAE4D8F80030D80510D5954BA5
:102DC800DB786BB1336899070AD5BAF8003013F08D
:102DD800010B0AD10CF028F801200AF05DF804E094
:102DE80001200AF049F8012300E00023D9F8002067
:102DF80052070DD563B101200AF03EF8BAF8003049
:102E08009B0708D40CF010F802200AF045F802E0FD
:102E180002200AF031F8BAF800307F4A13F0030FA5
:102E28004FF4884114BF91611185326812F00A0F7E
:102E380027D0D9F80020D00609D559070AD404208C
:102E48000AF02AF8754B1B88A4F8F83002E0042031
:102E58000AF012F8D9F800309A0607D5BAF8003007
:102E68005B0606D440200AF017F802E040200AF07A
:102E780003F8D9F80030580642BF684B1B88A4F8FD
:102E8800FA303368990609D4D9F800301A0540F1A8
:102E980091804FF4807009F0FFFF8FE0604B1B7842
:102EA8009B0753D55F4B1B78042B4FD9D9F80030BB
:102EB80013F4007B0FD0BAF80030DE063AD41020A5
:102EC80009F0EAFF202009F0D7FF5748011D05F057
:102ED800FDF902232AE0BAF8006006F01006B6B23F
:102EE8002EB1102009F0C8FF012684F8FCB0D9F8EB
:102EF8000030580512D5D4F800314C495A89B1F937
:102F08000030002BB8BF5B42934207DAB1F90230B8
:102F1800002BB8BF5B429342C0F2F780BAF800308A
:102F2800990608D5202009F0A7FF002384F8FC3073
:102F3800012600E0002694F80431BBB90E200DF0FC
:102F4800DBFB3B4B012283F804210FE0BAF8003089
:102F580003F03003002B97D0102009F08DFF2020BC
:102F680009F08AFF002384F8FC3001E0002E8BD0A2
:102F7800304B002003F1280603F150042E4A0021AB
:102F880022F810102D4A596022F81010043271608E
:102F980022F8101000221A609A603260B260226033
:102FA8006160A26014331436143400287FF46CAFC7
:102FB8000120E3E74FF4807009F05EFF6B79082B7E
:102FC80001D00E2B02D1402009F056FFD8F800306E
:102FD8005A0540F1B08095F80C321BB93B7813F0D4
:102FE800040F03E0D9F8003013F4002F2AD0144B53
:102FF80000221A703C2005F03DFC002800F09B8060
:103008000CF06CFFF6E700BF782C00202827002082
:1030180034120020582D002000100048AC12002067
:10302800A41A0020AA1A00203C120020B412002082
:10303800000F002008100020B02D00208010002074
:10304800C51D00200FF0F6F809B0BDEC028BBDE8F5
:10305800F04F05F010BB012000E002205FFA80F974
:1030680009F1FF3385F8A43709F058FF0AF014F87E
:1030780048460DF063FBFFF7FFBABAF1000F02D024
:103088007E2B3FF4F7AA94F8B930972B05D12C4B37
:103098004FF4C8721A80FFF7EFBAA72B06D1294A56
:1030A800137843F004031370FFF7E6BA0022BB2B32
:1030B800079201D1022303E0B72B04D14FF6FE7328
:1030C800ADF81E300AE0BE2B01D1022304E0BD2B6F
:1030D8007FF4D2AA4FF6FE73ADF81C30DBF800304F
:1030E800BDF81C10B3F858200A44A3F85820BDF8BE
:1030F8001E10B3F85A200A44A3F85A200AF07CF9A3
:10310800002384F8BA30FFF7B7BABAF800309B0644
:103118003FF511AF202009F0BFFE0B480B4B011DF6
:103128001A685B684360026005F0D0F8084B012616
:1031380083F8FC60FFE609B0BDEC028BBDE8F08FB8
:103148004E200020A41A002044120020AC1A0020AF
:10315800000F00202DE9F04FC14BB3F90610C14B09
:103168002DED028B1F687A8985B0914201930EDBA1
:10317800B1F5FA6FFC79BDBF8B1A6343A2F5FA6407
:10318800C4F16404BCBF93FBF4F4643400E0642429
:10319800B54BB64AB3F896B193F95E31126802920C
:1031A8009BB2154603930022AD4B33F912E0CBEBEB
:1031B8000E0303F2F31640F2E63086424FEA420C61
:1031C80003D8002BB8BF5B4201E04FF4FA73022A20
:1031D8002ED0029E96F811611EB1B342CCBF9B1B44
:1031E8000023A34E6FF0630A642093FBF0F836F8CF
:1031F80018900AFB083A08F1010836F918600FFA26
:1032080089F8C8EB060606FB0AF696FBF0F699481D
:103218004E4420F80C60BE18642036797343964EED
:1032280093FBF6F364339BB2634393FBF0F02DE01A
:10323800029890F812611EB1B342CCBF9B1B0023C9
:10324800DFF860926FF06308642093FBF0F008FBEE
:10325800003A39F910600130002B39F91000A0EB61
:10326800060000FB0AFABDF80C009AFBF8FAC6EB58
:103278000A0A1AFB00FA7F48A0F804A0B879B8BF78
:103288005B4243437C4893FBF0F064306B787B4EA1
:103298004FF06408434393FBF8F3B354784EEB7A4A
:1032A800434393FBF8F3B3546B7D724E5843754B0D
:1032B80090FBF8F0022A9854734B0ED1DE4583F840
:1032C80002800DDB684CB4F89821914214DBB1F50B
:1032D800FA6FA8BF4FF4FA610FE0DE459C5404DA98
:1032E80036F80C305B4226F80C300132032A05F11F
:1032F80001057FF459AFE5E71146DFF8BCE15D4D04
:10330800891A4FF47A736FF063075943C2F5FA626A
:103318006423B1FBF2F191FBF3F23EF8120007FBD4
:103328000211013207B23EF91220D21B514391FB20
:10333800F3F30344F380554B1B885F0635D5544B94
:10334800544A1B881288DFED547A9B1A1BB208EE88
:10335800103AB8EEC88A28EE278AB0EE480A09F073
:1033680083FDF0EE408AB0EE480A09F01DFDB5F97C
:10337800023006EE903AB5F90030F8EEE66A07EE4C
:10338800903A20EE667AF8EEE77AA7EEA87A67EE2A
:10339800807ABDEEC77AE6EEA87A17EE103AFDEE0F
:1033A800E77A2B8017EE903A6B803C4D2B68980794
:1033B80040F1A1803A4B3B4F1A687B6945F20721DF
:1033C800D31A8B4240F397807A6105F017FF364B8A
:1033D800DFF8E8901A78032A9846B9F8003022D125
:1033E8000A2B2AD90023282088F800300DF051F93B
:1033F80005F004FF2D4B18880EF0FEFD2C4B1A68C3
:10340800D37890FBF3F0013008282A4BA8BF082096
:103418001870537980B213FB00F33B83137913FBC5
:1034280000F0788309E00A2B07D80323214A88F89B
:103438000030002313703B837B8398F800301A4ACE
:10344800012B3DD002D3022B4CD054E03A8BB9F873
:1034580000309A424FDD012388F8003040E000BF79
:10346800782C002034120020BC12002010120020FA
:103478006C270020B41200200CFEFFFF242000203F
:103488009610002038200020A01F0020681B002074
:10349800AC120020FA0F002035FA8E3C9829002043
:1034A800942D002088100020F01A0020381E0020DB
:1034B8008C1A0020F40000203A1F0020901A0020E7
:1034C800B9F800107B8B8B4202DD022313700FE0EA
:1034D800A34B1B8B0133994202DD002313700AE0D2
:1034E800082006E07B8BB9F8002001339A42B2DC51
:1034F80007200DF001F92D68290577D5994B984FCC
:103508001A68FB69C3EB020845F2072398456DDD8D
:10351800954BB6F906B0D3F80090FA6199F80A30DD
:10352800B4F84E11914E012B4FF47A70ABF57A7BBB
:1035380098FBF0F803D042D3022B20D041E08C4B0B
:10354800396A5A7B8B4B33F812204FF0080E92B22F
:1035580091FBFEF3C91A8B18BA843B6240F6E44229
:1035680093FBFEF39BB25343B9F80820C2EB133325
:103578005843B9F9063090FBF3F0306021E07E4BF8
:10358800B9F808A01B78C6F800A05A0719D57B48D7
:103598000DF013F820B915F0100F18BF4FF0000BFD
:1035A80032220BFB0BF393FBF2F3B9F906205B44D1
:1035B8005A434FF47A7392FBF3F3534400E0002329
:1035C8003360D7E90A0133686D4A03FB08F84FF402
:1035D8007A7398FBF3F810EB080041EBE8710023CD
:1035E800C7E90A010FF048F9664B1860664E336860
:1035F800DB0427D52F0622D5644B1B789D071ED5E3
:10360800634B187804281AD90022624BD718052171
:10361800951C4FF00A0E122AD154E9B287F801E03E
:1036280004D0B0EB510F2A46EFD800E014215A1805
:10363800322002F8010CFF225A540F2000E00A2021
:103648000DF05AF8544D2A68002A50D0534B544F65
:10365800186839688142984649D8524BDFF850912A
:1036680019785268E1B94FF0010A83F800A0B9F857
:103678000030D35C23B350460DF024F84A4B83F84E
:1036880000A00EF031FDB9F80030CBB92B681B78DB
:10369800053B534514D80CF0D5FF444B18600FE098
:1036A8004FF0000A83F800A0B9F80030D35C3BB1B2
:1036B80050460DF007F83C4B83F800A00EF014FDBF
:1036C8002A68B9F8003052683948D25CFE2A01D11C
:1036D80000230BE0FF2A02D10CF0FAFF07E0D8F82C
:1036E80000500A2111FB02523A6001330380224D37
:1036F8002B78580704D52F4B4FF488529A6171E004
:103708003268D1075CBF43F001032B701F4B1B7855
:103718001F075EBF2B7823F001032B70D60248BF2A
:103728002B78214A44BF23F001032B70224B1B68DE
:1037380013F0040F02D02149098851B9204909889A
:1037480009B1980705D41F4B1B88003318BF012304
:10375800D3B3022313702B7823F001032B7038E0C6
:1037680088100020942D00208C1A0020981A002020
:10377800201E0020301E0020B62D002044140020FA
:10378800407E05009C1A0020D4110020A41A0020B5
:10379800AA1A00205427002090270020BC290020C6
:1037A80088270020842700207C2D0020742B0020EF
:1037B8008C27002000100048A01A0020AC2D002003
:1037C8004E200020AE2D00202978C90758BF0223BB
:1037D80013700CF037FFB24B1B68C01A002801DBCE
:1037E8000EF082FC0EF026FDAE4B1E789846002E99
:1037F80000F0A980AC4E3368002B00F0D786306803
:103808000DF00FF8002800F0D186A74BA74C1868D8
:103818000DF004F8092801D03F2850D14FF0000AD4
:10382800D4F80090A24D5746B9F1000F05D0A14831
:1038380029684A4611F0FEFE10B9AA4607B92F4674
:103848009D4B10359D42EFD3C7B1D7F800E0DAF8A9
:1038580000C023681EF803501CF80300A8420DD1CD
:103868005A1C944938B92D2B05D8904D2A6020252B
:10387800CD54885402E0CD542260EAE723680BB1A6
:10388800574511D08D480CF01DFC574507D857F8FF
:10389800100B0CF017FC09200CF00CFCF5E788481D
:1038A8000CF010FC4FF0000923689945A7D2814B12
:1038B80013F809000CF0FEFB09F10109F4E723688D
:1038C800002B40F05786042840F09986794807F085
:1038D80089F900F06BBED9F80000DFF8F4A10CF00C
:1038E800A0FF30B3DAF800000CF098FFDBF80030E6
:1038F80093F848100246002933D124286AD10122BE
:1039080083F84820DBF80030DFF8C0A193F848209E
:10391800062AE0D193F8490001F0EEFB002800F0F8
:1039280083803B6898790CF016FB3B68002283F88B
:103938004820644B93F83530002B40F0FB854C361B
:10394800982E00F03386604BF21892F84A1001293D
:10395800F5D15E4FF3583A605D4ABB461360914615
:10396800B9E7012904D14D2814BF00220222C7E774
:10397800022904D13C2814BF00220322C0E70329EE
:103988000CD140284FF0000102D983F84810B9E75C
:1039980058711971D97198710422B1E7042906D1B7
:1039A800997983F849004A409A710522A8E70529C0
:1039B800A8D1587919798842987906D950409871D0
:1039C800481C18710B441A729CE790420CBF0622DF
:1039D800002295E72B783F49580793D4232ADAF831
:1039E800003014D1012088F800002F4803910360AB
:1039F80034480292036338480CF064FB30480CF0FA
:103A080061FB0399029A0B7843F002030B70334B66
:103A18001B681B78934201BF314B324A1A60324B04
:103A280004BF324ADA606DE7DAF8002092F84930CC
:103A38004C2B00F08A8478D8332B00F0C18421D82D
:103A4800292B00F04E8409D8252B00F02584272B3C
:103A580000F02984232B40F0CE8541E22D2B00F085
:103A6800518407D82B2B40F0C6850CF057FA6071AB
:103A780000F05BBD2F2B00F01085312B00F0228564
:103A880000F0B9BD3C2B00F00D8131D8372B00F088
:103A9800CC84392B00F01484352B40F0AC855AE2E5
:103AA800802D0020B92D002044270020901F0020E1
:103AB800087B0108601F0020B87C01088393010877
:103AC8008893010888100020241D0020481B00202E
:103AD8004C1B0020B62D0020B8930108C81D0020FB
:103AE800FC9F0020EFBEADDE00ED00E00400FA050B
:103AF800412B00F06A840CD83E2B40F07C850CF0FA
:103B08000DFA84F8E0010CF009FA84F8DF0100F0FE
:103B18000CBD432B00F06684442B40F06C85E94BC8
:103B2800012283F8352000F000BDD02B00F00A8375
:103B380055D8CA2B00F0C58009D8C82B00F085805D
:103B480000F221834E2B00F00D8400F054BDCD2BE4
:103B580000F0038304D8CC2B00F0258200F04BBD85
:103B6800CE2B00F00383CF2B40F045850CF0E0F915
:103B78006FF4AF6283189BB2C62B98BFA4F8960166
:103B88000CF0D6F9A4F840010CF0D2F9A4F84201DF
:103B98000CF0CEF9A4F844010CF0CAF9A4F8D80145
:103BA8000CF0BCF984F8ED010CF0B8F90CF0B6F99A
:103BB80084F8EE010CF0B2F984F885010CF0AEF946
:103BC80084F892010CF0AAF9BF4BD3F800900CF0DE
:103BD800AFF900EB80004000A9F8560070E3D62B3F
:103BE80000F034820AD8D22B19D0C0F0F382D32B3C
:103BF80025D0D42B00F0368200F0FDBCEF2B41D04D
:103C080005D8D82B40F0F7844FF0000AEBE0F22BF0
:103C180000F07082FA2B00F0B28200F0ECBC2B7836
:103C2800590700F182840CF079F9022884F8A40776
:103C380040F28E82A54B002283F8A42788E20CF07C
:103C480077F9A34B188000F070BC92F805904FEA02
:103C58005909B9F1120F03D904F008FE00F065BC48
:103C68004FF0000ACA4507D20CF062F9994B23F8C5
:103C78001A000AF1010AF5E7924B012283F8342071
:103C880000F053BCDFF84092D9F800A00CF050F9CE
:103C9800AAF85A00D9F800900CF04AF9A9F8580087
:103CA80000F043BCDFF82092D9F800A00CF036F9F8
:103CB8008AF80000D9F80030187808F00DFD00F0F7
:103CC80034BC814B1A681278022A824699466FD111
:103CD800D9F800B00CF022F907EE900AF8EE677AEE
:103CE800B2EE048AC7EE887A0BEB8A0BCBED087A22
:103CF800D9F800B00CF012F907EE900A9FED767A29
:103D0800F8EE677A0BEB8A0BC7EE877ACBED0B7A66
:103D1800D9F800B00CF002F907EE900A9FED6F7A1F
:103D2800F8EE677A0BEB8A0BC7EE877A0AF1010A7D
:103D3800BAF1030FCBED0E7ACAD1BAF1070FD9F851
:103D480000B01CD10CF0EAF807EE900AF8EE677A9A
:103D5800C7EE887ACBED117AD9F800B00CF0DEF80E
:103D680007EE900AF8EE677AC7EE887ACBED127AFA
:103D7800D9F800B00CF0D2F88BF84C0012E00CF037
:103D8800CDF8D3448BF80100D9F800B00CF0C6F890
:103D9800D3448BF80B00D9F800B00CF0BFF8D3442B
:103DA8008BF815000AF1010ABAF10A0FC5D1BCE374
:103DB800D9F800B00CF0B2F8D3448BF80100D9F868
:103DC80000B00CF0ABF8D3448BF80B00D9F800B076
:103DD8000CF0A4F8D3440AF1010ABAF10A0F8BF8DF
:103DE8001500E5D1A1E3DFF8E0909FED3C8AD9F812
:103DF80000B00CF09DF807EE900AF8EE677A0BEB2E
:103E08008A0BC7EE887ACBED087AD9F800B00CF0A7
:103E18008FF807EE900AF8EE677A0BEB8A0BC7EE7D
:103E2800887ACBED0B7AD9F800B00CF081F807EE60
:103E3800900AF8EE677A0BEB8A0BC7EE887A0AF1DC
:103E4800010ABAF1030FCBED0E7ACCD1BAF1070F04
:103E5800D9F800B01CD10CF06BF807EE900AF8EE18
:103E6800677AC7EE887ACBED117AD9F800B00CF0F2
:103E78005FF807EE900AF8EE677AC7EE887ACBED1E
:103E8800127AD9F800B00CF053F88BF84C0012E015
:103E98000CF04EF8D3448BF80100D9F800B00CF0C0
:103EA80047F8D3448BF80B00D9F800B00CF040F871
:103EB800D3448BF815000AF1010ABAF10A0FC5D1EB
:103EC80033E300BF8810002010120020BC1200202D
:103ED800F80F0020782C00200000C84200007A4427
:103EE8000CF01CF8132883463FF6B6AEDFF84CA357
:103EF800DAF800900CF012F80023CB4A0C2101FBF1
:103F08000322117A814222D10FFA8BFB09EB8B092C
:103F1800137889F879300CF001F889F87A000BF0F9
:103F2800FDFF89F87B000BF0F9FFC04BC04A1A600F
:103F380089F87C00BF4BDAF800001860002179305E
:103F48000CF02AFBBC4B80F001001870EDE2013345
:103F58001C2BD2D180E60BF0E1FF0B2882463FF6FE
:103F68007BAEB64BD3F800900BF0D8FF03283FF692
:103F780073AE062303FB0A9989F8CE000BF0CEFF37
:103F880089F8C9000BF0CAFF89F8CA000BF0C6FF10
:103F980089F8CB000BF0C2FF89F8CC000BF0BEFF0C
:103FA80089F8CD00C1E25379092B7FF655AE019B04
:103FB800D3F800900BF0B2FF019B89F80000D3F80A
:103FC80000900BF0ABFF89F801000BF0A7FF019BF5
:103FD80064281B68A8BF642018710BF09FFF019B21
:103FE80064281B68A8BF642058710BF097FF019BD9
:103FF800FF281B68A8BFFF2098710BF08FFF019B5B
:104008006428D3F8009028BF642089F807000BF0D3
:1040180085FF019B89F80200D3F800900BF07EFF22
:10402800019B89F80300D3F800900BF081FF3B68EF
:10403800A9F80A005B790A2B40F27782804BD3F803
:1040480000900BF06BFF89F808006EE282460BF0D7
:104058006FFF7C4B23F81A000AF1010ABAF1080F26
:10406800F5D162E253790F2B7FF4F6AD0BF056FFD2
:10407800072881463FF6F0ADDFF8C0A1DAF800B0B6
:104088000BF056FF0E2303FB09F9CB44ABF81901DB
:10409800DAF800B00BF04CFFCB44ABF81B01DAF8B0
:1040A80000B00BF045FFCB44ABF81D01DAF800B0C7
:1040B8000BF034FFCB448BF81F01DAF800B00BF09B
:1040C8002DFFCB448BF82001DAF800B00BF026FF67
:1040D800CB448BF82101DAF800B00BF01FFFCB447A
:1040E800DAF800A08BF822010BF02CFFD144C9F8B4
:1040F80023011AE20BF012FF0F2881463FF6ACAD00
:104108000BF00CFFC9EBC909A14489F8D0000BF0EA
:1041180005FF89F8D1000BF001FF89F8D2000BF0F8
:10412800FDFE89F8D3000BF0F9FE89F8D4000BF0F6
:10413800F5FE89F8D5000BF0F1FE89F8D6000CF0F1
:104148001DFDF2E12B785B0700F1EF810CF07AFDA1
:1041580008F0E4FE08F0A0FFE7E12B78580700F12B
:10416800E481394B4FF4C8721A80DEE12B78590785
:1041780000F1DB81354A137843F0040328E02B78FB
:104188005A07E5D537E20BF0C9FE304B1A7810B163
:1041980042F0020201E022F002021A700BF0BEFEA9
:1041A8002B4BDFF8C49018700BF0CCFEC9F8000058
:1041B8000BF0C8FEC9F804000BF0BAFE254B1880B6
:1041C8000BF0B6FE244B254A1880137843F00203FF
:1041D8001370AAE10BF0A2FE02900BF0B3FE834627
:1041E8000BF0B0FE82460BF0ADFE81460BF0A0FE50
:1041F8000BF09EFE0BF092FE029BBBBB184B1020EF
:10420800C3F800B0C3F804A008F036FE0F4A1378CC
:1042180043F001031370B9F1000F00F08681114BD0
:10422800C3F8009081E100BF38740108F00F002046
:10423800FC130020F40F00200300002010120020BF
:10424800341200202A2700204E200020A41A002023
:10425800AA1A0020A81A0020A61A00203A12002044
:104268003C1200204C120020AC1A0020102B40F009
:104278005C81B94BC3F800B0C3F804A0B9F1000FD2
:1042880002D0B64BC3F80090B348B54B0222011DCB
:104298001A7004F01BF848E1A0600BF053FEA36805
:1042A8001843A06041E10BF043FEA4F858010BF05D
:1042B8003FFEA4F85A010BF03BFEA4F85C0134E180
:1042C8000BF02CFE84F87A010BF028FE84F87E01AE
:1042D8000BF024FE84F87D010BF020FE84F87F01AA
:1042E80023E10BF025FEA4F880010BF021FEA4F8D1
:1042F80082010BF013FE84F884010BF019FEA4F878
:10430800860112E10BF00AFE84F890010BF010FE12
:10431800A4F89A010BF00CFEA4F896010BF008FE25
:10432800A4F898010BF0FAFDDAF8003084F891014E
:104338005B79082B40F2F9800BF0FAFDA4F89C0198
:104348000BF0F6FDA4F89E01EFE00BF0E7FD84F812
:10435800D6010BF0E3FD84F8D7010BF0E9FDA4F8D2
:10436800D801E2E092F805900323B9FBF3F9B9F11B
:10437800120F3FF671ACDFF8F8A14FF0000BCB45F8
:1043880080F0D3800BF0CAFD8AF8A0010BF0D0FDB5
:1043980040F2ED23984205DD40F6CA039842A8BFD3
:1043A800184601E040F2EE20A0F2EE2019230BF1AE
:1043B800010B90FBF3F00AF1020A8AF89F01DEE78D
:1043C8000BF0ACFD84F89201AFE082460BF0A6FD3D
:1043D80004EB0A030AF1010ABAF1080F83F888010D
:1043E800F4D1A2E00BF09AFD0023A36060710BF0FA
:1043F800A9FDA3681843A0600BF090FD84F8900114
:104408000BF096FDA4F858010BF092FDA4F85A01A0
:104418000BF08EFDA4F85C010BF08AFDA4F8800176
:104428000BF086FDA4F882017FE053794FF0070A6C
:10443800B3FBFAF2C2EBC2029A1A12F0FF0F7FF432
:104448000BACB3FBFAFA0AF1FF3A5FFA8AFABAF14F
:10445800FF0F6AD00BF062FD5FFA80FB4FFA8BF01A
:1044680005F0B6FB814600283FF4F6AB80F800B0B3
:104478000BF05EFDA9F802000BF050FD89F804006E
:104488000BF04CFD89F805000BF048FD89F8070092
:104498000BF044FD89F80600D5E7DFF8D49009F160
:1044A800400A0BF045FDA9F89C020BF037FD89F88E
:1044B8009E020BF033FD09F1040989F89B02D145EE
:1044C800EFD132E00BF02AFD1F2881463FF6C4AB3E
:1044D8003B685B79082B7FF4BFAB0BF029FD09F132
:1044E800860904EB890900F03F00A9F806000BF0E3
:1044F8001FFDB9F80630800100F4FE501843A9F8F2
:1045080006000BF00BFD000189F804000BF006FD16
:1045180099F8043000F00F00184389F804000BF0F4
:10452800FDFC89F805000AF01BFD00200BF042FD98
:10453800FFF7F7B90B4B98590CF06AF918B9322004
:104548000CF0A7F8F6E70CF0D9FA08F0BDFC064B1A
:10455800064ADA60FFF7F3B9441200204C12002033
:10456800FC0F0020241D002000ED00E00400FA05E7
:10457800BC1200200C2844D00A284BD1534D544873
:104588000BF0A0FD2846232111F03DF808B1401B8F
:1045980020602368002B60D14C4823600021302222
:1045A80010F0FBFF98F80030002B2DD1494B1B6809
:1045B8009B0615D5484B49491B688A6B9A1A002AED
:1045C8000EDB474A1278042A0AD9464A03F5123301
:1045D80003F5F8738B63938A9BB283F488439382C1
:1045E800414B9B68002B6BD0404805B0BDEC028B5B
:1045F800BDE8F04F184704F039F9FFF792B90C28D5
:1046080004D13B480BF05EFD3A480DE07F2812D1FB
:10461800FFF7F5B80D28B1D07F2809D1013B2B4A07
:10462800354823600021D1540BF04CFDFFF7E7B863
:104638002F2B3FF6E4A8A0F12002D2B25E2A3FF663
:10464800DEA813B920283FF4DAA85A1C22601F4AB2
:10465800D0540BF02FFDFFF7D2B85A1EA95C2029C1
:1046680001D1134696E7194A23600021D154234B00
:10467800234DD3F800A0D5F800B0DFF85090584685
:1046880010F0CFFF07463A464846594610F0D2FF89
:104698001C4A28B919F8073053445B785B0703D0E4
:1046A80010359542E7D306E0954204D2781CEB68B2
:1046B8004844984702E014480BF004FD00236BE7D8
:1046C80005B0BDEC028BBDE8F08F00BF601F002075
:1046D8004C9F0108A01A0020942D0020881000206B
:1046E800AA1A002000100048E8250020C410002065
:1046F8008D93010888930108B493010804010020F0
:10470800087B0108B87C01089893010810F80A3C56
:104718000133DBB20A2B84BF10F8131C044A00F8DB
:104728000A3C82BF002322F8113000F80A3C704787
:104738009C2C0020334A136C90681944081A40F6E0
:104748008C23984270B513469160D06051603BD974
:10475800127893F945108A4210460BD1111F082987
:1047680008D893F84610182901D8013103E083F8D6
:10477800442002E0002183F8461093F9444021497F
:10478800A24219D191F84740B4B10C3100249442A7
:1047980006DA1D4D51F8046F25F814600134F6E768
:1047A8000C2805D01849002421F810400130F7E7FB
:1047B800164801780131017083F845200022012153
:1047C8001A7083F8471070BD92F84710C9B1A0F26B
:1047D800EF2440F2DA518C4208D811780B2905D819
:1047E8000B1D0131117042F8230070BD002283F8BF
:1047F8004720074B03F13002002143F8041F93427E
:10480800FAD170BDA40100209C2C00209C06002039
:10481800B0010020024A136C013319441164704737
:10482800A4010020024B53F820301B681960704720
:1048380094270020064B53F820301A681B89A1F5ED
:104848007A7159434FF47A7391FBF3F11160704711
:1048580094270020054B98420CBF054A054A138847
:1048680001339BB213800020704700BF0054004002
:10487800D0110020D2110020F0B5046D866823689D
:1048880023F0010323608379054613F0020F407972
:104898000CBF4FF0000E4FF4005E13F0040F14BF6E
:1048A8004FF48067002710F0010F14BF0421002186
:1048B8008307206820F001002060626822F44052DB
:1048C8004EEA02026260226822F4B05323F00C031D
:1048D80048BF41F008013B430B432360A36895B0F0
:1048E80023F44073A360684604F03AFA284B9C42CC
:1048F80001D10C9B0EE0274B9C4201D10D9B09E096
:10490800254B9C4201D10E9B04E0244B9C420CBFDA
:104918000F9B109B2268A879170448BF5B00B3FB64
:10492800F6F206FB1233B3EB560F236828BF0132A9
:104938001E0441BF4FF6F073C2F34201134041EA2F
:1049480003026B7992B213F0020FA28100F0010109
:1049580014BF4FF400320022DC0748BF42F4803213
:104968002B6D11B159680A4302E0596821EA020225
:104978005A609A6801074CBF42F0080222F0080208
:104988009A601A6842F001021A6015B0F0BD00BFC3
:10499800003801400044004000480040004C0040FE
:1049A8003D4B1B78012B30B514BF00240324B1B94B
:1049B800036A23F0010303628169036A21F0F301AA
:1049C80023F00A0341F0010142F001021A4341EACF
:1049D800041181610262836923F00C031BE004293E
:1049E8001DD1016A4FF6EF730B4003628169056AB6
:1049F800120121F473414FF65F7342F0100241F443
:104A080080712B4092B2134341EA04318161036201
:104A1800836923F4406383618369836130BD082916
:104A2800016A1AD14FF6FF630B400362C169036A3A
:104A38009BB289B223F4206343F4807321F0F3011D
:104A480043EA022241F0010192B241EA0411C16134
:104A58000262C2694FF6F37319E04EF6FF730B401A
:104A68000362C369056A40F6FF41194045F6FF73C2
:104A78002B4043F4805343EA023241F4807192B2EE
:104A880041EA0431C1610262C2694FF2FF33134047
:104A9800C361C369C36130BDA001002038B510F8F7
:104AA8000E2C50F8043C044652B9012200F80E2C92
:104AB80020F80C1C997A18680222BDE838406FE784
:104AC80030F80C2C20F80A1C891A89B220F8081C26
:104AD800074A10F80F0C002522F8101004F80E5C95
:104AE8001868997A2A46FFF75BFF04F8065C38BD18
:104AF8009C2C0020044B53F820301BB107289CBF86
:104B08001B681960704700BFCC020020084A136870
:104B18009B050BD5074B00211970074908684FF60C
:104B2800FE7303400B604FF400735360704700BF7F
:104B380000000240B52D0020300002402DE9F0476A
:104B4800664D2B6866490A78581C02F0FF068E46A7
:104B58000AB10346F6E72B60687BAB6895F80C80D2
:104B6800AA7B374639B2202900F09B80DFF880C144
:104B78000CEB81033CF82110DC789B78C3F1FF0330
:104B88009BB2002B65D0C3F1FF0363434FF03C0C8D
:104B98001B12B1FBFCF9B9F1050F5DD8DFE809F08C
:104BA800030B1A293A4AE01ADAB24143B1FBFCF086
:104BB8001044C0B251E0B1FBFCF00CFB101189B2FB
:104BC800DAB2C1F13C01E31A4B432046B3FBFCFCCB
:104BD80094442CE0B1FBFCF00CFB10115FFA83F855
:104BE800E21A89B24A43B2FBFCF24244D2B22046EE
:104BF80032E0B1FBFCF90CFB191189B25FFA83F8BA
:104C0800E01AC1F13C014843B0FBFCF04044C0B29B
:104C1800224621E0B1FBFCF80CFB1811D8B289B28E
:104C2800E31A01FB03F2B2FBFCFC224684445FFA60
:104C38008CF412E0B1FBFCF80CFB181189B2D8B265
:104C4800C1F13C01E31A4B43B3FBFCF20244D2B27C
:104C580003E02246204600E044464FEA042C4CEA92
:104C6800004C4CEA020C172306F117014FF001081B
:104C780008FA03F8C91A18EA0C0F89B2DFF8748029
:104C880014BF4FF011094FF0090913F1FF3308F869
:104C98000190E9D218360137B6B2BFB2114BA0461F
:104CA80060E7AA73AB60104AE98001238EF80030F0
:104CB8000E4985F80C8040F22A336873AE80536041
:104CC80000234B620B889BB243F001030B801368EF
:104CD80043F001031360BDE8F08700BFC81000204F
:104CE800B52D0020D41000203000024000440140BF
:104CF8007A0E00204903002073B506460D460024AD
:104D080001232A88A34013421AD0AA78009302F0FC
:104D180003038DF80430EB78022B03D0032B0CBF70
:104D2800032301238DF805303046C2F30113694689
:104D3800C2F381028DF806308DF8072004F086F959
:104D48000134102CDCD102B070BD2DE9F04F734E48
:104D5800F57B07460C4687B011469A4600686B1CDF
:104D6800914622464FF0020BF37308F057FC3B893B
:104D78007868ADF8043001A98DF806B08DF807B051
:104D8800FFF7BAFF0023ADF80A30ADF81230ADF8DE
:104D9800163070230193BA7A3C68CDF80CA0012331
:104DA80006F110082D01ADF808304FF48073A844BF
:104DB800ADF810B0ADF814300C2A7ED8DFE802F058
:104DC800077D7D7D0F7D7D7D387D7D7D5E00204664
:104DD80001A903F087FFA36943F0080326E0236ACB
:104DE8004F4823F010032362236A6168A26922F006
:104DF800807222F4E642844242F4E04206D000F592
:104E08000060844202D043F0300307E023F0E0035F
:104E180021F4406143F0300341F480616160A26194
:104E2800C4F838A02362A36943F40063A36144E093
:104E3800236A3B4823F480732362226A6168E3692A
:104E4800844223F0730343F0700306D000F500603A
:104E5800844202D042F4407207E022F4606221F4F6
:104E6800405142F4407241F480516160E361C4F8FA
:104E78003CA02262E36943F008031DE0236A284846
:104E880023F480532362226A6168E369844223F42D
:104E9800E64343F4E04342F4405203D000F5006097
:104EA800844201D141F480416160E361C4F840A0CB
:104EB8002262E36943F40063E3613A7B3B681AB119
:104EC8005A6C42F400425A641A8892B242F00102C3
:104ED8001A80BA7A0C2A18D8DFE802F007171717D1
:104EE8000B1717170F1717171300721903F134014F
:104EF8000AE0721903F1380106E0721903F13C0166
:104F080002E0721903F14001116135444046A5F8E9
:104F180018906B6107B0BDE8F08F00BFC810002083
:104F2800002C0140F8B53A4E3A4C4000C7B24FF455
:104F380020453068C4F8D050D0F818E01EF4004F6F
:104F480005D0AE46013DBEF1000FF5D116E0D0F810
:104F580004E0314D0EEA050545F490353D434560C2
:104F68004FF42045C4F8D050D0F818E01EF0020FD6
:104F78002DD1AE46013DBEF1000FF5D1C4F8D05099
:104F88001FE02946013D0029F8D081694906F8D576
:104F9800C4F8D05020494568294041F0007141F4D7
:104FA800105141EA0241394341604FF42041A2B116
:104FB800306885696D071ED411F1FF31F9D2C4F844
:104FC800D010FFF747FC003018BF0120F8BD4FF4A0
:104FD80020458162C4F8D050D7E73068C4F8D010B3
:104FE8000B46826992060CD41A46013B002AF8D176
:104FF800C4F8D030E5E7416A03F8011B013AD2B2A0
:10500800D3E7C4F8D0302023C3610120F8BD00BF26
:10501800CC110020C8100020009800FC400070B59A
:10502800C5B23248324B00684FF42044C3F8D04030
:105038008669360404D52646013C002EF8D113E0D3
:1050480046682C4C344044F0807444F490342C432B
:1050580044604FF42044C3F8D0408669B60729D489
:105068002646013C002EF8D1C3F8D0401CE021466A
:10507800013C0029F8D081690E06F8D544681D491D
:10508800214041F0007141F48031294341604FF4DF
:105098002041C3F8D0108469A40711D40C46013903
:1050A800002CF8D1C3F8D010FFF7D4FB003018BF9C
:1050B800012070BD4FF420448162C3F8D040DAE784
:1050C80082624FF42042C3F8D0208169890606D451
:1050D8001146013A0029F8D1C3F8D020E4E7C3F813
:1050E800D0202023C361012070BD00BFCC11002057
:1050F800C8100020009800FC2DE9F0474D282DED40
:10510800028B044600F0348600F29480302800F0C8
:10511800CF8651D8222800F06D8423D8032800F0C8
:10512800CC8114D8012800F0BC81022840F0FE860A
:1051380004200AF03FFF43200AF00DFF4C200AF03C
:105148000AFF46200AF007FF4C2000F037BE04286B
:1051580000F0BC81052840F0E9861A200AF02AFFF1
:105168000024DDE1282800F0C28515D8242800F0A5
:10517800A585262840F0DA86DC4C06200AF01AFFBE
:10518800B4F858010AF019FFB4F85A010AF015FFEB
:10519800B4F85C0100F08FBD2C2800F0BB852E28E8
:1051A80000F059862A2840F0C18601200AF002FF43
:1051B800CE4B587900F002BE3B2800F014841AD870
:1051C800362800F029860BD8322800F0F1853428DB
:1051D80040F0AC8648200AF0EDFE002500F02CBC1B
:1051E800382800F071853A2840F0A08604200AF09B
:1051F800E1FE00F096BE422800F0ED850BD83D2870
:1052080000F0B182402840F0918608200AF0D2FED2
:10521800002400F0D6BD462800F06F864B2800F029
:105228009885452840F0828613200AF0C3FE0024A2
:1052380000F06DBE702800F0EB8200F2E58069286E
:1052480000F04C8200F2B680662800F0A68100F2D9
:10525800A680642800F07D81652840F06786A44C0C
:105268000B200AF0A7FE20880AF0A7FE6268A14B6F
:105278009A420CBF2089608980B20AF09EFE9E4B3C
:105288001B68C3F3C000C3F38002800040EA4200F9
:10529800C3F340021043C3F3401240EAC20003F0D4
:1052A800100318430AF089FE944B1A88E368247C9B
:1052B80002F0080103F4475949EA010903F480415F
:1052C80049EA010903F4004149EA010903F480317C
:1052D80049EA010903F4003149EA010903F480218C
:1052E80049EA010903F4002149EA010903F480119C
:1052F80049EA010903F0007349EA0303DFF81C9245
:1053080099F8009012F0010FC9F3800914BF4FF00B
:1053180002084FF0000843EA090312F0020F43EABB
:10532800080314BF4FF0040C4FF0000C12F0040FE8
:1053380043EA0C0C14BF4FF0100E4FF0000E12F0A1
:10534800400F14BF202700274CEA0E0E12F0100F52
:1053580014BF4FF4007600264EEA070712F0200F1C
:1053680014BF4FF4806500253E4312F4807F14BFBC
:105378004FF400600020354312F4007F14BF4FF44F
:1053880000110021284312F4806F41EA000114BF84
:105398004FF080630023002019430346E9E06728A3
:1053A80000F02381682840F0C18510200AF002FE31
:1053B80000248AE16C2800F0A48117D86A2800F03C
:1053C800FF836B2840F0B28505200AF0F3FD4C4BB3
:1053D80018880AF0F2FD4B4B18880AF0EEFD444B92
:1053E80093F8720000F0010000F0E8BC6E28404D10
:1053F80000F0948100F2C28106200AF0DBFD686E9D
:105408000AF0E4FD404B87E1782800F0FB8018D8CB
:10541800742800F032830AD8722800F09183732828
:1054280040F0848508200AF0C5FD0124C1E37628F0
:1054380000F0E68300F25A832F200AF0BBFD334CBC
:10544800C9E2A42800F0038414D87B2800F06982FC
:10545800A02840F06B850C200AF0ACFD2C4B186896
:105468000AF0B4FD2B4B18680AF0B0FD2A4B1868F7
:1054780000F058BDF12800F00181FE2800F00E84EC
:10548800F02840F053851A4C04200AF093FDA36CD1
:10549800B3F85A000AF091FDA36CB3F8580000F075
:1054A8000ABC03200AF086FD00200AF054FD2046BD
:1054B8000AF051FD0D2000F081BC0AF07BFD0120AF
:1054C8000AF049FD0A200AF046FDBEE306200AF06C
:1054D80071FD43200AF03FFD48200AF03CFD4620BC
:1054E8000AF039FD33200AF036FDE3E3BC12002050
:1054F800C811002000540040A01A0020681B00209A
:105508001E1B0020201B0020A41200200774010885
:10551800ACF7FF1FB0F7FF1FB4F7FF1FB62D002031
:10552800AA4B185D01340AF016FD0B2CF8D10024A3
:10553800A74B185D01340AF00EFD082CF8D10024A1
:10554800A44B185D01340AF006FD072CF8D100F0D1
:10555800EBBC07200AF02EFDE7200AF0FCFC9E4B6E
:1055680058790AF0F8FC00200AF0F5FC042000F055
:10557800D9BCA3420AD2994A9D5C012202FA05F5D8
:105588000D421CBF9A4010430133F2E70AF01EFD9A
:10559800914B93F8A40700F011BC12200AF00AFD01
:1055A8008F4B1B88B3F5806F8CBF0825012500241D
:1055B8008C4B33F9140090FBF5F0013480B20AF0FB
:1055C800FCFC032CF4D1884CA08D0AF0F6FCE08D8D
:1055D8000AF0F3FC208E0AF0F0FC608E0AF0EDFC75
:1055E800A08E0AF0EAFCE08E65E310200AF0E2FCE7
:1055F80000247E4B185D01340AF0ADFC102CF8D164
:1056080000F092BC70200AF0D5FC0026764D0E24DE
:10561800AB6C744323440136B3F819010AF0CDFC8E
:10562800AB6C2344B3F81B010AF0C7FCAB6C2344F2
:10563800B3F81D010AF0C1FCAB6C234493F81F01B9
:105648000AF089FCAB6C234493F820010AF083FC30
:10565800AB6C234493F821010AF07DFCAB6C234426
:1056680093F822010AF077FCAB6C1C44D4F82301B0
:105678000AF0ACFC082EC9D100F056BC7020564C7C
:105688000AF098FC04F1700594F8D0000AF063FC65
:1056980094F8D1000AF05FFC94F8D2000AF05BFCA1
:1056A80094F8D3000AF057FC94F8D4000AF053FC9D
:1056B80094F8D5000AF04FFC073494F8CF000AF0AC
:1056C8004AFCAC42E0D100F02FBC494B185D0134D4
:1056D8000AF041FC102CF8D100F026BC454D287882
:1056E800400000F0FE000AF065FC00242B789C4284
:1056F80080F01A84404B33F814000AF05EFC013441
:10570800F4E73E4C06200AF055FC20880AF055FCC8
:1057180060880AF052FC3A4B1888CCE207200AF05D
:1057280049FC384B1888FF28A8BFFF20C0B20AF0F0
:1057380012FC354B186880F3100080B20AF03DFC6B
:10574800B5F868000AF039FC234B93F885212F4BF4
:10575800186822B10A23584380F3100001E000F3CF
:105768000F0080B2A7E21C4C02200AF023FC94F838
:10577800E0010AF0F0FB94F8DF011FE30B200AF0C8
:1057880019FCEB6E18780AF0E6FBEB6E58780AF015
:10579800E2FB0026EB6E144C3344013618790AF00C
:1057A800DAFB032EF6D1E36ED8790AF0D4FBE36E68
:1057B80098780AF0D0FBE36ED8780AF0CCFBE36E59
:1057C80058890AF0FAFBE36E187AF7E2B8900108F4
:1057D800C490010899900108BC120020D91100203A
:1057E800040000209E120020C81100200012002092
:1057F80014120020C01D0020782C002090290020C1
:10580800AC120020901A00209C1A0020981A002040
:10581800C64C1E200AF0CEFBA36C1B78022B4FF05F
:1058280000056BD1A36C03EB850393ED080AB2EE78
:10583800048A20EE080A10F0BFF880F30800C0B20E
:105848000AF089FBA36CDFEDBA7A03EB850393EDCD
:105858000B0A20EE270A10F0AFF880F30800C0B258
:105868000AF079FBA36CDFEDB37A03EB850393EDC4
:105878000E0A20EE270A10F09FF880F30800C0B245
:1058880001350AF068FB032DCCD1072DA36C23D179
:1058980093ED110A20EE080A10F08EF880F3080044
:1058A800C0B20AF058FBA36C93ED120A20EE080A66
:1058B80010F082F880F30800C0B20AF04CFBA36C29
:1058C80093F84C3000EE103AB8EE400A10F074F835
:1058D80080F30800C0B20BE02B4458780AF03BFB79
:1058E800A36C2B44D87A0AF036FBA36C2B44587D62
:1058F80001350AF030FB0A2DC7D115E3A36C2B4400
:1059080058780AF028FBA36C2B44D87A0AF023FBBA
:10591800A36C2B440135587D0AF01DFB0A2DEDD1EF
:1059280002E33C200AF046FB0024804D9FED818A6B
:10593800AB6C03EB840393ED080A20EE080A10F021
:105948003BF880B20AF039FBAB6C03EB840393EDB0
:105958000B0A20EE080A10F02FF880B20AF02DFB8F
:10596800AB6C03EB840393ED0E0A20EE080A10F0EB
:1059780023F8013480B20AF020FB032CD5D1072C80
:10598800AB6C16D193ED110A20EE080A10F014F84A
:1059980080B20AF012FBAB6C93ED120A20EE080AF3
:1059A80010F00AF880B20AF008FBAB6C93F84C00D0
:1059B8000BE0234458780AF000FBAB6C2344D87AF8
:1059C8000AF0FBFAAB6C2344587D01340AF0F5FA6F
:1059D8000A2CD4D1A8E214F8010F002800F0A48200
:1059E8000AF0B9FAF7E701200AF0E4FA4F4B9B6C8A
:1059F8001878E3E150200AF0DDFA00254B4B9C6C47
:105A08004D4B04EB85040C2194F8792001FB0233FB
:105A1800013593F838000AF09EFA94F87A000AF0F3
:105A28009AFA94F87B000AF096FA94F87C000AF047
:105A380092FA142DE2D177E23C4B9C6C062303FBCF
:105A48000544013594F8CE000AF085FA94F8C900A7
:105A58000AF081FA94F8CA000AF07DFA94F8CB00AB
:105A68000AF079FA94F8CC000AF075FA94F8CD00A7
:105A78000AF071FA0C2DDFD156E24FF0000801262A
:105A880000272A4B1A7C974227DA11330024FA5C44
:105A9800294D0C2305F130016343595C914207D12C
:105AA8002B44586B0FF0BDFD82462EB9B14605E078
:105AB80001341C2CECD10EE080440CE0D1450ADA0C
:105AC8000C2303FB04535B6B13F809000AF043FA39
:105AD80009F10109F2E70137D3E7002E00F024822B
:105AE8005FFA88F00AF066FA0026C9E70F4D287CAD
:105AF8000AF060FA00242B7C9C4280F015820F4B40
:105B0800E65C00210C480C2200F1300702FB01F38F
:105B1800DA5DB24205D1034493F838000AF01BFA63
:105B280002E001311C29EDD10134E4E7C81100205D
:105B38000000C84200007A4408740108D911002006
:105B4800D04C16200AF036FAB4F896010AF035FA65
:105B5800B4F840010AF031FAB4F842010AF02DFA1B
:105B6800B4F844010AF029FAB4F8D8010AF025FA81
:105B780094F8ED010AF0EFF900200AF0ECF994F836
:105B8800EE010AF0E8F994F885010AF0E4F994F8CE
:105B980092010AF0E0F900200AF0DDF9BA4B9B6C9B
:105BA8000A20B3F9563093FBF0F080B20AF005FAF8
:105BB8008EE0E0B201340AF0CEF9092CF9D1B3E154
:105BC80010200AF0F7F9B14BB14C187800F0020038
:105BD8000AF0C1F9AF4B18780AF0BDF920680AF04D
:105BE800F5F960680AF0F2F9AB4B18880AF0E5F9A4
:105BF800AA4B18880AF0E1F9A34BB3F870005AE0F1
:105C08000AF08CF9074612200AF0D4F99E4C17B90D
:105C1800666FA56F06E0102F13BF0025E66FD4F856
:105C280080502E4638460AF096F930460AF0CEF9EA
:105C380028460AF0CBF9D4F884000AF0C7F9002006
:105C48000AF0BBF900200AF0B8F90020B6E08E4D42
:105C580095F8880080000130C0B20AF0ABF995F8D9
:105C680088000AF078F900242E4696F888309C427D
:105C780080F05A818A4D285D0AF06DF905F110030C
:105C8800185D0AF068F905F120033035185D0AF04F
:105C980062F9285D0AF05FF90134E6E708200AF0A6
:105CA80089F900200AF089F900200AF086F9002015
:105CB8000AF083F900200AF080F935E104200AF09F
:105CC80079F9704B98682DE104200AF073F96D4C4E
:105CD80094F87A010AF03FF994F87E010AF03BF94A
:105CE80094F87D010AF037F994F87F0166E0654C75
:105CF80007200AF05FF9B4F880010AF05EF9B4F8F9
:105D080082010AF05AF994F884010AF024F9B4F8E7
:105D18008601D0E75B4C0C200AF04CF994F890010E
:105D28000AF019F9B4F89A010AF047F9B4F896019B
:105D38000AF043F9B4F898010AF03FF994F8910190
:105D48000AF009F9B4F89C010AF037F9B4F89E0191
:105D5800B1E74C4C04200AF02DF994F8D6010AF06A
:105D6800FAF894F8D7010AF0F6F8B4F8D801A2E7DF
:105D78004C4C4D4D207800EB4000C0B20AF01AF9A7
:105D8800002623789E4205F1020580F0CD8015F8A3
:105D9800020C0AF0E0F815F8010C00EB800000EBAB
:105DA800800000F2EE2080B20AF007F90136E8E739
:105DB80001200AF0FFF8334B93F892010AF0CBF870
:105DC800B2E0304B2344013493F888010AF0C3F859
:105DD800082CF6D1A8E02B4C10200AF0EBF86079DB
:105DE8000AF0B9F8A0680AF0F1F894F890010AF0FE
:105DF800B2F8B4F858010AF0E0F8B4F85A010AF019
:105E0800DCF8B4F85C010AF0D8F8B4F880010AF0BC
:105E1800D4F8B4F882014EE71B4B1A4C93F8C9002A
:105E2800C0EBC000C0B20AF0C5F804F118051F4A5B
:105E380094F8F40192F9001043B2994278D092F99B
:105E48000C10994274D092F918209A4270D00834F4
:105E5800AC42ECD168E040200A4C0AF0ABF804F1FF
:105E68004005B4F89C020AF0A8F894F89E020AF0DB
:105E780072F8043494F89B020AF06DF8AC42F0D141
:105E880052E000BFBC120020C8110020A41A002054
:105E9800AC1A0020AA1A0020A81A0020A61A00206E
:105EA80051120020C01D00205C140020CC1D0020D1
:105EB800E0202D4C0AF07EF804F18005B4F81E02AB
:105EC80000F03F000AF079F8B4F81E02C0F386101B
:105ED8000AF073F894F81C0200090AF03CF894F8E8
:105EE8001C0200F00F000AF036F8043494F8190286
:105EF8000AF031F8AC42E1D116E00D200AF05AF868
:105F080000200AF028F800200AF060F806E0174B95
:105F1800185D01340AF01FF80B2CF8D100200AF0A4
:105F280055F800200AF052F8012018E0002016E089
:105F38000AF011F8B4F8F6010AF03FF894F8F801FD
:105F48000AF009F894F8F9010AF005F894F8FB0149
:105F58000AF001F894F8FA0109F0FDFF77E7BDECC3
:105F6800028BBDE8F08700BFBC120020B890010882
:105F78002DE9F047C94CCA4E237886B00746002B56
:105F880000F0138232686368D31A7C2B40F20D82CA
:105F9800237A6260013323724FF0000808F124006D
:105FA800BE4DC0B20CF036F905F10A0333F91830CA
:105FB80007EE903ABB4B1B88B8EEE77A07EE903AAB
:105FC800F8EEE77A08F10108C7EE277A9FEDB67A6E
:105FD80067EE877AFDEEE77ACDED037ABDF90C001E
:105FE8000CF006F9B8F1030FD8D130200CF012F9F3
:105FF800B5F910000CF0FCF80CF004F92B7A9A07AC
:106008002CD16A6841F288339A4218D910200CF0D2
:1060180001F94FF06408686990FBF8F000B20CF0E1
:10602800E7F821200CF0F6F8686990FBF8F308FB14
:1060380013000028B8BF404200B20CF0D9F8142071
:106048000CF0E8F8B4F918000CF0D2F81C200CF0A9
:10605800E1F800200CF0CCF80CF0D4F8237ADFF843
:106068003C825B0740F07E8102200CF0D3F8D8F820
:106078001C00DFF848926423323090FBF3F000B242
:106088000CF0B6F80320B8F926500CF0C3F8874B8B
:106098001B7813F0040F4FF0050A95FBFAF5ADB223
:1060A8000DD008F5D87039460AF087FA28B9D9F81A
:1060B800003013F0100F18BF002528B205E0D8F8FB
:1060C800F8379889B0FBFAF000B20CF091F8D9F8DB
:1060D80000309F0740F18A80DFF8E491B4F8FE773A
:1060E80099F80030B4F8FC276C4D3F014FF0640874
:1060F800BFB208FB02325B00B2FBF3F347EA0327A7
:10610800BFB2C3F303231F4306200CF083F838B251
:106118000CF06EF8B4F8FE3799F8001001339BB212
:1061280093FBF1F201FB1233A4F8FE37D4F80038E0
:106138009B7B012B05D139200CF06CF8B5F9FC07D5
:106148001AE0B5F8FC576E233A205D4315270CF08A
:1061580061F895FBF7F5AFB2B7FBF8F528B20CF08C
:1061680047F808FB15753B200CF054F8A8B2451DFC
:106178000A2095FBF0F000B20CF03AF828200CF059
:1061880049F8D4F80438454D0A2093FBF0F000B2E2
:106198000CF02EF804200CF03DF8D4F8F837D5F8B8
:1061A80008089A894FF6FF739842A8BF1846C2B1EB
:1061B8000028ACBF131A134607EE903A9FED3C7ABD
:1061C800F8EEE77A67EE877A07EE102AB8EEC77A14
:1061D800C7EE877AFDEEE77A17EE900A6428A8BF23
:1061E800642020EAE07000B20CF002F8D4F80C3811
:1061F8002A4F9D0640F1AB8097F8103898071DD5B7
:1062080011200CF007F8B7F812082A4B4FF4F36581
:10621800684390FBF3F000B20BF0EAFF19200BF093
:10622800F9FFB7F812084543642095FBF0F595FB94
:10623800F0F300FB135000B20BF0DAFF94F81038BB
:10624800B4F8145813F0020F08BF002501200BF012
:10625800E1FF28B20BF0CCFF09200BF0DBFF002098
:106268000BF0C6FF144B94F816581A88B2F5967FAF
:106278000AD90A4B1B7A03F00F03072B04D842F202
:106288000F75954228BF154605200BF0C3FFD4F8BB
:1062980000385B7BC3B928B233E000BF94120020FA
:1062A800BC2900200400002000007A44B62D0020FC
:1062B8000000C842A0860100F600002098290020AE
:1062C800F40000206666E63FA5F1200307EE903A49
:1062D8001FED047AF8EEE77AF6EE006AC7EE877AE1
:1062E800BEEE007AF5EEC07AF1EE10FA58BFB0EEC5
:1062F800667A77EE877AFDEEE77ACDED037ABDF917
:106308000C000BF075FF94F81028C94B910703D4C3
:1063180093F81728012A04D1012384F81738C548AF
:106328001CE0D3F80038DFEDC46A93ED017AD3EDB1
:10633800027A27EE267A67EEA67ABDEEC77AFDEED8
:10634800E77A8DED047ACDED057A04A806E0BB4A1C
:1063580092E8030004AB83E80300184604F0C2FA8D
:106368000BF050FF237A282B1FD1B14B00221A7251
:106378003C2733684FF47A70B3FBF0F817200BF022
:1063880049FFB8FBF7F5B5FBF7F007FB1050000223
:1063980000B20BF02DFF18200BF03CFF07FB158017
:1063A80000B20BF025FF0BF02DFF94F82038A04D1C
:1063B800002B00F062810AF045F9D5F82438A04A8C
:1063C800C31A9342074640F2C680002385F82A384C
:1063D80085F82C38B5F8FC37DAB21B0A85F8462858
:1063E80085F8473885F83C2885F83D38D5F854288D
:1063F80033689A1AD5F85838D97B4FF47A734B43D7
:106408009A420ED38F4B1B68C5F8543895F85C3800
:10641800013B012B9FBF102385F82A38022385F8FA
:106428002C380A20D4F8042892FBF0F284F8442887
:10643800121284F8452894F81028D4F8083893FBE9
:10644800F0F384F848381B1284F84938920794F816
:106458001638774984F8773803D42D2381F87838AB
:1064680077E0042BD4F81898D4F81C68DFF8E48196
:10647800754A8CBF3323322381F878384FF0060CE5
:10648800724B99FBF3F096FBF3F308FB009108FBC2
:10649800036803EB83030CFB01F103EB830391FB1C
:1064A800F2FE642502FB1E119B0091FBF5F184F8B6
:1064B800691809120CFB08FC84F86A189CFBF2F1B5
:1064C80043FA81F39BB202FB11C292FBF5F284F806
:1064D8006E28121284F86C3884F86F281B0AB4F8F6
:1064E800122884F86D382423534393FBF5F5B4F848
:1064F8008A3884F8703800EB80001B0A00EB8000B3
:10650800800084F871380A22B4F81438B3FBF2F327
:1065180003F5FA739BB240FA8EF080B284F87238B1
:106528001B0A4FEAD97984F86708F60F000A84F83D
:10653800645884F87338C5F30725B4F88C3884F8A0
:10654800669884F8680884F86B6884F8655884F855
:106558007938C4F8247894F88E88354DB8F1000F4E
:106568000DD1D5F894080AF05CF9012807D902285A
:10657800374E00F0628204F0A7F90123B370D4F813
:1065880098282B4D002A78D095F88E683EB1D5F81A
:10659800A03840F6B731FB1A8B4219D86DE00123B9
:1065A800D5F8940885F88E3803F0BBF9D5F8A438E7
:1065B80093F9000002238DE84800082132464FF481
:1065C800964303F0C9F985F8A868C5F8940852E01D
:1065D80095F89C68CEB9D5F89408C5F8986885F8F8
:1065E8008E6803F09EF9D5F8A43893F900000123CA
:1065F8008DE84800082132464FF4964303F0ACF981
:10660800C5F8940804F060F935E0013EF6B285F863
:106618009C6895F8A81895F8A938EEB94A1C013372
:1066280085F8A82885F8A938D5F8940821E000BF8E
:1066380094120020AC1A00208096184B947501081B
:106648003F0D0300BC29002040420F0080969800AF
:1066580004000020806967FF12F8016BC5F89828CC
:10666800701885F8A8080133D5F8940885F8A93872
:1066780031460AF0D9F8C4F8A07894F8AA38A24D9F
:10668800F3B1D5F8AC38DBB1D5F8B038C3B1C5F83B
:10669800B4381B689D4AC5F8B838D5F8BC381344D7
:1066A800187AFEF729FDD5F8B438987909F053FC23
:1066B800D5F8BC380133092B88BF0023C5F8BC388E
:1066C800934D94F8C0282E688F4B002A00F0F08173
:1066D800D3F8C428002A00F0EB8193F8C838013BAE
:1066E800012B00F2E581D4F8C408874F0AF099F825
:1066F800E0B1D7F8C4080AF091F897F8C938D5F886
:1067080000907E2B80460ED102231B2887F8C838BC
:1067180009D1D7F8C4080AF084F820B90123C7F8CA
:10672800CC9887F8D03884F8C988DCE7D7F8CC2823
:106738002B689B1A41F6583293421ED9032387F8D7
:10674800C838B5E1734A32F8130010B903464FF45C
:1067580003600133B0F5C06FDBB279D01ED9B0F554
:10676800006F7FD032D9B0F5036F3FD184F8D138AC
:10677800D4F80C38644F99063FD494F8D01894F89C
:10678800D138002900F056812A68921B012AD9D9EC
:1067980084F8D138002384F8D03889E1B0F5007F37
:1067A80043D007D8B0F5807F49D0B0F5887F00F096
:1067B8008D80E6E7B0F5806F00F0B080B0F5826FAD
:1067C80000F0F580B0F5047FDBD123E0B0F5E26F8F
:1067D80000F08D80B0F5E46F00F08E80B0F5E06FCA
:1067E800CFD184F8D138B4F90A1089E0B0F5046F34
:1067F80076D0B0F5026FC4D105E197F810389A0742
:10680800BBD5B7F8121824234B431233642193FBEA
:10681800F1F109E184F8D1383F4B3B4F1B689B07E6
:10682800ABD5B7F8FC370A21FDE084F8D1383A4BEC
:10683800354F1B681905A0D5D7F80418F4E084F87B
:10684800D138D4F80C38304F5A0796D57969EBE02F
:1068580084F8D138304B2C4F1B681B058DD5D7F8E1
:106868000818E1E0D4F80C18274A84F8D1388F06C4
:1068780083D592F8101888077FF57FAFD90712D50E
:10688800D2F81C3883EAE371002BA1EBE37101EB2A
:1068980051014FF01902B1FBF2F1ACBF41F00041D8
:1068A80041F040410FE0D2F8183883EAE371A1EBD8
:1068B800E371002B01EB51014FF01902B1FBF2F12A
:1068C800B8BF41F080414FF400608BE084F8D138C4
:1068D800D4F80C380C4F5B077FF54FAF3969A3E04C
:1068E800B4F9181084F8D138642359437AE084F84D
:1068F800D138B4F90C1003E0B4F90E1084F8D1388B
:106908002C2391FBF3F16DE094120020947501089B
:10691800BC290020D69401089829002084F8D13891
:1069280094F8D238644A0133DBB2032B88BF0123C1
:1069380082F8D23894F8D21842F2107359435F4B58
:106948001B78D80748BF01319A0748BF02315F0753
:10695800B4F8D43848BF0431D80748BF0A319A0779
:1069680048BF14311F0648BF2831D80548BF283111
:106978005A0748BF64311F0748BFC831980548BF48
:1069880001F5C8719A0648BF01F57A71DF0648BF5C
:1069980001F5FA61580648BF01F57A614FF4806045
:1069A80003F05EFF444B002283F8D028E5E6D4F8D4
:1069B8000C18DFF8048184F8D13811F0200717D0BB
:1069C80098F8102812F0020F14BF4FF47A710021C2
:1069D80012F0010F14BF4FF4FA6300230B4494F82C
:1069E8001618194403F03CFF002384F8D038C4E695
:1069F800334B1B6819067FF5C0AE394603F030FFEC
:106A080088F8D078B9E684F8D138D4F80C382A4F09
:106A18009A067FF5B2AE97F810389B077FF5ADAEB2
:106A2800B7F814386421594303F01AFF002387F894
:106A3800D038A2E684F8D1383AE0B37823B1C5F863
:106A4800907886F802809AE5D5F89038FB1AB3F565
:106A58007A6FFFF494AD0123D5F89408B37009F068
:106A6800DDFE0646D5F8940809F0D8FE76067FF4D0
:106A780086AD8A2802D08E280DD080E5D5F80C384E
:106A880098067FF57CAD95F88E38002B7FF477ADAE
:106A980005F65D0306E095F88E38002B7FF46FADA0
:106AA80005F62803C5F898382D2385F89C3866E53F
:106AB80006B0BDE8F08700BF94120020B62D002074
:106AC800982900200D4B0E491A680E4B92B21344B8
:106AD8005B000D4A1B68C3F3090310B51360136804
:106AE8009BB201335B1000229A4206D0074851F846
:106AF800044B20F812400132F6E710BD505C00400C
:106B0800206200401E300020DC260020E126002004
:106B1800014B00221A607047D826002013B50622C0
:106B28000446A82119206B46FEF7FCF9F8B19DF838
:106B380000309DF8012043EA022202219DF803302B
:106B480012B292FBF1F222809DF8022042EA03225F
:106B580012B29DF8053092FBF1F262809DF8042094
:106B680042EA03231BB2012093FBF1F3A38002B096
:106B780010BD08B5242180221920FEF74FFA6420A1
:106B880009F087FD202197221920FEF747FA0A20ED
:106B980009F07FFD102223211920FEF73FFA642017
:106BA80009F077FD024B4FF480521A8008BD00BFF0
:106BB80004000020154B37B5082205461A85E82041
:106BC8000AF0CAFB002400200AF0C6FB0DF80400F6
:106BD8000134062CF7D10D4B08229A619DF800204C
:106BE8009DF8013043EA02232B809DF802209DF88E
:106BF800033043EA02236B809DF804209DF805309A
:106C0800012043EA0223AB8003B030BD00100048E6
:106C1800274A73B55369274C43F400135361032380
:106C28006946082501268DF80530204600238DF891
:106C380006308DF8073000958DF8046002F006FAEA
:106C48001D4AA561138823F040031B041B0C138005
:106C5800138823F038031B041B0C2B431380138861
:106C68009BB243F040031380242025850AF074FB6F
:106C780080200AF071FBA561642009F0FFFC2585DE
:106C880020200AF069FBAF200AF066FB3046A561B8
:106C980009F0F4FC258523200AF05EFB60200AF049
:106CA8005BFBA561642009F0F4FC02B070BD00BF75
:106CB800001002400010004800300140024B4FF421
:106CC80080221A60704700BF140401402DE9F04F7C
:106CD800944D954C2B68954E9BB223802288318821
:106CE8000A40900585B007D54FF6FF53904A2B60B0
:106CF80013780133DBB2137023880B40190440F179
:106D080043830023ADF80A302B6887499AB21804E8
:106D1800228040F139830B8803F00F038B70002B1E
:106D280040F00483834A844F136884489BB23B80B5
:106D38003B8803F0300303803B8803F440533B80D7
:106D4800D2F800E04BF6BF730EEA030383F4005356
:106D580083F0200343F4004343F0800313600B885F
:106D680013F0100F804626D1116848F60F730B40B8
:106D7800734913600B681A7A022A894601D0042ADB
:106D880005D101F0CFFDD9F800301B7A3FE1062A82
:106D98006ED15A78052A09D11A78520606D1D878C0
:106DA80001F0A4FD674B1B681B6A9847664B1B687C
:106DB8009B6898475CE013689BB2ADF80A30BDF851
:106DC8000A301B0540F1F38111685D4840F68F7366
:106DD8000B405E4913600A685D4B92B213445B0036
:106DE80081461A68036893F808E0BEF1090F8A46DD
:106DF80017D092B2520002F1804202F5C0421178D7
:106E08001970517859709188C8B2090A41EA00216D
:106E180059801189C8B2090A41EA002199809289EA
:106E2800DA8001221A72DA8893F801B0002A40F059
:106E3800F1801A7812F07F0250D1BBF1090F10D1FE
:106E4800DA78012A00F2CA809978002940F0C680D1
:106E58009988002940F0C2809A723A4B1B685B6897
:106E6800BAE0BBF1050F10D193F90320002A01DA2B
:106E78000823CCE09A78002AFAD19A88002AF7D118
:106E88009B7A002B00F0B480F2E7BBF1030F0FD11F
:106E9800DA78012A40F0A2809A88002A40F09E8081
:106EA8005A7A42F020025A72264B1B68DB6993E03B
:106EB800BBF1010F40F09280DA78012A40F08E8011
:106EC8009A88002A40F08A805B7A980640F186808A
:106ED80001F0D6FD002800F08B807FE0012A39D12F
:106EE800BBF10B0F7AD1184A58791268D978926990
:106EF8009047D9F800309A7A002A6FD000286DD1CF
:106F08001A79002A6AD19B78002B67D10D4B1B6830
:106F1800DB6898470A4B1B685A79DA72DA781A7371
:106F280066E000BF445C00406C1B00202227002064
:106F3800B72D0020005C0040F21D0020F01D00204D
:106F48001C1D0020201D0020341F0020505C004024
:106F580004300020022A41D1BBF1010FB8D0BBF1A7
:106F6800030F3BD1587920F0800E4FEA8E0202F1D0
:106F7800804101F5B84110F0800F096814BF01F095
:106F8800300101F44051BEF1030F27D8B3F802E0F5
:106F9800BEF1000F22D109B39B7AFBB102F1804206
:106FA80002F5B842010613684BBF23F4E04323F40B
:106FB800804323F0400323F070034BBF9BB29BB286
:106FC80083F0100383F4805343F4004343F08003B9
:106FD8001360A94B1B689B69984709E0A74B1B687E
:106FE80058465B699847032810D000287FF440AFC3
:106FF800DAF80020A24B92B213445B001A68002210
:107008001A603023A8F80030062300E00923D9F8D5
:10701800002065E1BBF1060F13D11A7850067DD127
:107028009A78964B012A02D11B68DB696AE0022A2A
:1070380002D11B681B6A65E0032A6FD11B685B6A73
:1070480060E0BBF1000F3AD15988002966D15A682F
:1070580022F47F42B2F5003F60D11A7812F07F0225
:1070680004D19B88002B00F0F48157E0012A0AD153
:10707800824A587912689269904700284ED1D9F807
:1070880000309B7A17E0022A48D15A7902F00F01A2
:107098000BB29B0003F1804303F5B84312F0800F55
:1070A8001B6814BF03F0300303F44053032935D899
:1070B80012F0700F32D1002B40F0CB812EE0BBF1E3
:1070C800080F04D11B78590600F0C58126E0BBF1F2
:1070D8000A0F23D11A7802F07F02012A1ED19A7A68
:1070E800E2B15988D1B95A6822F47F42B2F5803F9B
:1070F80014D1624A5879126892699047002800F0C2
:10710800AC810BE053B1D9F800204FF0000AA2F887
:1071180012A093615046984750460BE0574BD9F858
:1071280000201B6850781B699847032802D1554BEB
:107138001B6806E0D9F800301A8A4FF6FF718A42B8
:1071480001D1092203E0022800D012B908221A72DC
:10715800C7E093F90010002923DAD988039103982E
:10716800DFF818E1824202D9039A1A8211E08A42B2
:107178000FD2DEF8001091F82C00824201D20021D3
:1071880005E092FBF0F100FB112212B901213E4A01
:107198001170DEF8002092F82C209A8201F0C2FBD0
:1071A8009FE003221A724FF440533B8099E0BDF8E8
:1071B8000A301BB2002BBFF6A7AD116840F68F73DB
:1071C8000B4013602F4AD2F8009099F80830022B30
:1071D800934600F08280042B7FD0032B01D0052B2F
:1071E80075D1D9F81830B9F810209BB9B9F8102022
:1071F800002A4FD04FF440533B80244B1968204B52
:1072080089B20B445B001968002119603023A8F883
:1072180000303FE0002AE9D0B9F814A0924528BF11
:1072280092461FFA8AF2104601929847019AB9F8D5
:1072380010309B1AA9F81030B9F812301344A9F885
:107248001230124B1A68124B92B213445B000AF1C7
:10725800010A1B689BB203F1005303F540534FEA40
:107268006A0A5B0000215145C0D053F8212020F85C
:1072780011200131F7E700BF201D0020341F002036
:10728800023000201C1D0020B82D0020505C00405A
:1072980004300020B9F814309342DBF8003001D8EC
:1072A800032201E012B105221A720CE006211972BC
:1072B8006C4B19686C4B89B20B445B0019681A60F7
:1072C8003023A8F80030DBF800301B7A06E0072BE3
:1072D80003D1664B1B68DB6898470823DBF800205E
:1072E800137201F0B1FB624B1A684BF6BF7313407F
:1072F8003A88D2043A8848BF83F480539004B8F897
:10730800002048BF83F40053D106B8F8002048BFD6
:1073180083F01003920648BF83F0200343F4004330
:1073280043F08003524A9BB213602DE09A0002F1A9
:10733800804202F5B842116889B2ADF80A10BDF86A
:107348000A1009B2002909DA106840F68F71014065
:107358001160013B474A52F823309847BDF80A307C
:107368001F067FF5D1ACA1788B0003F1804303F5AC
:10737800B84348F60F72186802401A603D4B03EB99
:1073880081039B699847BFE42288338813405905D5
:1073980005D54FF6FF332B60374B5B68984722883B
:1073A80031880A40920444BF4DF6FF732B6023884E
:1073B800324A0B40DB0452D54EF6FF732B60002394
:1073C800D370D378052B41D8DFE803F0030D1418E8
:1073D800222DA368294D1BB908F064FC062300E0A0
:1073E8000523EB703BE008F05DFC0423E370012308
:1073F800A36034E002232371032328E02379013BAF
:10740800DBB22371237953BB1C4B0422DA7026E0CC
:107418001B4A13689BB243F0100313600523E37003
:107428000A2323711BE02379144A013BDBB2237141
:10743800237903F0FF0093B911490C684FF6EF73F5
:1074480023400B600623D370906008E00623E370A6
:1074580005E00C4B57E60C4B55E60C4B53E605B0D4
:10746800BDE8F08F505C004002300020341F00203F
:10747800005C0040A87501080C0000206C1B00206F
:10748800405C004057850008FD850008DD85000840
:10749800704770477047FEE7FEE7FEE7704730B574
:1074A8000024E3B293420DD2030F092B94BF30336B
:1074B800373301F8143001EB4403002500015D70F7
:1074C8000134EEE730BD0248024906F03EB800BF7D
:1074D80000480140E02800200148024906F035B87C
:1074E80000400140902800200148024906F02DB8CC
:1074F80000340140682800200148024906F025B8F8
:1075080000340140682800200148024906F01DB8EF
:1075180000080040402800206D4B6E4A9FED6E7AAF
:10752800D2ED007ADFED6D4ADFED6D3A30B51C889B
:10753800B3F90AE01D8A06EE904AB8EEE76AF8EE5B
:10754800666ADFED687AB3F9044067EEE67AB7EE6B
:10755800004AE6EE077A9FED647A67EE666A9FED69
:10756800637AE6EE076A27EEA77A07EE904AB3F940
:1075780002409FED5F6AF8EEE77A67EE277A07EE3A
:10758800104AB8EEC77ADC89E6EE877AB6EE007A5A
:10759800FDEEE76A87EE866AC3ED066AF8EEE66AEC
:1075A800D2ED017A9A89E6EE874A06EE90EAB3F9B7
:1075B80008E09FED507A05EE90EAF8EEE66AF8EEFC
:1075C800E55A66EEA46A65EEA45A66EEA46AB3F8B4
:1075D80006E0E6EE875A65EE875AA5EEA34AF0EE76
:1075E800445A04EE10EAB8EE444A25EE844AB5EE51
:1075F800404AF1EE10FA5BD02DB205EE905A24B253
:1076080024EEA45A07EE104AF8EEE55A12B265EED7
:10761800255AB8EEC75A65EEA35A64EE854AB0EE0D
:10762800007AE4EE875AB5EE007A65EE875A07EEDF
:10763800102AB8EEC75A9FED307ADFED306AB3F9F9
:107648001620E5EE075AF8EEE77A9FED2D7A76EEEA
:10765800E77ADFED2C6AE5EEC77A05EE902AB0EE00
:10766800677ADFED297AB3F91420B3F9123067EE9F
:10767800277A07EE102AC7EE847AF8EEE55AB8EEB4
:10768800C77A65EEA75A27EE877A65EEA75A27EEDE
:10769800237AA5EEA67AF0EE476A07EE103AB8EE1E
:1076A800C77A36EE877ADFED196AE7EE267A01E0C7
:1076B800DFED177A18B1FDEEE77AC0ED007A31B147
:1076C800FDEEC67A642217EE903A53430B6030BD44
:1076D80008030020781B00200000003700007AC74C
:1076E80000000038000000390000803A00008038AF
:1076F8000000A045000000360000804700008049D7
:1077080000008039000000300050C3450000803D73
:1077180000000000704770476C4B6D4A2DE9F04F30
:107728005E8994684FEA062AB4EB0A0A9C884FEAF5
:1077380004481C894FF000054FF0000B65EB0B0B5C
:10774800A4FB0A6704FB0B77F40944EA476418EBC7
:1077580004065C884FF000094FEAE7154FEAC43881
:10776800DC8849EB050787B0CDE90467A4FB0A6705
:1077780004FB0B77340A44EA076418EB04064FEA63
:1077880027259C894FF0000949EB0507CDE90067DB
:10779800AAFB046704FB0B77F40D44EA472414F5AD
:1077A800FA664FEAE75545F10007B6F5FA6F77F143
:1077B8000003CDE90267964667DAA4FB046704FB79
:1077C80005F34FF0050C07EB4307DDE90489A6FB39
:1077D8000C230CFB07335F104FEA3206B8EB0608A0
:1077E8004FEA920669EB070946EA83769F10DDE9BE
:1077F8000023921B63EB0703DDE90267CDE9002351
:10780800344A4FF0FF33964277EB0303CDE90489FE
:1078180028DA40F6AC52A4184FF000035D4104FB8F
:1078280005F3A4FB044505EB43056FF00602664229
:1078380002FB0566A4FB0223334418EB020649EB5E
:107848000307CDE904670B26A4FB062306FB0533D3
:10785800DDE900455B104FEA3202A41A65EB030527
:10786800CDE900450AFB0BF3DDE90245AAFB0AABAB
:107878000BEB430B4FEADA7242EA4B02A41A4FEAC7
:10788800EB7365EB0305CDE90245DEF80C40009B80
:10789800019DA4FB032304FB05334FEA52584FEA2A
:1078A800635948EAC328DDE90423B8EB020269EB0F
:1078B80003039946D30B43EA494300B1036009B176
:1078C800029B0B6007B0BDE8F08F00BFF6020020F6
:1078D800781B002024FAFFFF054B1A7C02F0FF01F9
:1078E80022B10122027000221A7470470170704799
:1078F800781B002007EE900AF8EEE77ADFED0C6AB5
:107908009FED0C0AF5EEC07AF1EE10FAD4BFB1EE95
:10791800677AC7EEA67A08B5D8BFC7EE267A27EEEB
:10792800800A05F0A1FA044B83ED000A08BD00BFE8
:107938008096184B35FA8E3C980000207620F4216A
:107948003122FDF76BBB772048210122FDF766BB8A
:10795800772058210122FDF761BB1FB5044602219B
:107968000C2001220DF10703FDF7DCFA08B900200D
:107978003BE09DF80730DB07F9D50321062202AB6F
:107988000C20FDF7CFFA0C20092101220DF1070385
:10799800FDF7C8FA0028EAD09DF8073013F00C0F5D
:1079A800E5D19DF809209DF8083043EA0223C3EB8E
:1079B80083339B009DF80B2023809DF80A3043EA0F
:1079C8000223C3EB83339B009DF80D2063809DF851
:1079D8000C3043EA0223C3EB83339B00A3800C20C3
:1079E8000A210122FDF71AFB012004B010BD07B5DA
:1079F800F7216B4606227620FDF794FA9DF80030B1
:107A08009DF801100B4A1B0343EA01139DF802106D
:107A180043EA111353609DF803309DF804101B03CB
:107A280043EA01139DF8051043EA1113136003B0EC
:107A38005DF804FB781B002007B5002101AB032289
:107A48007720FDF76FFA9DF805309DF804001B02BA
:107A580043EA00439DF80600184303B05DF804FBB1
:107A680008B5FFF7E9FF014BD86008BD781B002077
:107A780008B5FFF7E1FF014B986008BD781B0020AF
:107A880013B506220446432168206B46FDF74AFADF
:107A9800A8B19DF800209DF8013043EA0223238015
:107AA8009DF802209DF8033043EA022363809DF885
:107AB80004209DF8053043EA0223A380012002B088
:107AC80010BD13B5062204463B2168206B46FDF71E
:107AD80029FAA8B19DF800209DF8013043EA022355
:107AE80023809DF802209DF8033043EA0223638037
:107AF8009DF804209DF8053043EA0223A380012065
:107B080002B010BD07B50A2100220C20FDF786FA45
:107B1800142008F0BEFD0A210F220C20FDF77EFA82
:107B28000A2008F0B6FD01AB102103220C20FDF756
:107B3800F9F90A2008F0ADFD0A2100220C20FDF712
:107B48006DFA0A2008F0A5FD0DF1030302210122B8
:107B58000C20FDF7E7F90DF10303092101220C20A0
:107B6800FDF7E0F90A2101220C20FDF757FA03B0CE
:107B78005DF804FB08B508F06DF86B2180226820D9
:107B8800FDF74CFA642008F084FD6B21032268207D
:107B9800FDF744FA0F4B19211A786820FDF73EFAD1
:107BA8000F2008F076FD0C4B1A211A786820FDF793
:107BB80035FA1B2118226820FDF730FA1C21102203
:107BC8006820FDF72BFA682037210022BDE808401D
:107BD800FDF724BA240300200000002008B508F0AF
:107BE80039F8074B1B7813B1012B03D008BD4FF4AC
:107BF800006201E04FF48052024B1A8008BD00BFBA
:107C0800F402002004000020F8B59E4B1B680546CE
:107C1800187818B1012800F06B81E6E2242D9A4CFF
:107C28000CD006D80A2D00F0DC800D2D00F0D9808C
:107C380048E12A2D06D02C2D04D043E16074A074AD
:107C4800E07451E1914BA17C677C8F4A0020585425
:107C58002FBB19781775472921D1597850291ED17A
:107C68009978472907D1D978472904D11979412921
:107C780001D1012111759978844A522903D1D1780B
:107C88004D2900F0B4829978804A472907D1D178E4
:107C9800532904D11279562A04BF03222275227D62
:107CA800794E022A3AD0032A4DD0012A40F0878023
:107CB800BA1E072A00F28380DFE802F004080F13D7
:107CC8001A25812B09F048FDA06178E01B78532B19
:107CD80075D1A3695B42A36171E009F03DFDE061E4
:107CE8006DE01B78572B6AD1E3695B42E36166E07C
:107CF8001B78302B664B1A788CBF42F0020222F0B8
:107D080002021A705BE0002009F086FD84F820006A
:107D180055E0002009F080FD608450E0072F06D070
:107D2800082F4CD1012009F077FDF08447E00120AD
:107D380009F072FD41F2184358434FF47A73B0FBCF
:107D4800F3F0B0843BE0022F07D0032F0BD10020C3
:107D580009F062FD4F4B187031E0002009F05CFD1E
:107D680086F828002BE02AD93A1F921096F8283076
:107D78000132D2B2013B02EB8303DBB2102B1ED8D7
:107D8800F91EC2F1010201EB8202D2B2012A0BD024
:107D9800042A11D100205E1E09F03EFD3E4B985585
:107DA8003E4B00229A5507E05E1E3D4A002093553F
:107DB80009F032FD3B4B9855E36A0133E362324BDD
:107DC8002A2D18BFDA7C07F101074FF000000CBF1D
:107DD800012255406774A0740CBF83F83020DD740D
:107DE80082E094F83000002847D02F4B13F8012D7B
:107DF8002E495A708B42F9D1244A234D1378527870
:107E0800402B85BF373B1B011B01DBB298BF03F03A
:107E1800F003402A8CBF373A303AD2B21344E27C9E
:107E2800DBB29A4226D121230B70287D6B6B1F4A47
:107E3800013301286B630AD002281DD17223137005
:107E48001B4BAA8C1A801B4BEA8C1A8014E0672300
:107E580013700F4B1B789F070FD5174BAA691A6031
:107E6800EA695A60154B95F820201A70144B6A8CF1
:107E78001A8002E03F230B700020002384F8303082
:107E880032E000BF30080020781B0020C429002001
:107E9800A41A002050120020811200207112002024
:107EA80051120020611200204803002034030020F2
:107EB800A61A002038120020AC1A0020AA1A0020A6
:107EC800A81A0020A37C94F830000E2B9FBFAC4A60
:107ED800591C9174AB4A98BFD554A94A18B9D37C98
:107EE8005D40D57400E00020003018BF0120F8BDC7
:107EF800A34B93F838100022082900F27681DFE8B6
:107F080001F0050C101A2B3B607E8B00B52D40F05C
:107F18006C8183F83920012250E0622D08BF0222CB
:107F28004CE0032283F8382083F83A5083F83B501A
:107F380083F83C5059E1042283F8382093F83B2019
:107F480093F83C1083F83D502A44D2B283F83B2082
:107F58000A4483F83C2048E1052283F8382093F846
:107F68003B2093F83C10DD872A44D2B283F83B20AB
:107F78000A4483F83C2038E1062283F8382093F835
:107F88003B2093F83C102A44D2B283F83B200A44A1
:107F980083F83C20DA8F02EB0525ADB2B5F5AC7F4E
:107FA80088BF774ADD8784BF012182F83910002213
:107FB800A3F84020002D40F01881072283F83820CC
:107FC80013E193F83B2093F83C102A44D2B283F88B
:107FD8003B200A4483F83C20B3F84020B2F5AC7F3C
:107FE8003CBF6749891802F1010238BF81F8445043
:107FF800D98F92B29142A3F84020DED9F5E0082249
:1080080083F8382093F83B30AB4200F0EE805C4BAD
:10801800012283F839200FE05B4C83F8382014F8EC
:10802800012D6270594A9442F9D193F83C10544A90
:10803800A94206D03F232370554A53680133536041
:10804800D3E0516B92F839000131516310B13E23EE
:108058002370CAE02121217092F83D10062941D0F1
:1080680004D8022907D0032923D0F8BD122959D0F2
:10807800302967D0F8BD502121704649946C4C6076
:10808800D46C0C60516D4FF47A7491FBF4F1424C4E
:10809800218092F89C11414A19B1117841F00201EE
:1080A80002E0117821F002011170012283F89D216C
:1080B8008DE05321217092F84910CE0705D592F82A
:1080C8004820D51E6A426A4100E0024602F00101DA
:1080D80083F89C11002A7AD130490A7822F00202EA
:1080E8000A7074E04F21217092F84F10CC0705D523
:1080F80092F84E20D11E4A424A4100E0024602F060
:10810800010183F89C1122B924490A7822F002025D
:108118000A70234A93F873101170224AB3F870104A
:10812800118054E0562121701F49946D0C8042F251
:108138001074D16D91FBF4F11C4C2180012182F85F
:108148009E1144E04921217092F84810184A1029DC
:1081580088BF10211170174914780022A24233D227
:10816800154D0E7A5655154D4E7A5655144DCE7AF4
:108178005655144D11F80C6F56550132EEE700BFF5
:10818800781B0020C4290020480300203403002065
:1081980010080020AC1A0020A81A0020A41A0020F9
:1081A800AA1A0020F6000020A61A00203812002083
:1081B80050120020BC1B0020511200206112002028
:1081C8007112002081120020DA6A0132DA6293F813
:1081D8009D310B4A93B192F89E317BB1002182F810
:1081E8009D1182F89E111846F8BD0020F8BD12793D
:1081F800432A7FF448AD0222227544E5F8BD00BF4A
:10820800781B00200449054B0968187000225A6140
:1082180099611A77704700BFBC2900201008002018
:1082280010B5121A07EE902A5B1A2DED028BF8EEA4
:10823800E78A07EE903A184B059CB8EEE78AD3ED2B
:10824800007A28EE278A28EE080AA8EEA80A0DF078
:108258002DFEDFED127A049B20EE270AF0EE480A85
:10826800BCEEC00A83ED000AB1EE680A04F029FDED
:10827800DFED0B7A9FED0B7AE0EE077ABDEC028B0F
:10828800FDEEE77A17EE903A002BBCBF03F50C43DE
:10829800A033236010BD00BF980000202C7D8E3FC6
:1082A80000A00C46A00CB34544F25063984203DD8D
:1082B800A0F50C40A0387047034B9842BCBF00F5AE
:1082C8000C40A030704700BFB0B9FFFF73B51A4C1F
:1082D800036823600B686360184D0068184EFFF749
:1082E80009FB184B009395E8030094E80C000196ED
:1082F800FFF796FF144B32681A6068686368134981
:108308001B1A07EE903A124B286893ED007A2368FF
:108318001B1A0B600F4BF8EEE77A1A600E4B67EEEC
:10832800877A1B68FDEEE77ADA880C4BC1ED017A93
:108338001A8002B070BD00BF78260020AC1A002059
:108348008426002080260020C026002088260020C1
:1083580098000020B826002000100020B426002035
:108368004279DFED2A5A2A4B9FED2A5A07EE902AC6
:10837800F8EE677AC27BC7EEA57AB2EE047AC3ED4F
:10838800007A07EE902AF8EE677A234ADA60C7EE99
:10839800A57AC3ED017A8179204B07EE901AF8EEA1
:1083A800677A017CDA60C7EE877AC3ED007A07EE58
:1083B800901A817E06EE101AF8EE677AB8EE466AD1
:1083C800C7EEA57A86EE056AC3ED017A83ED026AE7
:1083D800C179134B06EE901A417CDA60F8EE666AB2
:1083E800C6EE876A07EE101AC17EC3ED006A07EE73
:1083F800901AB8EE477AF8EE677A87EE257AC7EED4
:10840800857A83ED017AC3ED027A70470000C8428D
:108418009026002000007A440000FA44A02600209C
:10842800C426002010B50C4C23789B0713D50B4BA2
:108438001B78042B0FD90A4A0A4B106852685A60F5
:108448001860FFF757FA084B1A88084B1A802378E8
:1084580043F00103237010BDA41A0020AA1A0020BB
:10846800AC1A00203C120020AC120020D4260020B8
:108478001C4B1B681B0307B530D51B4A1B4BD2EDA1
:10848800007A1B788DF80030B2EE047A67EE877AAE
:10849800174B9FED187A1B788DF80130FCEEE77AC0
:1084A8000A2017EE903AD2ED017A8DF8023067EE85
:1084B800877A6946FCEEE77A17EE903AD2ED027AAF
:1084C8008DF80330FCEEE77A17EE903A8DF8043019
:1084D800094B1B788DF8053001F032FE03B05DF8CA
:1084E80004FB00BF98290020AC2900208A2900201D
:1084F800A829002000007A448E290020054A137814
:1085080083F001031370044A00231360034A1360C5
:10851800AEE700BF8E290020A4290020A029002052
:1085280007B5232008F0B5F86820752101220DF160
:108538000703FCF7F7FC28B19DF80700A0F16803D2
:108548005842584103B05DF804FB00BF704708B5B6
:108558001F4A18B9536802221A8208BD00205168C0
:1085680010800B7813F07F030DD14B7A990644BF26
:108578000221117013F0400F137814BF43F0010368
:1085880023F0010315E0012B1FD0022B1ED14B79DC
:1085980013F0800F03F00F034FEA830303F18043C6
:1085A80003F5B8431B6806D003F03003102B07D13E
:1085B8000123137004E003F44053B3F5805FF6E73A
:1085C80093681B699847024808BD104608BD00BF5C
:1085D800181D002010B5064C18B9636801221A82CC
:1085E80010BDA3689B68984760680C3010BD00BF39
:1085F800181D002010B5064C18B9636801221A82AC
:1086080010BDA3681B68984760680A3010BD00BF9A
:10861800181D0020084BDA68D10709D4DA68D20699
:1086280008D4DB6813F0040F14BF0320042070473C
:1086380001207047022070470020024010B5044610
:10864800B0F9000008F081FEB4F9020008F07DFEE0
:10865800B4F90400BDE8104008F077BE10B5044630
:10866800006808F072FE606808F06FFEA068BDE858
:10867800104008F06ABE2DE9F74F012001F090FB89
:10868800002488B3012C2FD8194E4FF04C0909FB50
:1086980004FA06EB0A0808F15407BD7815B101344D
:1086A800E4B2EEE790F9003090F804E01846114B78
:1086B80003228DE8240001212A4653F82E3001F0C8
:1086C8004BF9834660B106F10C00504429464A46EE
:1086D8000CF063FF01231C44C8F80CB0BB70E4B273
:1086E800012001F041FBCCE703B0BDE8F08F00BFEB
:1086F800181D0020E075010810B5184C002120460F
:108708001A220CF04AFFA4F5F970142380F8F4310A
:1087180005230022042180F8F83180F8FA3180F826
:10872800003280F8023280F8083280F80A32522388
:10873800012480F8F91180F8FB2180F8011280F8F3
:10874800032280F8091280F80B2280F8F23180F8B1
:10875800FC2180F80442A0F8F64110BDAE140020B8
:1087680010B5FFF757FF4FF43024012806D11CB18C
:10877800FFF750FF013CF8E7052010BD002C08BFAB
:10878800052010BD70B50646441E14F8011F89B1B6
:10879800094D28460CF037FF0028F6D005F10803EC
:1087A80098423FBF054B401BC018A31B38BF80F839
:1087B8008831EAE770BD00BFF6940108BC120020BA
:1087C800031EB8BF2D2210B5B8BF58420C46B8BF1B
:1087D80001F8012B0A2204F045F900230370204612
:1087E80010BD07B51C4B03F1A802C3F8A4201B4A0F
:1087F80092F890215AB1012A14D1032183F8AA10C2
:10880800072183F8AC2083F8AB100C2208E0022182
:1088180083F8AA10032183F8AC2083F8AB10072251
:1088280083F8A8200E4B0F4A1A60402001F0B8FACE
:1088380070B10122002390F9000040218DE80C005E
:10884800094A4FF4E13301F087F8003018BF0120DE
:1088580003B05DF804FB00BF181D0020BC12002007
:1088680008000020D91C01086D1E01080120002104
:1088780007F082BBF0B51C4A92F8AD30D2F8B05080
:1088880092F8B47092F8C06092F8CCE0022B0ED83F
:1088980005EBC304591CA31CC9B206D02346A488FF
:1088A80014F0010F01D0204205D10B46EEE782F803
:1088B800AD300020F0BD93F902307CB29C4201D16A
:1088C800002307E074B29C420CD04FFA8EF49C420D
:1088D800EBD1022382F8AD100C2101FB0322D2F860
:1088E800B800F0BD0123F5E7181D002030B50022BF
:1088F80002F1805303F5B8539B0042F400441D680D
:1089080040F60F7144F08004294001322143042AC3
:108918001960EDD1024B40F08000186030BD00BFF7
:108928004C5C00402DE9F843324D6E68328A377A44
:10893800BAB9042F15D130480378012B0CD12F4B2D
:1089480019682F4B89B20B445B0019681A603023F1
:10895800A5F8D830027049E01023A5F8D8300727C9
:1089680044E0B48AB369A24294BF04270227944220
:1089780028BF14461FFA84F8404698471F4A1368D0
:108988009BB203F1005303F540535B0004F1010E61
:108998001B689BB203F1005303F540534FEA6E0E78
:1089A8005B000021714500F1020009D010F8019C1C
:1089B80010F802CC4CEA092C23F821C00131F1E768
:1089C80012680F4B92B213445B001A681C60338A1A
:1089D800C8EB03033382738A98443023A5F8D83050
:1089E8004FF44053A6F81280A5F8DA306B681F726E
:1089F800BDE8F883181D0020B82D0020505C004009
:108A0800023000200E4B0F4A1B689BB203EBC000DC
:108A180002443E294FEA420209D94B09C80604BF5D
:108A280003F1FF339BB29B0243F4004304E04B087D
:108A3800C90748BF01339B0211681360704700BF24
:108A4800505C00400630002008B50B4B002093F81E
:108A58003010FFF7D7FF094B5A68107A082801BF72
:108A68004FF48052A3F8DA201022A3F8D820A0F1FE
:108A780009035842584108BD08000020181D00206D
:108A880038B5444D6A68107810F07F0004D1537AE5
:108A980023F02003537238BD022879D15388002B64
:108AA80077D11379002B74D1537923F08000840097
:108AB80004F1804101F5B84113F0800F096814BF33
:108AC80001F0300101F44051032861D800295FD03A
:108AD800927A002A5CD004F1804404F5B84419065F
:108AE800226825D502F03002102A4CD103F07F030A
:108AF8009B0003F1804303F5B8431A68510641BF50
:108B0800196840F60F720A4042F4004244BF42F02E
:108B1800C0021A601A6822F4E04222F0400292B2BF
:108B280082F0300242F4004242F080021A602AE0E9
:108B380002F44052B2F5805F25D128B9164B93F85C
:108B48003010FFF75FFF11E09B0003F1804303F54E
:108B5800B8431A68520441BF196840F60F720A40B8
:108B680042F4404244BF42F080021A60236823F472
:108B7800804323F070039BB283F4405343F40043D3
:108B880043F080032360AB685B699847002038BDD9
:108B9800022038BD181D00200800002000230360B3
:108BA800436083608381036143618361C3610362BE
:108BB8004362836270478A68036810B50C6A14437D
:108BC8000A6914434A6914438A691443CA691443F5
:108BD8004A6A14438A6A23F4FF4323F0700322434A
:108BE800134303608B8943600B6883604B68C360E1
:108BF80010BD02684FF6FE73134003600023036044
:108C080043608360C360294B984201D1284A27E01A
:108C1800284B984201D1264A2AE0274B984201D195
:108C2800234A2DE0254B984201D1214A30E0244BBC
:108C3800984201D11E4A33E0224B984204D11C4A83
:108C4800536843F470032EE01F4B984204D1184A2E
:108C5800536843F0706326E01C4B984204D11C4AC9
:108C6800536843F00F031EE01A4B984204D1184A88
:108C7800536843F0F00316E0174B984204D1144AA6
:108C8800536843F470630EE0144B984204D1104AC1
:108C9800536843F4704306E0114B984204D10C4AE0
:108CA800536843F470235360704700BF08000240C4
:108CB800000002401C000240300002404400024014
:108CC800580002406C000240800002400804024044
:108CD800000402401C0402403004024044040240E4
:108CE80058040240036A23F001030362036A70B563
:108CF800446882690D6822F4803222F073021543B9
:108D08008A8923F0020313438A881343134A904243
:108D18000FD002F5006290420BD002F540629042FB
:108D280007D002F58062904203D002F5806290423B
:108D38000DD1CA89CE8823F0080313430A8A24F484
:108D4800407414434A8A23F00403334314438A6863
:108D5800446085614263036270BD00BF002C01401E
:108D68009D4A536803F00C03042B2DE9F04105D00C
:108D7800082B06D099490160B3B916E0974B0360F8
:108D880012E053685468C3F38343991CE30349BF53
:108D9800D36A934B914C03F00F0344BF0133B4FBE8
:108DA800F3F34B43036000E0002351688D4FC1F398
:108DB8000311394491F834500168EDB221FA05F4F1
:108DC80044605668C6F302263E4496F8346024FA96
:108DD80006FEC0F808E05668C6F3C2263E4496F878
:108DE8003460F6B2F440C460D2F82C80C8F304189A
:108DF80008F00F0C07EB4C0C18F0100FBCF844C02F
:108E08001FFA8CFC07D0BCF1000F04D0B3FBFCFCAC
:108E1800C0F810C000E00161D2F82CC0CCF3442C9B
:108E28000CF00F0807EB48071CF0100FB7F8447058
:108E3800BFB204D01FB1B3FBF7F7476100E041614F
:108E4800176BFF065ABF654F87618161176BBF06B5
:108E58005ABF624FC761C161176B7F065ABF5F4F28
:108E680007620162176BFF0506D5994204D1AE422D
:108E780002D14F00476200E04462176BFF0406D539
:108E8800994204D1AE4202D14F00876200E0846269
:108E9800176BBF0506D5994204D1AE4202D14F00E7
:108EA800C76200E0C462176B7F0506D5994204D1FA
:108EB800AE4202D14F00476400E04464176B3F059F
:108EC80006D5994204D1AE4202D14F00876400E032
:108ED8008464176BBF0406D5994204D1AE4202D10F
:108EE8004B00C36400E08464156B3B4BAD0701D1B4
:108EF800046315E01C6B04F00304012C01D1016329
:108F08000EE01C6B04F00304022C02D14FF4004362
:108F180005E01B6B03F00303032B01D12F4B036305
:108F2800146B2D4B14F4403F02D1C0F834E018E024
:108F38001C6B04F44034B4F5803F01D1416310E068
:108F48001C6B04F44034B4F5003F02D14FF40043E5
:108F580006E01B6B03F44033B3F5403F01D11F4BD0
:108F68004363146B1C4B14F4402F02D1C0F838E053
:108F780018E01C6B04F44024B4F5802F01D1816300
:108F880010E01C6B04F44024B4F5002F02D14FF418
:108F9800004306E01B6B03F44023B3F5402F01D1D7
:108FA8000E4B8363146B0C4B14F4401F02D1C0F8B2
:108FB8003CE021E01C6B04F44014B4F5801F01D19F
:108FC800C16319E01C6B04F44014B4F5001F0BD105
:108FD8004FF400430FE000BF0010024000127A0077
:108FE80000093D00080000201B6B03F44013B3F593
:108FF800401F01D1134BC363126B134B12F4400F84
:1090080003D1C0F840E0BDE8F0811A6B02F44002D9
:10901800B2F5800F02D10164BDE8F0811A6B02F449
:109028004002B2F5000F02D14FF4004306E01B6B7B
:1090380003F44003B3F5400F01D1024B0364BDE8CC
:10904800F08100BF00127A0000100240F0B5002342
:109058000E681C460125A54005EA060EAE452BD133
:109068000F797A1E012A15D8856803229A4025EAC5
:10907800020282604D7982689D401543856082882E
:1090880092B222EA0E0282808A798588A2402A4317
:1090980092B28280032205689A40D2431540056047
:1090A80005689F402F430760C7681740CA7902FACE
:1090B80003F547EA0502C2600134102C03F10203EC
:1090C800C8D1F0BD38B52DED048B4A4C0368C4F8FF
:1090D800DC308388A4F8E030013A0D46072A42D8EC
:1090E800DFE802F0040A101822292F35B4F8DC3022
:1090F8000B80B4F8DE3013E0B4F8DE300B80B4F83F
:10910800DC3005E0B4F8DC305B420B80B4F8DE30CC
:109118005B4205E0B4F8DE305B420B80B4F8DC302B
:109128006B80B4F8E0301DE0B4F8DC305B420B80B3
:10913800B4F8DE3012E0B4F8DE300B80B4F8DC307E
:109148000CE0B4F8DC300B80B4F8DE3005E0B4F89D
:10915800DE305B420B80B4F8DC305B426B80B4F8E5
:10916800E0305B42AB80244B93F86430002B3ED157
:10917800B5F9003094ED3C0AD4ED397A09EE103A8D
:10918800B5F9023008EE103AB8EEC88AB5F90430DD
:10919800B8EEC99A28EE000A08EE903AA7EE890AB6
:1091A800F8EEE88AD4ED3F7AA7EEA80A0CF004FCA2
:1091B80094ED3D0AD4ED3A7A288028EE000AA7EE0D
:1091C800890AD4ED407AA7EEA80A0CF0F5FB94EDD5
:1091D8003E0AD4ED3B7A688028EE000AA7EE890A99
:1091E800D4ED417AA7EEA80A0CF0E6FBA880BDEC06
:1091F800048B38BD181D00200800002008B50A4857
:1092080090F8093100EB43030A22B3F8181189B228
:10921800A0F8201100F5947007F009FB80B208F05F
:10922800EBFE024B188008BD181D0020901A002084
:10923800F8B504460E4617460025204620210CF0B6
:10924800E2F90446D0B1013420460CF041FAB0F5F9
:10925800617F05DB40F634039842A8BF184601E059
:109268004FF46170A0F56170192390FBF3F00DB90C
:10927800307000E070703B7801333B700DB9012508
:10928800DBE72046F8BD30B505460C4613462946AF
:1092980022460248BDE8304003F0E5BCDC950108F1
:1092A8007FB504780646E4B9354B1B6803EB8403A5
:1092B800192193F87B0093F87C6093F8792093F850
:1092C8007A304FF4617511FB005011FB0651009084
:1092D80001912C482146013403F0C5FC142CE3D13C
:1092E8004BE00CF0F5F91328054641DC244B701CC3
:1092F8001C68202100238DF80F300CF084F91E35EE
:10930800064670B1013630460CF0E2F91A289FBFC4
:1093180004EB850358709DF80F30013398BF8DF822
:109328000F30304620210CF06EF9064670B1013638
:1093380030460CF0CDF90D289FBF04EB85039870DB
:109348009DF80F30013398BF8DF80F3004EB85047A
:109358003046E11C0DF10F02FFF76AFF9DF80F3050
:10936800042B0AD0601C002104220CF016F904E03A
:10937800054800211322FFF786FF04B070BD00BF27
:1093880010120020FB95010810960108014806F00C
:1093980099BE00BF16960108F8B50478064674B958
:1093A800304DB5F8C421B5F8C6312F4821460134EF
:1093B80003F059FC042C05F10405F2D1F8BD2B4942
:1093C8000CF0F4F8A8B9274B4FF47A714FF4FA620D
:1093D800A3F8C411A3F8C621A3F8C811A3F8CA2199
:1093E800A3F8CC11A3F8CE21A3F8D011A3F8D22169
:1093F800F8BD30460CF06CF9032805462BD83046EA
:1094080020210CF000F9044630B1013420460CF05C
:109418005FF90126074600E00646204620210CF0A9
:10942800F2F810B9BDE8F840B0E701300CF050F997
:10943800012EF7D1A7F2EE2240F2DC539A42F1D87E
:10944800A0F2EE229A42EDD8064B703503EB850365
:109458009F80D880F8BD064800210322BDE8F84067
:1094680011E700BFBC1200202496010837960108B6
:1094780052A101082DE9FF4104780546002C39D195
:109488007348744D06F01EFED5ED047AF5EE407A69
:10949800F1EE10FA00F0D88021466F4803F0E3FBA4
:1094A80095ED040A684603F073FA01466B4803F029
:1094B800DAFB95ED050A684603F06AFA0146674843
:1094C80003F0D1FB95ED060A684603F061FA014600
:1094D800624803F0C8FB95ED070A684603F058FA9E
:1094E800013401465E4803F0BEFB0C2C05F1100563
:1094F800CAD1A9E05B4905220CF09CF840B9554B4C
:1095080003F1C002002143F8101F9342FAD19BE0F7
:109518002846554904220CF08DF804462846002CAC
:1095280040D120210CF06FF8002800F08D80451CF8
:1095380028460CF076F807464C4B53F824601EB9C1
:109548004B4806F0BFFD7FE028463146FAB20CF0E2
:1095580071F801340028EFD13E4B03F1C0029E465A
:10956800002143F8101F9342FAD1424B03EBC40287
:109578009846D2F804C0BCF1000F04D131463E48E9
:1095880003F071FB57E0002718F834309F42F5DAF2
:109598003B010EEB030563440FCB103585E80F0044
:1095A8000137F1E70CF094F80B28064647DC28460B
:1095B80020210CF028F8054650B10135284603F063
:1095C8005DF9244B03EB061383ED040A012400E044
:1095D8000446284620210CF016F8054648B1013506
:1095E800284603F04BF91B4B03EB061383ED050AE2
:1095F8000134284620210CF006F8054648B101350B
:10960800284603F03BF9134B03EB061383ED060AD8
:109618000134284620210BF0F6FF10B9FFF7B6FEFB
:1096280012E0013003F02AF90A4B032C03EB06166B
:1096380086ED070AF2D11148FFF71CFF04E0104835
:1096480001210C22FFF71FFE04B0BDE8F08100BF26
:109658003D960108BC120020589601085E96010844
:109668008E9E010837960108629601089C8D0108B4
:10967800679601080C95010876960108B7930108CA
:1096880010960108F0B5047887B006461CBB514B0C
:109698001968062303FB0411192091F8CA5091F8A0
:1096A800CB7091F8CE2091F8C9304FF4617610FB59
:1096B800056510FB07600095019091F8CC000290B9
:1096C800C8314548497903912146013403F0CBFA62
:1096D8000C2CDCD17CE00BF0FBFF0B28044672DC81
:1096E8003C4B701C1D68202100238DF817300BF0AF
:1096F8008AFF064680B1013630460BF0E9FF0328A1
:109708009FBF062303FB045383F8CE009DF8173050
:109718009CBF01338DF81730304620210BF073FFC2
:10972800074680B1013738460BF0D2FF0D289FBF9E
:10973800062303FB045383F8C9009DF817309CBF28
:1097480001338DF8173006266643A9193846CA3101
:109758000DF11702FFF76CFD20210BF054FF0746AF
:1097680070B1013738460BF0B3FF14289FBF9DF83E
:1097780017307619013386F8CC0098BF8DF817306A
:10978800384620210BF03FFF78B101300BF0A0FFE5
:109798000D289FBF062303FB045383F8CD009DF8D3
:1097A80017309CBF01338DF817309DF81730062B02
:1097B8000ED0062202FB04500021C9300BF0EDFE4A
:1097C800FFF7E4FD04E0054800210B22FFF75BFDED
:1097D80007B0F0BD1012002082960108109601080B
:1097E8002DE9F347047807464CB9204601A9FEF74E
:1097F800E7FF0134FFF7F4FF122CF6D179E00BF004
:1098080067FFC5B2112D6FD8781C20210BF0FBFE25
:10981800394C3A4F05F1D006034614F8168030B992
:10982800A8F10202D2F1000848EB020843E000F177
:10983800010A597838460BF0E6FE60B1032D8CBF5B
:1098480003230023C01B3B4453FA80F090F8049094
:10985800B9F1030F02D1FFF799FD4AE0A9F102031C
:10986800D3F1000850464FF0200148EB03080BF0F5
:10987800CAFED8B1B8F1000FEDD001300BF028FFC7
:1098880040F2ED2380B2984205DD40F6CA039842C3
:10989800A8BF184601E040F2EE2004EB4603A0F210
:1098A800EE20192290FBF2F0587002E0B8F1000F98
:1098B800D1D104F8169014F81630FA5CB8F1000FFC
:1098C8000DD00D4B0E4803EB46062946737840F23F
:1098D800EE24192505FB034303F0C5F909E02946E1
:1098E800084803F0C0F904E0074800211122FFF7F7
:1098F800CAFC02B0BDE8F087BC120020047601085B
:10990800A2960108B496010852A1010810B50446B0
:10991800204606F07DFF18B90A2006F0BAFEF7E7E0
:1099280010BD0C4B5A6882421A4607D01B69834205
:1099380006D0D36983420BD1022302E0002300E062
:1099480001230021C1620C2000FB03231972596016
:10995800704700BFCC1D00202DE9F04F06468A480D
:1099680090F9004087B0B44288469DF844501146AB
:109978001A469DF8403009D090F90C40B44207D0FF
:1099880090F91840B44209D1022702E0002700E00C
:1099980001270C2404FB0700047A0CB10020EFE037
:1099A800012E00F0DC80142E05D0002E40F0E78058
:1099B80000957648D5E0DFF814A2DAF8183043F0BD
:1099C8000103CAF81830DAF814304FF0904543F420
:1099D8000033CAF814304FF0010903224FF4805BBA
:1099E80004A94FF090408DF815200392CDF810B0DF
:1099F8008DF814908DF816908DF81740FFF726FB18
:109A0800A5F828B0C82006F044FEC5F818B0DAF862
:109A18001430039A43F40033CAF8143028464FF43C
:109A2800C0534FF0020B04A904938DF815208DF84C
:109A380014B08DF816408DF81740FFF707FB6B6AD6
:109A480023F470436B626B6A43F460436B626B6A26
:109A580023F470236B626B6A43F460236B624C4B94
:109A68004C4D4FF480221A6002F18042A2F53F3239
:109A78001223AB64082385F84D30136885F84E909F
:109A880023F480231360536823F48023536095F8EC
:109A98004C3003F1804303F582331A6842F4802284
:109AA8001A60AA6C3C4B22F01F0002F01F02C1583A
:109AB80009FA02F221EA0202C250AA6C374922F0DE
:109AC8001F0002F01F0250F801E009FA02F22EEA24
:109AD80002024250AA6C22F01F0102F01F02C8586D
:109AE80009FA02F20243CA502D4B2E4A1C60DAF8DA
:109AF8001C3043F40003CAF81C302B4B04A8DA606E
:109B08008DF810608DF811B08DF812408DF8139013
:109B180007F04AFC2A238DF810309DF813308DF891
:109B280011908DF812401BB104A807F03DFC04E029
:109B38001E4B4FF48062C3F884201D4B1D4C1C60E3
:109B4800022385F858301C4A1C4B1D49EB661160EE
:109B58001B6898471B4B2B60A4F1500006E01A487D
:109B6800009503F061FE00283FF418AF064B06711C
:109B78000C2202FB073787F80880786000E020464F
:109B880007B0BDE8F08F00BFCC1D002000380140B1
:109B980014040140C81E0020080401400C040140C0
:109BA800D80042420005FA0500ED00E000E100E0BF
:109BB8001C1D0020181F0020201D00200C00002064
:109BC8007000002010760108004400400010024098
:109BD8000C4B1B6893F90220824209D093F90A20A2
:109BE800824207D093F91220824208D1022002E073
:109BF800002000E0012003EBC00002307047002085
:109C0800704700BFC81D0020F0B5027887B0AAB918
:109C18004C4C04F118064C4B94F9F41193F90020BC
:109C28008A4273D093F90C208A426FD093F9183086
:109C38008B426BD00834B442EDD181E0002204920B
:109C48000592451C0BF044FDC4B260B2FFF7C0FF9B
:109C5800074618B18DF81040012400E00446284654
:109C680020210BF0D0FC054638B1013528460BF011
:109C78002FFD0134ADF81200E4B200262846202159
:109C88000BF0C1FCB0B3451C28460BF021FD0022A7
:109C98002E4951F8223083425FFA82FE04D0013205
:109CA800082AF5D1002300E0734651F823208242A8
:109CB80020D1022E0FD0032E12D05A1E012ED2B25E
:109CC80004D0042A13D88DF814300EE0042A0ED8D4
:109CD8008DF8153009E0052B09D88DF8173004E008
:109CE8009A1E052A03D88DF816300134E4B20136DD
:109CF800042EC3D1052C04D807B0BDE8F040FFF707
:109D080045BB04AB03CB3860796019E094F8F901DE
:109D18000E4B94F8F85153F82000B4F8F62100904F
:109D280094F8FB0153F82000019094F8FA0153F8D5
:109D38002000029053F82530054802F094FF79E797
:109D480007B0F0BDBC120020CC1D0020E075010852
:109D5800C396010838B1438811EA030003D08B4247
:109D68000CBF01200220704730B50B4B0B491C6813
:109D780091F87020022A0BD8134604EBC303551C34
:109D8800EAB29D882842F5D081F87020981C30BD31
:109D980081F87020002030BDC81D0020C81E00209A
:109DA800024B002283F87020DEE700BFC81E0020A7
:109DB8002DE9F047877890F803C0214DBBB2C7F171
:109DC800640E03EB83065C42C3F178005FFA8EFEF3
:109DD8007600CCF16408A4B280B2A3B20FFA83F97A
:109DE800B9F1000F05DC002B14BFBA464FF0010A89
:109DF80000E0F24613FB03F303FB0CF21AFB0AF331
:109E080092FBF3F3434403FB09F30A2293FBF2F3B7
:109E180033449BB225F8023FB1F800904A880A34CF
:109E2800C9EB020AA4B21AB202FB0AF24FF47A731F
:109E3800844292FBF3F34B442B80CED1BDE8F087EC
:109E4800381F00202E4B2F4A1B68126810B51A6065
:109E58002D4A1168596051689268DA602B4A9960F6
:109E680011681961516892689A61294A59611168A3
:109E7800D961516892685A62264A1962118819850F
:109E8800518859859188D288DA85234A998511881D
:109E980019865188598692889A86204A1188D986C7
:109EA800518819871946928821F83A2F1C4A107848
:109EB8000022824206DA1B4C34F8124021F8024F85
:109EC8000132F6E7184A1288A3F86420174A128864
:109ED800A3F86620164A1188A3F86C105188928856
:109EE800A3F87020134AA3F86E1012689A66124AF3
:109EF8001288A3F87220114A5289A3F85E2010BD77
:109F0800F4290020942D0020EC1F0020F81F0020C9
:109F180004200020B4120020F41100209E1200201A
:109F2800C427002014120020381E0020AC10002086
:109F3800FA110020A8120020301200200012002080
:109F48002DE9F8430E4B93E8800305460E4600249E
:109F5800B44213DA7B1933F9140008EB050333F91B
:109F6800142009EB050333F914301344022293FB40
:109F7800F2F3C01A07F0E9F90134E9E7BDE8F8831C
:109F8800F429002070B5472007F02EF9174B1B68FD
:109F98001B0307D5164B174A5B6810681B68C01A65
:109FA80007F0C4F9144E154C154D307807F0BEF97A
:109FB80023682868C01A07F0C8F963686868C01A77
:109FC80007F0C3F90F4B188807F0B0F90E4B188843
:109FD80007F0ACF90D4B188807F0A8F9337823740B
:109FE8002B68A3606B68E36070BD00BF602B002026
:109FF800F4290020942D0020AA1A0020E02900202E
:10A00800AC1A0020A81A0020A61A00203812002036
:10A018007FB5264C264E274D2749284A284B20B184
:10A0280028480088B0F5805F31D23088ADF8040048
:10A0380028781E4D91F8201012788DF806008DF8BA
:10A0480007108DF808201B788DF8093001A82946DB
:10A0580006220BF087FA30B30198BDF80830286063
:10A06800AB80532007F0C0F8208807F05FF9A0788C
:10A0780007F05CF9E37801932379029301A86379E7
:10A08800039307F0B9F80F4B00221A800BE03088D1
:10A09800208091F82010287812781B78A070E17041
:10A0A80022716371DDE704B070BD00BF541F00204A
:10A0B800681B0020A41A0020582D00202B0F002018
:10A0C800900F0020802B0020A0F17D03012B70B59C
:10A0D80004460D460A4E05D830687D2106F0A4FBDB
:10A0E80084F020043068214606F09EFB35B12B88A9
:10A0F8001C4404EB142404F0FF042C8070BD00BF42
:10A10800581B00200A4A138801331380094A136830
:10A1180001331360084A138801339BB2202B01BF17
:10A1280000231380054A138808BF01331380704742
:10A13800802B0020682B00206C2B00206E2B002029
:10A1480038B53A4B1B78083B012B05460C466BD8B3
:10A15800452007F049F8284607F046F80C2D23D08B
:10A1680004D80A2D0AD014D835B138BD0E2D4BD0DD
:10A178002ED3FF2D50D038BD206849E0207807F055
:10A1880033F862796378002A14BF802000201843CE
:10A1980000E0207807F028F8A07807F025F8E078A4
:10A1A80007F022F820793BE0B4F9000007F0B4F892
:10A1B800A07807F019F8E07807F016F8B4F9040069
:10A1C80007F0AAF8B4F90600BDE8384007F0A4B8CB
:10A1D800637820788BB180F0800007F005F8A468D8
:10A1E800E0B207F001F8C4F3072006F0FDFFC4F35E
:10A1F800074006F0F9FF200E12E006F0F5FF606850
:10A20800BDE8384007F0A1B8206807F08FF860680B
:10A21800BDE8384007F08AB8054806F0C3FF0020BB
:10A22800BDE8384006F0E0BF38BD00BFD82900209F
:10A23800E29601082DE9F04FB74BB84F1A888BB05A
:10A248000193002A40F0A380B7F8CA07B44E42F23F
:10A258000103C21A50425041FFF7DAFEFFF7F2FD40
:10A268003468492006F0C0FFAE4B2546186807F051
:10A278005DF855F8040B07F059F82846FEF7EEF993
:10A2880004F11000FEF7EAF904F11C094FF0100878
:10A29800A54D01232A6803FA08F3134203D0D9F81D
:10A2A800000007F052F808F10108B8F1130F09F19E
:10A2B8000409EDD104F12800FEF7C0F9B7F84031E0
:10A2C800B4F92E00C01A07F031F82B68DB0408D562
:10A2D800964BB4F864001B88181AC0F30D0007F0F9
:10A2E80025F82B68980403D5B4F8660007F01EF823
:10A2F8002B68590503D504F16C00FEF79FF92B680C
:10A308001A0502D5A06E07F020F82B681B0403D5A8
:10A31800B4F8720007F00AF804F13000A046FEF71E
:10A328008DF904F13600FEF789F9B7F8403138F9AC
:10A338003C0FC01A06F0FAFF01277D4B1B789F429D
:10A3480008DA38F9020FB4F93C30C01A06F0FDFFFC
:10A358000137F2E72B68980505D5B4F95E00A0F23D
:10A36800DC5006F0F2FF326872487260B260121A6E
:10A378009110714A4A43531C032293FBF2F202EBF9
:10A3880042029A1A742303FB02033360C9E16B4B40
:10A398006B4A1B6811688B4206D00AA9002041F855
:10A3A800203D1360FFF7CCFE019B97F8CA171B8866
:10A3B80097F8CB070B44013BB3FBF0F200FB1233D9
:10A3C8008B4280F07981564C0120FFF721FEFFF780
:10A3D80039FD50202668656806F006FFA2682368E4
:10A3E80010681B68626803441068A3EB400006F01D
:10A3F800ACFF6A6873689B1A0293AA68B3689B1AD1
:10A408000393EA68F36802A89B1A0493FEF726F9F7
:10A418002A6933699B1A02936A6973699B1A0393C1
:10A42800B369AA6902A89B1A049306F0E5FE06F12F
:10A438001C0905F11C0B1027A0463B4801210368A5
:10A44800B9401942824606D0D9F80000DBF800303E
:10A45800C01A06F07AFF0137132F09F104090BF12E
:10A46800040BEAD106F1260005F12601002331F993
:10A47800024F30F9022F121B02AC44F8232001339B
:10A48800042BF4D10322002702ABBF0053F822307B
:10A49800FFB26BB103F108010F2902D847F0010799
:10A4A80006E08033FF2B94BF47F0020747F003070D
:10A4B80012F1FF32E8D2384606F096FE00240DF17C
:10A4C8000809A34607F00302022A10D0032A17D06E
:10A4D800012A4AD1BBF1000F41D0D9F8000000F0A1
:10A4E8000F00204306F080FE4FF0000B3DE0BBF16B
:10A4F800000F0CD0D9F80000C0F3031020432CE063
:10A50800BBF1000F1ED199F8010006F06DFE99F815
:10A51800000006F069FE28E06C2B0020BC12002029
:10A52800F4290020682B0020602B00205C2B0020E1
:10A53800C4270020002A002035C2724F742B002047
:10A54800702B0020D9F80000C0F30330204306F038
:10A558004BFED9F80000C0F3071006F045FED9F805
:10A5680000402401E4B24FF0010B09F1040906ABE5
:10A5780099454FEA9707A5D1BBF1010F02D12046B3
:10A5880006F032FEDAF8003013F480541FBFB6F834
:10A598006420B5F86410521A029218BF0124990475
:10A5A8000AD50AAA02EB8401B5F86600B6F8662057
:10A5B800121A41F8202C01345A0513D502AA02EBCD
:10A5C800840E06F16A0705F16A00002237F9021FB6
:10A5D80030F902CFCCEB01014EF822100132032AE8
:10A5E800F4D103341F0508D50AAA02EB8400A96E2A
:10A5F800B26E521A40F8202C013418040BD50AAB5D
:10A6080003EB8402B5F87210B6F872305B1A42F8A0
:10A61800203C013400E0F4B1012C03D1029806F08B
:10A6280094FE18E0631E002002AA400052F823207E
:10A63800C0B20AB140F0010013F1FF33F4D206F0C2
:10A64800D3FD002702AB53F8270008B106F07DFEC2
:10A658000137A742F6DB30200321FFF771FC3620D3
:10A668000321FFF76DFC314B3C201978FFF768FC9C
:10A67800DAF80030990506D5B6F95E00B5F95E300E
:10A68800C01A06F062FED8F800202948D8F804302D
:10A69800C8F80420121A9110264AC8F808304A430C
:10A6A800531C032293FBF2F202EB42029A1A742320
:10A6B80003FB0203C8F800301F4B1B681A0630D58D
:10A6C8001E4C1F4D22682B689A420BD162686B683A
:10A6D8009A4207D1019B1B88102B11D1194B1B885B
:10A6E8005B060DD1482006F07FFD206806F02DFEA0
:10A6F800606806F02AFE23682B6063686B600EE0D2
:10A70800114A0F4B11782A7C914208D10F4A996857
:10A718001068884203D15268DB689A4201D0FFF77B
:10A7280031FC06F031FD0BB0BDE8F08FC4270020E6
:10A73800002A002035C2724F982900203C120020C0
:10A74800E02900206E2B0020AA1A0020AC1A002055
:10A758002DE9F84F0C9E3A4CC2EB030B0B9BF61AF3
:10A768006368002914BF4FF0060A4FF0040A01334A
:10A778000546904613D1236853455ED2314A324884
:10A7880052F82320032B98BF294606F01BFD636867
:10A79800013363602D4B002205469A7113E00025B2
:10A7A80011E02B4A1278954240DA0B9BE3B109FB82
:10A7B80006F2995C01228A40264909680A4213D1A7
:10A7C800636801336360D4F804900A9B1C4F994571
:10A7D800E7DB2BD10A2006F007FD3B6801333B601D
:10A7E8004FF0FF337B6021E0184A917921B12C208A
:10A7F80006F0FAFC013501E001219171226809FB9C
:10A808000BF308EB030752B958F8030006F0CAFC2B
:10A8180097F904104B1C0544D2D00F4802E03A4483
:10A828000E48117906F0CEFC0544C9E7206850456A
:10A838002CBF00200120BDE8F88F0020BDE8F88F6C
:10A84800782B0020F07A0108ED960108541F0020AB
:10A8580000010020602B0020FC960108A69E01083C
:10A8680030B585B004AC002524F8025D0091ADF840
:10A87800060021461020FFF727FC9DF80600214618
:10A88800FFF722FC9DF807002146FFF71DFC9DF805
:10A8980000002146FFF718FC9DF801002146FFF74C
:10A8A80013FC9DF802002146FFF70EFC9DF80300FB
:10A8B8002146FFF709FC9DF80E00C043C0B22946A7
:10A8C800FFF702FC05B030BD10B5054C206805F057
:10A8D800A8FF18B1206805F0A1FFF6E710BD00BF7A
:10A8E800281B002013B5044601A9006807F056FC90
:10A8F800132007F08FFCBDF9040007F079FC1B203A
:10A9080007F088FCBDF9060007F072FC232007F069
:10A9180081FC2368002BB4BF53204E2007F068FC4D
:10A9280001A9606807F03AFC122007F073FCBDF932
:10A93800040007F05DFC1A2007F06CFCBDF9060066
:10A9480007F056FC222007F065FC6368002BB4BFB3
:10A958005720452007F04CFC02B010BD38B5002444
:10A968000B4D6059254405F0ADFB696811B10948E4
:10A9780002F079F9A96811B1074802F074F907489B
:10A98800103405F09FFBB4F5D87FE9D138BD00BF7E
:10A99800087B010820970108269701084C9F0108A9
:10A9A800F0B585B004460AF03CFE082826D1621EA0
:10A9B800E01D1F4912F8013F09681944497801F060
:10A9C8000301022908BF203B82421370F1D12546BA
:10A9D80004F1080715F8016B164831460AF013FE12
:10A9E80020B1284631460AF00EFE10B1FEF7CEFC23
:10A9F8001CE0BD42EED12046FDF7C4FE0E4805F02E
:10AA080061FB00230D4A1A4404A992F888210A44DC
:10AA18000849595C02F80C1C0133082BF2D10023B9
:10AA280007488DF80C3001A902F01DF905B0F0BDFA
:10AA380004010020F69401082C970108BC1200209C
:10AA48008E9E0108234B244C1D68206880B5FEF7B4
:10AA58005DFF2846FEF75AFF206841798B0704D42A
:10AA6800036841F002015B6998471C4B4FF4885218
:10AA78001A854FF488421A85206805F0D2FEA0B1E5
:10AA8800164E4FF48853B361134B186805F0C6FE91
:10AA98000746FDF7B9F808B104F0BCFA284639466C
:10AAA80005F0C2FE4FF488533385284605F0B9FEF9
:10AAB8000028E1D0094ED4F800804FF48847B761E8
:10AAC800284605F0ABFE0146404605F0ADFE378549
:10AAD800D2E700BF442700205C1F00200010004878
:10AAE8002DE9F04705460AF09CFD314E0446D6F89C
:10AAF800088090B92F4805F0E5FA2F4B53F8241039
:10AB080049B10123A34013EA080F02D02B4802F0F1
:10AB1800AAF80134F1E72A4822E0284629492246C2
:10AB28000AF088FD58B92848284C05F0CBFA54F8A3
:10AB3800041F0029EFD0214802F095F8F7E72B7899
:10AB48002D2B03BF013504F1FF344FF0010A4FF0FC
:10AB5800000A4FF00009184B53F8297027B91C4810
:10AB6800BDE8F04705F0AEBA2846394622460AF055
:10AB780061FDC8B9012000FA09F0830501D515481F
:10AB8800EEE7BAF1000F03D002F096F9124803E09D
:10AB980040EA0800B060114805F094FA39461048B8
:10ABA800BDE8F04702F05FB809F10109D3E700BF3B
:10ABB800BC12002032970108B87C01083C970108B4
:10ABC8004C9F01084097010845970108B47C01088B
:10ABD80067960108519701085F970108689701086F
:10ABE8008D9E010810B5084805F06CFA074B002443
:10ABF8001C715C63064B1C7005F0A4FF05F046FC55
:10AC0800044B1C6010BD00BF709701085C1F00203A
:10AC1800B92D00204427002070B5064600240B4BB0
:10AC2800E518AA8816420AD0E158094802F01BF82C
:10AC38002846002105F0D3F9064805F043FA1434F4
:10AC480040F644439C42EAD170BD00BF58810108D8
:10AC58009C9701084C9F0108F0B504788BB0054615
:10AC68000CB1002436E04B4B19680E2303FB04118A
:10AC780001F58C70B1F91D51B1F91921B1F91B31E8
:10AC8800009591F82051019591F82151029590F97C
:10AC98000700039001F590713F4891F90210049163
:10ACA8002146013401F0DFFF082CDCD170E02D2BA8
:10ACB80014D1072C1BDC28460AF00AFD0AAB661CD7
:10ACC80003EB440424F8100C15F8013F303B092B22
:10ACD800FAD934462B78002BE9D104E0A3F13002ED
:10ACE800092A09D8E5E7082CBDF8182009D00BB0C7
:10ACF800BDE8F040FEF74ABB202BF8D101352646C7
:10AD0800E7E7072AF3D8BDF81A00224BA0F2EE2194
:10AD180089B240F2DC55A9421B68E8D8BDF81C107E
:10AD2800A1F2EE24A4B2AC42E1D8BDF81E6004B290
:10AD380037B2A742DBDB0DB2AF42D8DCA542D6DB87
:10AD4800BDF8247007F16404A4B2C82CCFD8BDF8AC
:10AD580026E00FFA8EF4112CC9DCBDF82050B42D72
:10AD6800C5D8BDF82240B42CC1D812B24FF00E0C91
:10AD78000CFB0233A3F81901A3F81B11A3F81D61FA
:10AD880083F8205183F8214183F81F7183F822E169
:10AD98000BB0F0BD10120020A6970108F0B50446CC
:10ADA8008FB020460AF03DFCC5B225BBAF48B04C79
:10ADB80005F088F994F8D21009B9AE4854E049B2C0
:10ADC80094F8D02094F8D130009194F8D3100191E0
:10ADD80094F9D410029194F9D510039194F8D610EF
:10ADE8000491A5482946013501F03DFF102D04F1D5
:10ADF8000704DFD1E1E72046A04905220AF01AFC42
:10AE08000546B8B929469E4870220AF0C6FB9D4BF4
:10AE1800196828460E2303FB001301300022082876
:10AE280083F8232183F8242183F8252183F8262118
:10AE3800F0D119E12046944904220AF0FBFB0546AB
:10AE48002046002D4AD120210AF0DDFB002800F021
:10AE58000B81461C30460AF0E4FB2C4607468B4B18
:10AE680053F824502DB98A480FB0BDE8F04001F0DE
:10AE7800FABE30462946FAB20AF0DCFB0134002853
:10AE8800EDD17B4A02F170011646002382F8D630D4
:10AE980082F8D23082F8D13082F8D03007328A4234
:10AEA800F3D17C4901EBC40191F80822934210DAEE
:10AEB800D1F80C72C3EBC302B0183A4400F1D001C8
:10AEC8001768C0F8D0709088888092798A710133A9
:10AED800E7E72946704801F0C6FE96E06F49072269
:10AEE8000AF0A8FB05462046002D4AD120210AF089
:10AEF8008AFB06460AF095FBC4B274BB684801F0A9
:10AF0800B2FE21466748013401F0ADFE0E2CF8D19F
:10AF1800584801F0A8FE00246348214601F0A3FE2A
:10AF28000025584A614811680E2202FB04120123C9
:10AF3800D2F823215E49AB4013425E4B05F101056F
:10AF480008BF194601F08FFE0E2DEAD14948013499
:10AF580001F089FE082CDFD186E0304656490AF018
:10AF6800BBFB2C46002852D0022C55D00AF0B0FB6F
:10AF780006AB514943F8240000200AF0ADFB013428
:10AF8800F0E74D490AF0A8FB002460B1082C3ED038
:10AF98000AF09EFB06AB484943F8240000200AF05B
:10AFA8009BFB0134F1E7082C31D1069B0F2B2ED8DF
:10AFB800DDF81CE0BEF1070F29D8089F0D2F26D811
:10AFC800099E06F16402C82A21D80A9DFF2D1ED8C1
:10AFD8000B9864281BD80C99642918D8884216DA6B
:10AFE8000D9C032C13D8224AC3EBC303134483F8E4
:10AFF800D0E083F8D17083F8D26083F8D35083F817
:10B00800D40083F8D51083F8D6402C4CC9E60FB08D
:10B01800BDE8F040FEF7BAB9069B072B20D8079980
:10B028000D291DD80278722A0DD06E2A18D1154A1A
:10B0380012680E2000FB032301228A40D3F8231153
:10B0480021EA020209E00F4A12680E2000FB0323DE
:10B0580001228A40D3F823110A43C3F8232101E0CF
:10B06800FEF794F90D4C9CE60FB0F0BDCE970108A1
:10B07800BC1200204C9F0108F99701083796010877
:10B088008C13002010120020629601089C8D010884
:10B0980067960108087B010876960108C69701089B
:10B0A8002A97010815980108A69E01081A98010810
:10B0B80085A201083FA301081E980108B79301085B
:10B0C8002DE9F743047805468CB9324D95F89F125F
:10B0D800B5F89C2295F89E322F48009121460134FC
:10B0E80001F0C1FD102C05F10405EFD14EE00AF086
:10B0F800EFFA0F28044636DC284620210AF083FAA6
:10B10800264EE4B2D6F83880451CA400002728460D
:10B118000AF0DEFA5FFA87F9B9F1010F83B208D0B5
:10B12800B9F1020F0BD0B3F5B47F24D2B26B13532D
:10B138000AE0FF2B1FD8B36B2344987004E0FF2B61
:10B1480019D8B36B2344D87028462C210AF05BFA2F
:10B15800054608B1013502E0B9F1020F0BD10137FC
:10B16800032FD4D112E00E4800210F2203B0BDE80E
:10B17800F043FEF788B808EB0400002104220AF027
:10B188000CFA03B0BDE8F043FEF700B903B0BDE820
:10B19800F08300BFBC120020209801085C1F00202B
:10B1A800109601082DE9F04304788FB00546002C6D
:10B1B80059D17C4B0021142209A807AED3F83C8052
:10B1C8000AF0EBF90722304600210AF0E6F905A853
:10B1D8000023A700059308EB070583801A467249E8
:10B1E800B5F802E031F813C01CEA0E0F0AD00DF1D1
:10B1F800380C0E3102F1010E6244595C02F81C1C35
:10B208005FFA8EF20133072BE9D100210B46674A1A
:10B21800B5F802E011F802C01CEA0E0F0AD00DF1D1
:10B22800380C063203F1010E63448A5C03F8242CBF
:10B238005FFA8EF301310629E9D118F807305C4925
:10B248008DE841006A78029209A81A0903F00F03F1
:10B2580006F008FB2146574809AA013401F003FD0E
:10B26800202CA6D19BE00AF033FA1F28044600F3ED
:10B27800898028462021E4B20AF0C5F91F2C02D99A
:10B28800FEF784F88BE0474BDB6B03EB8404451C2B
:10B298000021204604220AF080F90027464B09AE17
:10B2A800304600210A2217F803905FFA87F80AF05F
:10B2B80074F9002315F8012B32B10A2B04D04A4542
:10B2C80002D0F2540133F5E74A4561D108F1FF3362
:10B2D800032B09D8DFE803F0100502420DF1230023
:10B2E80037E00DF123011FE030460AF0F1F9237829
:10B2F800C0B243EA001006E030460AF0E9F92378C4
:10B3080000F00F001843207034E00133062B0BD0F7
:10B318002A4800F2F3269E5D9642F6D1034493F83C
:10B32800ED2263881343638011F8012F12B30023C1
:10B33800EEE70133072B0CD0204A02F2E6269E5D89
:10B348008E42F6D102EB4303B3F8D8226388134345
:10B35800638010F8011F69B10023EDE730460AF059
:10B36800B7F90F2804DC30460AF0B2F9607001E042
:10B37800002363700137052F90D1012403F0F0FDFD
:10B388006CB97DE70E4800211F22FDF77CFF06E01F
:10B398002046002104220AF000F90024EEE70FB04D
:10B3A800BDE8F0835C1F0020E07D0108F57D010801
:10B3B8003498010843980108017E0108087B0108B8
:10B3C800109601082DE9F0412DED048BB1498AB0A2
:10B3D80004460AF0EBF8B049002820460CBF0126C5
:10B3E80007260AF0E3F8AD490028204608BF0226E0
:10B3F8000AF0DCF8002808BF0426F10740F1EF80C6
:10B40800A748A84C04F05EFE002004F067FCA6489C
:10B4180004F058FEA54804F055FE6379A44AA548EF
:10B42800013B254652F8231001F01DFCA24801F00B
:10B438001AFC4FF00008274695ED048AB5EE408ABD
:10B44800F1EE10FA04D19D4801F00DFC002570E0E2
:10B458009B48D5ED059A95ED069AD5ED078A4146A4
:10B4680001F001FCB5EEC08AF1EE10FA02D52020F9
:10B4780004F020FEB0EE480A06A801F089FA014659
:10B48800904801F0F0FBF5EEC09AF1EE10FA02D503
:10B49800202004F00FFEB0EE690A06A801F078FA41
:10B4A8000146884801F0DFFBB5EEC09AF1EE10FACC
:10B4B80002D5202004F0FEFDB0EE490A06A801F0EE
:10B4C80067FA01467F4801F0CEFBF5EEC08AF1EE3F
:10B4D80010FA02D5202004F0EDFDB0EE680A06A8A7
:10B4E80001F056FA08F101080146774801F0BBFB64
:10B4F800B8F10C0F05F110059ED1A4E749B294F8F4
:10B50800D02094F8D130009194F8D310019194F997
:10B51800D410029194F9D510039194F8D61004919F
:10B528006A482946013501F09EFB102D04F10704F5
:10B5380003D094F8D2100029E0D16548654C04F096
:10B54800C1FDD7F8088054F8041F19B1624801F00A
:10B558008AFBF8E70D46614B53F8254054B10123A7
:10B56800AB4013EA080F03D05D48214601F07BFB8E
:10B578000135F0E75B4804F0A5FD21467B180AAACF
:10B5880093F888311344584A8A5C03F8102C013127
:10B598000829F3D1002306A954488DF8203001F07A
:10B5A80062FB534804F08EFD5248FEF72DFB5248CB
:10B5B80004F088FD4F48FFF7F5FD504804F082FD80
:10B5C8004C48FFF77DFD4E4801F04DFB4020FFF74A
:10B5D80023FB4C4804F076FD4648FEF701F9B20714
:10B5E80039D5494804F06EFD484804F06BFD4148E0
:10B5F80004F0B4FB464804F065FD3E48FDF750FEF4
:10B60800444804F05FFD3B48FEF73CF8424801F02F
:10B618002AFB3848FDF7C0FE404804F053FD354882
:10B62800FFF71AFB00270E257D4300243C4A126CC5
:10B638002A440123D2F80A20A34013421ED1013420
:10B648000E2CF3D10137082FEDD12D4801F00BFB5B
:10B658008020FFF7E1FA730716D5324804F032FD6F
:10B66800314804F02FFD234804F052FB244801F030
:10B67800FAFA4FF48070FFF7CFFA05E03946224610
:10B688002A4801F0F0FADAE70AB0BDEC048BBDE80D
:10B69800F08100BF4F9801085F9C01085698010887
:10B6A8005C980108BC1200206A9801087C9801087F
:10B6B8009C8D01088898010893980108A0980108B2
:10B6C800AD980108299701088E9E0108C5980108C0
:10B6D800B5980108B47C0108E4980108B87C010811
:10B6E800F2980108FF980108F69401080B990108DF
:10B6F80014990108B7930108239901082F990108A3
:10B708004C9F01083D9901084A9901085D99010873
:10B718006B990108759901088499010892990108A3
:10B728005C1F00209E990108AF990108C199010882
:10B73800D0ED024A91ED016A90ED015A91ED027A3D
:10B74800D0ED005AD1ED007A66EE646AE5EE076A3C
:10B7580027EE657AC2ED006AA4EEA77A67EEC57A8D
:10B7680082ED017AE5EE867AC2ED027A7047D0ED75
:10B77800017A91ED017AD1ED026A91ED006A37EE16
:10B78800877AD0ED027A77EEA67AD0ED006A82ED5C
:10B79800017A76EE866AC2ED027AC2ED006A7047D7
:10B7A80090ED017AD0ED027AD0ED006A20EE077AAA
:10B7B80060EE277A26EE800A81ED017A81ED000A93
:10B7C800C1ED027A70472DE9F04F2DED028B85B05F
:10B7D80080460293924B1B889807934637D5109B57
:10B7E8009048DC89B0F900301B1B03F2F31540F2D6
:10B7F800E632954203D8002BB8BF5B4201E04FF414
:10B80800FA73B0F90220121B02F2F31440F2E63088
:10B81800844203D8002AB8BF524201E04FF4FA72BA
:10B828009342B8BF1346C3F5FA73052293FBF2F3AC
:10B838000A22643B534398F81C20D21053436422D5
:10B8480093FBF2F3134423EAE373DBB200E06423CF
:10B858000093CB1C019347460025019BDFF8E4A128
:10B8680013F8016F0193022D4FEA450905D1BAF982
:10B8780004301B365E43761148E06B493AF81520D0
:10B8880031F91510022012FB0011CBF10002914290
:10B8980003DB59450A46A8BF5A466449029B31F959
:10B8A8000940141B33F91520144402F015FC88B123
:10B8B80007EE904A5E4AB8EEE70AB2EE048A505D97
:10B8C80080EE080A05F0BAFD20EE080AFDEEC07AFF
:10B8D80017EE904A524A1288D10713D43AF9093020
:10B8E8001B365E4393074FEA26160FD598F8123099
:10B8F8005C439DF900305C43642394FBF3F406EB4E
:10B90800241603E098F8086074432611494B042470
:10B9180033F9093093FBF4F4341B474EAB5D9A4678
:10B928007B78524663435343022D4FF0640293FBE6
:10B93800F2F34FEAE31308EE103A304609D1B8EEB5
:10B94800C80A04301E21D6ED030A00F06DFFBDEED3
:10B95800C08A394A308AFE7A02F1140E00FB04F3D9
:10B968005EF82510DB1206FB0316B6F5001F334BF5
:10B97800A8BF4FF4001602F120019E42B8BF1E4630
:10B9880051F8253041F82540E31A4FF6FF710009B8
:10B99800B1FBF0F098F850104EF825605843831129
:10B9A8004FEA850C761300EE103A79B102F12C00BB
:10B9B800B8EEC00A00EBC500D2ED030ACDF80CC002
:10B9C80000F032FFDDF80CC0BDEEC00A7B7D10EE42
:10B9D800102A18EE101A534352465A43134631445C
:10B9E800642293FBF2F3164A1B12194422F8091039
:10B9F80018EE100A02F1080101354CF8010002F1B5
:10BA080014012032032D4CF801604CF8023007F184
:10BA180001077FF422AF05B0BDEC028BBDE8F08FC3
:10BA2800681B0020782C0020B02D002090290020D1
:10BA3800C47E0108F4110020A01F00200000E0FFD0
:10BA4800E41F0020B41200202DE9F04F2DED0A8BE1
:10BA580085B08246039390F85030029190461BB10E
:10BA6800322BA8BF322300E0012307EE903AB8EE4C
:10BA7800E7BADFEDD97AD94BDFEDD9BA1B88D94CB3
:10BA8800019487EE8BBA002B08BF0123D64D07EE31
:10BA9800903AF8EEE79A238869EEABBA13F0020FF2
:10BAA8003BEE2BBA8BEE8BBA26D0B5F90030B5F940
:10BAB800022083EAE37182EAE270A1EBE371A0EB72
:10BAC800E27088420646B8BF0E46B6F5E17F16DA40
:10BAD8008842DFEDC6AA05DD002AD8BF524207EE2C
:10BAE800902A04E0002BD8BF5B4207EE903AF8EEAC
:10BAF800E77AC7EEAAAA04E0DFEDBDAA01E0F7EEF7
:10BB080000AA9FEDBB9ABB4C56464FF0000BB0EE17
:10BB180049AADFF8189339F91B300CEE103AB8EE41
:10BB2800CCCAF5EE047A35F91B302CEE27CA08EE9C
:10BB3800903A019BBDEECCCA1988F8EECC7A9FEDFD
:10BB4800AECA89074FEA4B0727EE8CCAF8EEE88A97
:10BB580000F08580A94931F91B3007EE903AF8EEDC
:10BB6800E77AB0EE007AE8EE877AC8F10000FDEED9
:10BB7800E77A17EE901A814203DB4145A8BF414698
:10BB880008469F49039B795E401A33F91B10084405
:10BB980007EE900AB8EEE78A02F09EFA50B199498A
:10BBA800B2EE049A88EE090A11F80B0005F046FC7B
:10BBB80020EE098A9AF81C30DFED936A0AEE103AF3
:10BBC8009AF8083007EE903AF8EE677AB8EE4AAA83
:10BBD80068EE277AB1EE047A67EEA67A2AEE077A3B
:10BBE800FDEEE77A17EE901AF1EE477ABDEEE7AA76
:10BBF8001AEE103A994208DBBDEEC7AA1AEE103ABF
:10BC08008B42A8BF0B460AEE103A804901EB8B0124
:10BC1800D1ED007AE8EE2B7ABBEE0E7AF4EEC77A15
:10BC2800F1EE10FAB8EECAAA09D4B3EE0E7AF4EE21
:10BC3800477AF1EE10FAC8BFF0EE477A01E0F0EE6D
:10BC4800477AC1ED007A9AF8123009EE103AB8EE48
:10BC5800499A67EE897A9FED6E9A27EE899A019B39
:10BC68001988CA0750D439F907000028B8BF4042DC
:10BC7800B0F5206F02DD0020206025E09FED657A99
:10BC8800737868EE877A07EE103AB8EE477A87EE4F
:10BC9800877AD4ED007A37EE4C7AE7EE2B7A9FED6F
:10BCA8005E7AF4EEC77AF1EE10FA09D49FED5B7A6A
:10BCB800F4EE477AF1EE10FAC8BFF0EE477A01E0E9
:10BCC800F0EE477AC4ED007AF37AD4ED007A08EE04
:10BCD800103AB8EE488A8B0768EE277A9FED508AAB
:10BCE80027EE888A14D578EECA8AF0EE4A7AEAEE08
:10BCF800A87A38EE498AF0EE678AF0EE497AEAEED9
:10BD0800887AB0EE678A03E0B0EE498AF0EE4A8A94
:10BD1800DFF81C919FED437A09F1840109F188004D
:10BD28001BF8013007EE903AF8EEE77A4FEA8B01FC
:10BD380067EECC7A0844E7EE878A0434013690ED42
:10BD4800007A80ED00CA3CEE477A09F1900087EE50
:10BD58002B7A0144D1ED007A37EE677AF0EE68CAA3
:10BD6800EBEE077A3CEE880AC1ED007A09F19801FA
:10BD78001BF8013008EE903AF8EEE88A67EEA87AE8
:10BD8800DFED298A67EEA88A30EE680A09F014FE0A
:10BD980009F14401FDEEECCAC8531CEE903A09F1D2
:10BDA8004C01BDEEC88AF1EE688A41F82B30FDEEF1
:10BDB800E88A09F1580118EE103A41F82B3009F1D8
:10BDC800640118EE903A4F4641F82B30BBF1000F52
:10BDD80030D14FF0010B9CE683F9223EC8110020B8
:10BDE800BD378635681B0020B41200200000E143EF
:10BDF8000000000010200020CDCC4C40B02D0020C9
:10BE080090290020C47E01086F12033C1C200020EA
:10BE18000AD7A33D0000A043000040C300004043F0
:10BE28000AD7233CA69B443BF7CC9238F411002058
:10BE3800A01F0020029AB5F90430947964002834D0
:10BE48005C434B4BB3F9043000EE103ABAEECF0A1C
:10BE580009F0B2FD6411201A002C07EE900AB8BF51
:10BE68006442322CF8EEE76A03DD0023C9F81C307F
:10BE780029E0FDEEE99A19EE903A23F0030307EE64
:10BE8800903AF8EEE79ADFED3B7A9AF80D30C9EE72
:10BE9800A77A07EE103AB8EE477AD9F81C3026EEA2
:10BEA800877A67EE277AFDEEE77A17EE902A134431
:10BEB800314A9342A8BF1346304A9342ACBFC9F8EF
:10BEC8001C30C9F81C20FB695B13B3F5807FA8BF41
:10BED8004FF480736FF0FF029342B8BF134607EE2A
:10BEE800903AF8EEE78AFDEEE67A9AF8032017EE24
:10BEF800903A53439B1107EE903A214B1B78032B42
:10BF0800B8EEE78A14D9BAF84E20B2F5FA7F0FD204
:10BF1800FDEEC87A534217EE901A994204DB91421B
:10BF280017EE903AA8BF134607EE903AB8EEE78AA4
:10BF380038EE280ABDEEC00A8DED010ABDF90430BD
:10BF480000EE103AB8EEC00A09F036FDBDEEC88A18
:10BF5800FDEEE88A0023A7F8480087ED158AC7EDAB
:10BF6800188AFB6605B0BDEC0A8BBDE8F08F00BFF0
:10BF7800F411002000803B45FEFFFF0F020000F097
:10BF8800C42700202DE9F0472DED0A8B064694B012
:10BF98008B4C94F89B802546B8F1000F0ED0B8F171
:10BFA800010F40F0868304F1E400D4ED376A94ED84
:10BFB800387A04F1F0030021804611E104F042FBD5
:10BFC800D4F8A4209FED7F7AC4F89C00831A07EE6A
:10BFD800903AF8EE677A7C4BC4F8A40067EE877A4B
:10BFE8005B68C4ED287A04F1A800984704F1A80713
:10BFF800002800F0DE80754B38461A783946FDF780
:10C0080061F8B4F8AE30002B42D0D4F8B000434603
:10C01800B5F8AE206E4937F913C0DFF8A4E1B2F5E0
:10C02800C87F04BF002241F823204FEA830851F853
:10C038000820624441F80820002127F8131020F84E
:10C0480013100133032BE3D1BEF8AE30012B1AD104
:10C05800DEF8B4304FF4C87CC83393FBFCF202809E
:10C06800DEF8B820C83292FBFCF24280594ADEF86A
:10C07800BC301288C83393FBFCF39B1A8380318051
:10C08800718001F0B9F9B4F8AE30013BA4F8AE30D4
:10C09800514B1B685B0778D5B4F8C020484B322A4F
:10C0A80011D1D3F8B0201188A3F8C2105188928812
:10C0B800A3F8C6203288A3F8C8207288A3F8C41051
:10C0C800A3F8CA2001E0002A3FD0D4F8B01000201D
:10C0D800B5F8C03037F910C0DFF8E480322B3F4B99
:10C0E80004BF002243F820204FEA800E53F80E20A8
:10C0F800624443F80E20002327F8103021F810304E
:10C10800013003281A46E3D1B8F8C030012B17D103
:10C118000C2088F8D82088F8D93004F0EDFAD8F83F
:10C12800B030B8F8C2201A80B8F8C4205A80B8F8DD
:10C13800C6209A80B8F8C8303380B8F8CA307380FF
:10C14800B4F8C030013BA4F8C03094F8DA301C4A87
:10C15800DBB1D2F8B050D2F8CC30002082F8DA0047
:10C16800322193FBF1F32B80D2F8D03093FBF1F31B
:10C178006B80D2F8D430174A93FBF1F312889B1ADC
:10C18800AB803080708001F037F9D4F8B020B4F873
:10C19800A83011885B1AA4F8A8305188B4F8AA30DE
:10C1A8005B1AA4F8AA309288B4F8AC309B1AA4F8A9
:10C1B800AC3094F89B30013384F89B30E8E600BF3C
:10C1C800A01F0020BD37863548270020BA2D002043
:10C1D8005420002004000020982900206C20002012
:10C1E800E04DE14F05F1A80232F8112027F811209F
:10C1F80012B207EE902ADD4AF8EEE77A32F91120FA
:10C2080067EEA67A0131E0EC017A07EE902AF8EEA3
:10C21800E77A032967EE877AE3EC017AE0D105F142
:10C22800F00005F1FC010246FFF7A1FA05F1F00064
:10C2380005F5847102AAFFF79AFA02A895ED280A73
:10C24800DFF820A30146FFF7ABFADDED034ADDED89
:10C25800027A9DED045A95ED484AD5ED473A95ED99
:10C26800453AB6EE007A64EE874A67EE875A64EE7E
:10C27800A47A25EE075AE5EEA57A05A80146B7EE99
:10C28800008AE5EE057A08AA0BAFF0EE482AE7EE39
:10C29800C72A0AF5987965EE846AD5ED467AE2EE02
:10C2A800A36A25EE236AE4EE836A23EEE57AB1EE0B
:10C2B800452AE2EE276AA2EEA76AA4EEA77A67EEFD
:10C2C800E57AF1EE641AE2EE837AA1EE846AA2EED0
:10C2D800847AE1EEA37AA5EE836AA5EE037AE2EE0C
:10C2E800047A85ED466AC5ED457AB1EE466AC5ED34
:10C2F800476A85ED487AF1EE666AB1EE477A8DEDC8
:10C30800077A8DED056ACDED066AFFF730FA95EDEF
:10C31800450A97480EA9FFF743FA05A8944911AAB8
:10C32800FFF706FA11A80EA93A46FFF720FA08A85F
:10C33800394611AAFFF7FCF93A468D4811A9FFF7CB
:10C3480016FA8C4BD5ED497A9DED0D7A1A78B4EE34
:10C35800E77AF1EE10FACCBF42F0080222F00802A8
:10C368001A70D4F828311B78F0EE489A0AF5A075AF
:10C378003BB3DAED4B8A4846B0EE680A0EA9FFF7E0
:10C388000FFA9AED4F8A0AF1E400B0EE480A11A9B3
:10C39800FFF706FA4A460EA811A9FFF7E8F928465A
:10C3A800B0EE680A0EA9FFF7FBF9384611A9B0EEFE
:10C3B800480AFFF7F5F90EA811A92A46FFF7D7F999
:10C3C80007E098E8070089E8070097E8070085E88C
:10C3D8000700D4ED3A7AD4ED396A94ED3B7A614D91
:10C3E80067EEA77A0023E6EEA67AE7EE077A9FEDD6
:10C3F800627AF4EEC77AF1EE10FA06DC9FED5F7A06
:10C40800F4EEC77AF1EE10FA06D5C4F80831C4F88C
:10C418000C31C4F8103112E005F5987005F5A071DB
:10C4280005F58472FFF784F9D5ED287A9FED540A53
:10C4380005F5847080EE270A0146FFF7B1F9B4F8D4
:10C448004C31484D01339BB2B3F57A7FA4F84C3197
:10C458002ED195ED460AD5ED456A95ED477AD5ED8D
:10C46800487A20EE000AA6EEA60AA7EE070AA7EE6B
:10C47800A70A09F01BFD89EE800A0023A5F84C31B4
:10C48800D5ED466A95ED477AD5ED487A95ED456A3A
:10C4980060EE266A20EE077A60EE277A26EE000A1A
:10C4A800C5ED466A85ED450A85ED477AC5ED487ABA
:10C4B800D4ED468A94ED48AA94ED45BAD4ED47AA3E
:10C4C8009FED309A68EECA7AB7EE007AEBEE2A7AD8
:10C4D80077EEA77AF4EEE97AF1EE10FA0EDCFFEEC9
:10C4E800006AF4EEE67AF1EE10FA24D4F4EE477A14
:10C4F800F1EE10FAC8BFF0EE477A01E0F0EE477AA5
:10C5080017EE900A06F014F941EC100B09F0CAFA7C
:10C5180051EC100B06F060F908EE100AB5EEC08A6F
:10C52800F1EE10FA09DD78EE497AF5EEC07AF1EE0F
:10C5380010FA10DC3FE09FED148AF1EE487A77EEAE
:10C54800C97AF5EEC07AF1EE10FAB5EEC08A2FDDA1
:10C55800F1EE10FA22DD38EE499ADFED0C7AB4EEEE
:10C56800E79A1FE0A01F00209E120020F41100206F
:10C57800C87E0108A41A0020B81E8D3F3D0A673FF7
:10C588006F12833ADB0FC93FDB0FC9BF35FA0E3C88
:10C5980035FA0EBC000000004D3D0F441FED057A32
:10C5A800F4EEC77AF1EE10FA4CBF0123002312E033
:10C5B800F1EE10FA06DD38EE499A5FED0B7AB4EE2B
:10C5C800E79A03E01FED0E7AF4EEC77AF1EE10FA5F
:10C5D800CCBF0123002353B1B0EE4A0AF0EE4B0A58
:10C5E80000F06FFB1FED15CA70EE008A41E02AEEDD
:10C5F8008A0A6AEEAABAABEE280AB0EE6B7A30EE77
:10C60800000AA8EEA87AB5EE400AF0EE007AF0EE3D
:10C61800690AF1EE10FAE7EE670AB0EE679A04D1FC
:10C62800F5EE400AF1EE10FA04D000F04AFBB0EE45
:10C6380040CA01E01FED29CA28EEAA0AEAEE0ABAA2
:10C64800ABEE0A0AF0EE690A30EE000AEBEEC90A10
:10C65800B5EE400AF1EE10FA04D1F5EE400AF1EE1B
:10C6680010FA04D000F02DFBF0EE408A01E05FEDF7
:10C67800378A1FED379A154D2CEE090A09F09CF9F7
:10C6880028EE090A288009F097F9DFED117A114A96
:10C69800688068EEE78AFDEEE88ACDED018ABDF88C
:10C6A800043013F4004F18BF03F5B473138000234C
:10C6B80000E00123002284F89B20002B7FF468AC63
:10C6C80014B0BDEC0A8BBDE8F08700BF90290020AC
:10C6D800E12E6542AC12002001380A4B042804D828
:10C6E800DFE800F00507090B0D00074A08E0074AD4
:10C6F80006E0074A04E0074A02E0074A00E0074A62
:10C708001A607047F800002069E70008CFB70008F2
:10C718006DEA000861E4000805E1000851BA000864
:10C72800F0B50124B0FBF4F58D4201D34C43F9E791
:10C738000026D4B1B0FBF4F504FB1500B4FBF1F40A
:10C748001EB9002D01DC002CF3D1092D03F1010ED7
:10C75800EFB204DD002A14BF3725572500E0302545
:10C768003D441D7001367346E3E71C70F0BDF0B51B
:10C778000124B0FBF4F58D4201D34C43F9E70026C0
:10C78800D4B1B0FBF4F504FB1500B4FBF1F41EB909
:10C79800002D01DC002CF3D1092D03F1010EEFB2BD
:10C7A80004DD002A14BF3725572500E030253D4415
:10C7B8001D7001367346E3E71C70F0BD03685A1C10
:10C7C8000260197070472DE9F843089E002B074650
:10C7D8008846144614BF4FF030094FF020093346FD
:10C7E80013F8012B0AB9254603E0002CFBDD013CB8
:10C7F800F6E7002D04DD38464946C047013DF8E715
:10C8080024EAE4743546A01B284415F8011B11B12D
:10C818003846C047F7E7BDE8F883024B186804F0CC
:10C8280003B800BFB810002090ED017A07EE901A07
:10C83800B5EE407AF1EE10FA01BFF8EEE77A9FED17
:10C848000E7A67EE877AB7EE007A04BFC7EE277ACA
:10C85800C0ED017A90ED017AD0ED007A30EE877A5A
:10C8680030EE670AC0EE870AE0EE807AB0EE670A1B
:10C87800C0ED007A704700BFDB0FC94010B50278E1
:10C88800202A034600F10100F9D0092AF7D02D2A01
:10C8980003D10346BFEE000A04E02B2A08BF034673
:10C8A800B7EE000ADFED387A1A46134612F8010B84
:10C8B800A0F13001CCB2092C0AD807EE101AB8EE54
:10C8C800C77AF2EE046AA7EEA67AF0EE477AECE7AA
:10C8D8002E2816D1F2EE046A1146B0EE666A0B46AF
:10C8E80011F8012B303AD0B209280AD807EE102ADD
:10C8F800B8EEC77A87EE267A66EE866A77EE877A8A
:10C90800EDE71A7802F0DF02452A35D15A782D2A48
:10C9180002D10233012004E02B2A14BF0133023371
:10C928000020013B002213F8011F3039CCB2092C3A
:10C9380003D80A2404FB0212F5E7B2F59A7F28BF50
:10C948004FF49A721346B7EE007A072B05D9DFED3C
:10C958000F6A083B27EE267AF7E702F007032BB1A8
:10C96800F2EE046A27EE267A013BF8E7F0EE476A12
:10C9780020B1C7EE877A03E0F7EE006A67EEA67A81
:10C9880020EE270A10BD00BF0000000020BCBE4CEE
:10C9980030B52DED028B87B0B0EE408A0C22002115
:10C9A800054603A808F0F9FDB5EEC08ADFED2A7A3E
:10C9B800F1EE10FACCBF38EE278A38EE678ADFED41
:10C9C800277A28EE278A6946FDEEC87A17EE904A3C
:10C9D80084EAE470A0EBE470FBF7F2FE002CACBF35
:10C9E80020232D2368468DF80C3008F01AFE012804
:10C9F80007D130238DF80D308DF80E308DF80F30BB
:10CA08000CE0022805D130238DF80D308DF80E305A
:10CA180004E0032804BF30238DF80D30694603A8CD
:10CA280008F0E2FD03A808F0FCFD0338C4B2224672
:10CA380003A9284608F022FE00232B55284608495A
:10CA480008F0D2FD03AB2846191908F0CDFD284699
:10CA580007B0BDEC028B30BD6F12033A00007A4478
:10CA6800D09D010870B5064615460846B6FBF2F497
:10CA780014B12046FFF7F6FF05FB1464024B1B5D5B
:10CA880000F8013B70BD00BFD29D01082DE9F04FB1
:10CA9800814689B08A4616461C4600253178002909
:10CAA80000F0DD80252902D00136484675E072780D
:10CAB800302A08BFB278A2F1300319BFB71C4FF073
:10CAC800000BF71C4FF0010B092B4FF0000819D889
:10CAD800A2F13003D9B2092905D80A2202FB083885
:10CAE80017F8012BF4E7A2F16103052B02D8A2F194
:10CAF800570305E0A2F14103052B03D8A2F1370340
:10CB08000A2BEADD6C2A31D13A78642A07F101064A
:10CB180000F083800BD8252A3DD003D8002A00F0E6
:10CB28009E80BBE7582A0CD0632A19D0B6E7732A2F
:10CB380022D002D86E2A37D0B0E7752A5CD0782A7E
:10CB4800ACD1271D2068A2F1580462424FF01001B1
:10CB5800624155E02CD9582A32D0632A2AD13E4660
:10CB680048462178271DD04701350FE0642A64D054
:10CB78000ED9732A14D13E4623680093484651467D
:10CB880042460023FFF71FFE271D05443C4685E764
:10CB9800252ADFD13E4648462521D04701357DE785
:10CBA8000AD86E2A06D13E46236804341D6075E70C
:10CBB800002A54D03E4671E7752A26D0782AF9D142
:10CBC800A2F1580304F1040C5A422068CDF80CC0B5
:10CBD8004FF010015A4105ABFFF7A2FDDDF80CC07C
:10CBE8003E46644605AB00934846514642465B467E
:10CBF800FFF7E9FD054451E72068271D0A210022B7
:10CC080005ABFFF7B4FD3C46ECE704F1040CCDF8A6
:10CC18000CC020680A210022DDE72068002804F102
:10CC2800040708DA2D238DF8143040420DF115035E
:10CC38000A210022E5E705ABFAE72068002804F19D
:10CC4800040C0ADA2D238DF8143040420DF1150337
:10CC5800CDF80CC00A210022BEE705ABF8E728464C
:10CC680009B0BDE8F08F0FB413B50B4904AB0868E1
:10CC78000A4953F8042B09680193FFF707FF044694
:10CC8800074B186803F0C4FD0028F9D0204602B00D
:10CC9800BDE8104004B07047740100207001002006
:10CCA800B810002080EAE073A3EBE0738B4206DB48
:10CCB800002801DD401A704702D008447047002060
:10CCC8007047B0EEE06AF0EEC05AB4EEE56AF1EEF5
:10CCD80010FAD4BFF0EE656AF0EE466AF5EE406AE7
:10CCE800F1EE10FA0BD0B4EEE56AF1EE10FA54BF8B
:10CCF800F0EE657AF0EE467AC7EEA66A01E0DFED5F
:10CD0800206ADFED207A9FED207A9FED205AA6EE6B
:10CD1800A77ADFED1F7AE7EE267A9FED1E7AA7EE57
:10CD2800A67ADFED1D7AE7EE267AF4EEC65AB1EE62
:10CD3800677ADFED1A7AA6EEA75AF7EE007AE5EEE3
:10CD4800267AF1EE10FAC7EE277AC8BF9FED147A5B
:10CD5800F5EEC00AC8BF77EE677AF1EE10FA48BF61
:10CD68009FED107AB5EEC00A48BF77EE677AF1EE0C
:10CD780010FA48BFF1EE677AB0EE670A704700BF55
:10CD88000000000039094E3DE3B59EBE69A2163E7B
:10CD980088FA16BE45FE7FBFA7DFA8B499FB243FDB
:10CDA800DB0FC93FDB0F4940FDEEC07A17EE903A22
:10CDB8002033402B43D8DFED237AB4EEE70AF1EEB7
:10CDC80010FA04DDDFED207A30EE670AF3E7DFEDD5
:10CDD8001F7AB4EEE70AF1EE10FA04D5DFED1A7AFD
:10CDE80030EE270AF3E7DFED1A7AB4EEE70AF1EE40
:10CDF80010FA04DD30EE670A37EEC00A0AE09FED4C
:10CE0800157AB4EEC70AF1EE10FA44BF30EE270ADD
:10CE180037EE400A60EE007ADFED0F6A9FED0F7A79
:10CE2800A7EEA67ADFED0E6AE7EE876A9FED0D7A28
:10CE3800A7EEA67A20EE276AA6EE070A70479FEDAE
:10CE4800060A7047DB0F4940DB0FC940DB0F49C0BA
:10CE5800DB0FC93FDB0FC9BF0000000092E741B9F3
:10CE68009730083C15A82ABEDFED027A30EE270A73
:10CE78009AE700BFDB0FC93F064B1A8822EA000079
:10CE8800904210B518801C4602D0012003F056FCD1
:10CE9800208810BD681B0020064B1A88104390425A
:10CEA80010B518801C4602D0012003F047FC2088EA
:10CEB80010BD00BF681B0020024A936823EA0000E7
:10CEC80090607047BC12002008B5104B1A780023F8
:10CED800D9B2914207D20E4951F8231009680020AF
:10CEE80008600133F4E7322003F0D3FB094B1B68D9
:10CEF8005A0309D5084B9B685B0305D440F2DC5004
:10CF0800BDE8084003F0C5BB08BD00BFC42700202A
:10CF18009427002098290020BC1200202DE9F34115
:10CF280005F0C0F8454A6C2313704FF4FA63538038
:10CF3800BE231371EF2382F8CD37002382F8CE3752
:10CF480019461646F25C0133B3F5FA6F81EA02011D
:10CF5800F8D13A4B83F8CE17394B1A69120604D523
:10CF6800384A5A6002F188325A6004270020013F8B
:10CF780017F0FF074FD0324B3422DA60002444B157
:10CF8800002356F804800193FBF7EAFB0428EED14E
:10CF980017E0FBF7E5FB0428E9D1294D2B6943F09D
:10CFA80002032B61284B6B612B6943F040032B6113
:10CFB800FBF7D6FB2B69042823F002032B61DFD093
:10CFC800D5E71F4D2B6943F001032B6104F1006382
:10CFD80003F57E331FFA88F21A80FBF7C1FB042899
:10CFE80010D11A4B23440193019B4FEA1848A3F828
:10CFF8000080FBF7B5FB2B69042823F001032B61A4
:10D0080005D0B4E72B6923F001032B61AFE70434A3
:10D01800B4F5FA6FB3D10A4A1369042843F08003C0
:10D02800136102D103F0ECFD10B9052003F09EFB5B
:10D0380005F022F802B0BDE8F08100BFBC12002064
:10D04800002002402301674500F8030802F803089E
:10D0580010B50E4C206803F05FFA2068047A0022AD
:10D0680002FB02F3193B634303F6C413534319212C
:10D0780093FBF1F3064921F812300132072AEFD168
:10D088000449BDE81040FCF793BE00BF34120020ED
:10D0980088100020FC1300202DE9F04103F0B0FDBA
:10D0A80010B9042003F062FBB04CB14D04F0FAFF54
:10D0B800B0494FF4FA62204608F064FA94F8A437AD
:10D0C800022B84BF002384F8A43794F8A4274FF4D4
:10D0D800CC7101FB02F3E018234400F53770286097
:10D0E80093F8300303F54A73022801FB024284BF18
:10D0F8000020187292F830339F4A13700C2202FBFA
:10D1080003439E4A03F2A6731360A36846F209021A
:10D118001A401AB9954A43F400539360A368D80794
:10D1280003D54FF40050FFF7C7FEA368590409D58B
:10D138000820FFF7C1FE4FF40050FFF7BDFE0120A5
:10D14800FFF7BAFEA3681A0706D54FF40050FFF799
:10D15800B3FE0120FFF7B0FEA3689B0406D54FF489
:10D168008030FFF7A9FE4020FFF7A6FE012284F8D1
:10D178000D2294F8DE217D4B2AB193F8E22112B1F9
:10D18800002283F8E2217E4B7E4E1E604FF0000C99
:10D19800674604EB0C03B3F8F6E14FEA5E0101F0D1
:10D1A80077314FEA9E0303F03333C1EB0E00C11A07
:10D1B8004FEADE0303F01133CB1A03EB23131EF0FF
:10D1C800010803F00F324FF0FF0392FBF3F3C3EBB8
:10D1D800032318BF0137A2EB030318BFFFB2012BCB
:10D1E8000ADD022B40F0BF80B8F1000F00F0BB80D1
:10D1F8001EF0BC0F00F0B7800CF1080CBCF1180F42
:10D20800C7D1013F012F00F2AE80FFF721FF302286
:10D2180000215D485D4F08F0C0F95D4BD5F80080EE
:10D228001F605C4B002108F17900C3F8008003F00F
:10D23800B3F9594B80F001001870584B07F12802D8
:10D248001A60574B07F1CC021A6098F80000FFF7F4
:10D2580043FA2868534B00F5C5721A60FBF780F84B
:10D26800514B94F8D601DFED516A07F196021A6026
:10D2780064214F4BC82211FB00225A6000229A6099
:10D28800DA601A615A619A61DA6183F8202083F8BA
:10D298002120484B07F12E021A602B68464A93ED6D
:10D2A800187A03F219111160444A03F289111160C6
:10D2B800434A07F108011160424A1760424A07F1E0
:10D2C800A201116067EE266A404A07F1AC01B6EE8A
:10D2D800007A116087EE267A3D490E60B4F8641131
:10D2E800101D07EE901AB4F86611F8EE677AC2EDD1
:10D2F800027A07EE901A93F85C10117193F878107F
:10D30800517194F8E1111174F8EE677AB3F81611B7
:10D31800C2ED037A07EE901A2E49F8EEE77A086014
:10D32800536182ED077A9FED2C7AC7EE277A03F1D5
:10D338006401916129492A4A0B602A499FED2A7A9A
:10D3480067EE877AC2ED007A03F168020A6027491E
:10D3580003F211130B60264B1F60264BBDE8F0410A
:10D368001A6004F089BEFBF7C7F94EE7BC1200202B
:10D378001012002000F8030828270020341200208B
:10D388004C2D002044140020BC0F0020FC1300206A
:10D39800F00F0020F40F00200300002038080020C0
:10D3A800740600200010002008260020DB0F4940EA
:10D3B800582D0020502000209C1F0020340A0020F7
:10D3C800082900200C29002048090020F02000200E
:10D3D8000C0A0020C8200020000061440C0800202E
:10D3E80044090020000800204C3D0F443409002067
:10D3F8003C0900200007002008B5FFF78FFDFFF764
:10D408004BFE0120BDE8084003F098B9026D036B9C
:10D4180070B50446D5699BB9A90611D5C36A1BB175
:10D42800908C80B298470BE0E169928C40694E1C61
:10D43800D2B2E6614254E169E268914228BFE361F1
:10D44800616BA1B92A0612D5636AA26A9A42236D52
:10D4580009D0501CA669A062B25C1A85236998425B
:10D4680005D3A16203E01A6822F080021A602B0734
:10D4780042BF236D08221A6270BD026BC168034661
:10D4880010B5406942B11A6C8C1A013A005D08BFA8
:10D498000A46C0B21A6410BD1A6A805C01328A4218
:10D4A80028BF0022C0B21A6210BD436B13B190F8B6
:10D4B80044007047836A406A1B1A584258417047B3
:10D4C800036B13B15B68016C01E0C369016A8B42AD
:10D4D8003CBFC2689B18581AC0B27047836A8169FA
:10D4E800426B1944D160416A99429DBF0169CB1AC8
:10D4F8005360CB1A96BF0023536083624FF000033A
:10D5080080F84430136888BF816243F001031360D8
:10D518007047436A8269D154436A0269013393426E
:10D5280028BF00234362436B1BB11B68DB0705D48C
:10D53800D4E7026D136843F08003136070474171AC
:10D54800F7F79AB98160F7F797B92DE9F0410369C0
:10D55800C76805460E461F40002F35D0B7FA87F238
:10D568004FF00043D340DB432B611F40A2F11B0364
:10D57800042BF1D8DFE803F0221F1C190300746A9A
:10D5880024B1013C0023A4B2736201E0EC6AA4B2A6
:10D59800D6F82080B8F1000FDED0D8F80030404629
:10D5A80021469847D8F80480F4E73068696B07E0AB
:10D5B8007068A96B04E0B068E96B01E0F068296C59
:10D5C800036889B29847C7E7BDE8F0810148024976
:10D5D800BBE700BF00040040182800204FF080403F
:10D5E8000049B2E7F027002010B5054C0548214650
:10D5F800FFF7ABFF04F1F0010348BDE81040A4E7D2
:10D60800C8270020002C014000440140014802497D
:10D618009BE700BF002C0140C8270020224B10B513
:10D62800224C5A43224BB3FBF2F203880139013AE8
:10D63800A04289B292B29BB20ED004F50064A04217
:10D648000AD0B0F1804F07D0A4F59834A04203D097
:10D6580004F58064A04202D123F070039BB2154CFC
:10D66800A04206D004F58064A0421CBF23F4407396
:10D678009BB203800D4BC162984202850FD003F51F
:10D68800006398420BD003F54063984207D003F536
:10D698008063984203D003F58063984201D1002348
:10D6A80003860123436110BD40420F00002C014056
:10D6B80000A24A0400100040164B800A984226D067
:10D6C8000AD84A3B984218D00133984217D0B0F58F
:10D6D800801F1AD1012070470F4B984211D004D8EF
:10D6E800033B984211D1042070470C4B98420AD052
:10D6F8000133984209D10720704702207047032060
:10D7080070470520704706207047FE2070470020AC
:10D71800704700BF4B00100050001000510010006F
:10D72800F8B50468064620460F461546FFF7C4FFBD
:10D7380007284BD8B27A910847B902238B40D4F80E
:10D748000CE0DB439BB203EA0E03E3600A23204AA2
:10D7580003FB001342F82370043342F823501546A4
:10D768003FB1B17AE268890802238B409BB2134328
:10D77800E360282202FB00522032EFF31286502386
:10D7880083F3128803B203EB8303DB0003F10C017C
:10D798001C3329442B4451F8047F17B117600A68D9
:10D7A80004329942F7D100231360F3B283F311884E
:10D7B800282303FB0050036A1BB1E36843F001030D
:10D7C80003E0E2684FF6FE731340E360F8BD00BF64
:10D7D800C8270020004819E610210020004815E657
:10D7E800642100200D4B0E484FF400525A600D4A38
:10D7F80011684FF6FE730B401360D0F8882011684B
:10D808004FF6FE730B401360826FC36F9A4201D0CC
:10D81800543063E6012380F89830704700000240D6
:10D8280010210020440002402DE9F0471E46A54B78
:10D838008CB09842894690469DF8507040F08B8095
:10D84800A14BA24A5A6503F1A8029A6603F5D4725D
:10D85800DA664FF480721A665A669D4AC3F88420C5
:10D86800143AC3F88820A2F54842203AC3F8A02009
:10D878000432C3F89C20C3F85C80C3F8A400954B1D
:10D888009A6942F480429A615A6942F001025A61E7
:10D8980002238DF80830032317F0010A8DF80930A8
:10D8A8004FF000038DF80A3014BF022301233A0712
:10D8B8008DF80B3019D54FF090444FF40075019551
:10D8C8008AF001038DF80A30636A23F0F00363627B
:10D8D800636A43F070036362204601A9FBF7B6FB55
:10D8E800BAF1000F27D1A56125E0B30710D50CA91F
:10D8F8004FF4007341F82C3D4FF09040436A23F0F9
:10D90800F0034362436A43F070034362FBF79EFBF4
:10D91800F50710D50CA94FF4806341F82C3D4FF062
:10D928009040436A23F470634362436A43F4E063BC
:10D938004362FBF78BFB0E238DF800300022012396
:10D9480068468DF801308DF802208DF80330624C5E
:10D9580003F02AFD74E0614B984240F003815A4B72
:10D968005A4A1A604FF48072DA601A6103F52A7213
:10D978005A6103F56A729A61564AC3F808801865B5
:10D98800D36943F40033D36102238DF808300323AD
:10D9980017F0010A8DF809304FF000038DF80A30AE
:10D9A80014BF022301233C078DF80B3017D54C4CCC
:10D9B800202501958AF001038DF80A30236A23F4A3
:10D9C80070032362236A43F4E0032362204601A91B
:10D9D800FBF73CFBBAF1000F23D1A56121E0B007AA
:10D9E8000ED50CA9202341F82C3D3D48036A23F4A9
:10D9F80070030362036A43F4E0030362FBF726FB48
:10DA0800F1070ED50CA9402341F82C3D3448036A90
:10DA180023F070630362036A43F0E0630362FBF779
:10DA280015FB26238DF800300022012368468DF867
:10DA380001308DF802208DF8033003F0B5FC224C3C
:10DA4800C4F82C900025012384F844302562E56150
:10DA5800A56265626671C4F80880A7712046F6F76A
:10DA68000BFFF20745D5236B002B3BD001A8FBF732
:10DA780095F8E36C01934FF480530A93802306933F
:10DA8800E368ADF8103020230993206B6369029393
:10DA98000B950595079508950395FBF7AAF801A935
:10DAA800206BFBF788F8236B216D1A6842F001029E
:10DAB8001A608A6842F040028A605B689BB22364FD
:10DAC80017E000BF0038014010210020D47E010873
:10DAD8005800024000100240642100200044004029
:10DAE800000C0048236D20221A621A6842F02002B6
:10DAF8001A60B3072FD5636B43B301A8FBF74EF841
:10DB0800A36C01934FF480530A93802306932369EF
:10DB1800ADF8103000251023606B03930B95059525
:10DB2800079508950995FBF764F8606B01A9FBF761
:10DB380042F8636B1A6842F002021A60226D5D6057
:10DB48005D60936843F08003936004E0226D13687E
:10DB580043F080031360226D136843F001031360E0
:10DB6800204600E000200CB0BDE8F0872DE9F74F13
:10DB7800A74C02F067FD26686568A768861BF64310
:10DB8800451BC71BED43FF43F60F8046ED0FFF0F04
:10DB98002EB93FB9002D00F08682B9462CE04FF02F
:10DBA800000929E0B14627E003EB8A0BBBF80230F5
:10DBB8001A050ED413F4805F1DBF964A9BF8011016
:10DBC8001268954A954B14BF52F82120126843F801
:10DBD8002A20BBF80230D80516D499050AD5904BEF
:10DBE8001B7813F0040F0CBF8E4A8F4A8B4B1268B8
:10DBF80043F82A2009F10109207B8C495FFA89FA48
:10DC080082450B68D0D326E0894A5046594601F030
:10DC180037F9884B1B885A0603D550465946864A19
:10DC280016E0580703D550465946844A10E01907AC
:10DC380003D550465946824A0AE09A0703D550460A
:10DC48005946804A04E0DB07D4D57F4A50465946F6
:10DC580001F016F9CEE7DFF808E20093BEF90630C6
:10DC68007822A3F57A7353434FF47A7293FBF2F355
:10DC780003F22B1301930022F3465FFA82FE8645D6
:10DC880017D2009B03EB820EBEF802E01EF4806FF1
:10DC98000DD0DFF88891019B39F822E040F2671A2D
:10DCA8009E449EFBFAFC0AFB1CEE29F822E0013296
:10DCB800E3E74DB308F5C333A0336360637B544A8D
:10DCC80013BB9373614B1B6813F0020F0AD0DFF884
:10DCD80094E19EF800E0BEF1000F03D04FF0010E72
:10DCE80082F80EE0DA0506D5594BDB781BB1A37B29
:10DCF80043F00203A3734A4B1B7813F0050F02BFCE
:10DD0800A37B43F00403A37394F80EE0BEF1000F65
:10DD180003D13F4B5B7B002B4FD094F80DC01CF018
:10DD2800010FACF10C031DD1BCF1030F07D8DFF8CC
:10DD3800E8903C4A1EF0040F08BF4A4600E0364A05
:10DD4800ACF1040CBCF1070F05D8DFF81CC11EF0BC
:10DD5800010F18BF6246DBB2032B0ED81EF0020F6C
:10DD68003C4B06E0DBB2032B06D82F4B2A4A1EF0A9
:10DD7800020F18BF1A4600E0274A4FF0000C5FFA5E
:10DD88008CF383420DD20B6803EB8C035B881B0674
:10DD980042BF224BD2F8009043F82C900CF1010CB2
:10DDA800EDE785B1BEF1000F08D0637B184A013357
:10DDB800DBB2142B06D1002304E025B1637B002BD2
:10DDC800F3D100E05373002E52D0234AB2F9025027
:10DDD800B2F90020002DB8BF6D42002A4FF032037F
:10DDE800B8BF524295FBF3F592FBF3F2EDB2D3B212
:10DDF800AB4238BF2B46194A13B192FBF3F300E04C
:10DE0800134643442360E37B014A7BBB01232EE096
:10DE1800B8250020941F0020609001087A0E002089
:10DE2800B62D0020288F0108188F0108981F0020A0
:10DE3800F47E0108681B0020FA7E0108007F0108B3
:10DE4800067F01080C7F0108127F0108982900202D
:10DE5800582D0020308F0108B4120020400D030017
:10DE6800782C0020F01A0020388F01080023D37383
:10DE78008E4D8F4B2D78E27BADB9002F00F00E81CF
:10DE88008C4B267B1A788C4B8C4D93F800C08C4BAE
:10DE9800D3F800E00B6802F004020021D2B203EBD1
:10DEA80086060F46B5E01AB9864A1A61002508E0C9
:10DEB800854AFAE70A68AB00D6187688760604D44D
:10DEC8000135EBB28342F5D3D7E7804EB6F900604F
:10DED800192E25DD12F803E094F814C026690EF017
:10DEE8000F09E1450CDCDFF8C8C19CF815C0BCEB94
:10DEF8001E1FDEBFDFF8D8E1D6F800C043F80EC019
:10DF080012F803E094F816C00EF00F09E14533DB70
:10DF1800DFF89CC19CF815C0BCEB1E1F2CDC26E06A
:10DF2800193629DA12F803E094F814C026690EF0BD
:10DF38000F09E1450CDCDFF878C19CF817C0BCEB91
:10DF48001E1FA2BFDFF888E1D6F800C043F80EC054
:10DF580012F803E094F816C00EF00F09E1450BDB48
:10DF6800DFF84CC19CF817C0BCEB1E1F04DBD6F8C9
:10DF780000E0574E43F806E0544EB6F90260192EF9
:10DF88001BDD12F803C094F814E026690CF00F09A1
:10DF9800F1450CDCDFF8189199F81590B9EB1C1FC6
:10DFA800DEBFDFF82CC1D6F8009043F80C90D25CA5
:10DFB80002F00F0CF4451EDD82E7193680DA12F8FC
:10DFC80003C094F816E026690CF00F09F1450CDB44
:10DFD800DFF8DC9099F81590B9EB1C1FDEBFDFF86D
:10DFE800F0C0D6F8009043F80C90D25C02F00F0C09
:10DFF800F445FFF665AF94F817E0BEEB121FA2BF19
:10E00800334A36689E505BE75888000504D40433C9
:10E018000435B342F8D122E04AB101EB0C0A0620DC
:10E028009AFBF0F900FB19A001280DDC01E057B9B3
:10E03800012793F801900EEB89003EF829A090F88B
:10E048000290C07803E017460020814682460131DD
:10E0580025F802AC85F800906870C9B2D7E7164A6F
:10E068001378013B13F0FF0308BF06231370114B0D
:10E078001B785B0741BFBBF90630A3F57A7303EB46
:10E08800C3034FF47A7243BF93FBF2F30133DBB25D
:10E098000123104A92FBF3F34344A36003B0BDE8A5
:10E0A800F04FF6F74BBD03B0BDE8F08F2B0F002003
:10E0B800B8250020B62D0020940000207C0E0020FA
:10E0C800941F0020348F010860900108B4120020CA
:10E0D8007A0E0020400D0300064B1B7803F0040362
:10E0E80003F0FF001BB1044B1888C0F3C01000F008
:10E0F80001007047B62D0020681B00202DE9F04F65
:10E108002DED028B87B000260493BD4B0391B3F924
:10E118000270B3F900300192002FB8BF7F42002B84
:10E12800B8BF5B429F42B8BF1F46B7F5FA7F80462B
:10E13800A8BF4FF4FA770090B246B446B3463446C7
:10E14800B04D2B8899075AD0AD4BAF4A33F81430ED
:10E1580032F91420022013FB0022019B5B429A42F1
:10E168004FEA440103DB019B9342A8BF1346A74A29
:10E1780031F90290049A32F91420C9EB030303EB36
:10E188000209FFF7A9FF88B107EE909AA04BB8EEF5
:10E19800E70AB2EE048A185D80EE080A03F04EF929
:10E1A80020EE080AFDEEC07A17EE909A98F808302B
:10E1B800642203FB09F393FBF2F398F81C206FF039
:10E1C800040B0BFB02FB5B4504DB02EB820B9B455C
:10E1D800A8BF9B468F4A52F8241009EB010342F26C
:10E1E80010718B42A8BF0B468B498B42B8BF0B46B8
:10E1F80042F8243098F8122053434FEA233C2D88E4
:10E2080005F00303012B38D07D4B844933F914A062
:10E21800009B51F824E093F80190814B33F91400E6
:10E2280080EAE073A3EBE073B3F5206F4FEA84064E
:10E2380016DC0AEB8A031A0192FBF9F3042290FB1D
:10E24800F2F0181A8644BEF57A5FA8BF4FF47A5EDA
:10E25800744B9E45ACBF41F824E041F8243002E0FD
:10E26800002341F824308B597D2693FBF6F6009B5A
:10E27800DB7A7343402693FBF6F6AA0710D5C7F559
:10E28800FA7307FB0AF907FB06F54FF4FA7103FB6B
:10E298000B9903FB0C5599FBF1F295FBF1F505E0A1
:10E2A800EB0759BF3546524665465A466300029306
:10E2B8005D495B4B615C33F814004FF0040E03B208
:10E2C80093FBFEF909FB01F16FF04F0991FBF9F996
:10E2D8009144564A32F9141022F814005B1A98F83F
:10E2E800501093FBFEF300EE103A79B1504B5148B1
:10E2F800D3ED000ACDF814C0B8EEC00A00EBC40094
:10E30800FEF792FADDF814C0BDEEC00A4A4A029937
:10E3180012F804E0494810EE103A09EB05020EFB2A
:10E3280003F34FF0200E93FBFEF3D21A0A5244492E
:10E33800444A41F82450444D42F824905B4245F841
:10E348002430009B013300930CB90124F8E62C4BD0
:10E3580098F80D70B3F90440039B9B790F335B0069
:10E3680063435B112E4C002B4FF00406B4F90440B4
:10E3780094FBF6F4294EA3EB0404B8BF5B42322B9E
:10E38800D6F808E00BDC314B07FB04E7BB42A8BF1B
:10E398003B462F4FBB42ACBFB360B76001E00023E0
:10E3A800B36098F803305C432A4B1B78032B4FEA81
:10E3B800A4140CD9B8F84E30B3F5FA7F07D25F42EF
:10E3C800BC4203DB9C42A8BF1C4600E03C46B36845
:10E3D800946043F34F33B3F5807FA8BF4FF4807345
:10E3E8006FF0FF06B342B8BF3346E6188B600023D0
:10E3F8008680AB6007B0BDEC028BBDE8F08F00BF34
:10E40800B4120020681B0020B02D002090290020A5
:10E41800C47E0108D0250020F0D8FFFFB41F0020DB
:10E42800F411002080C1FFFF24200020D8250020FF
:10E43800AC1F0020CC1F002038200020E41F002043
:10E44800F81F0020EC1F002004200020FEFFFF0F13
:10E45800020000F0C42700202DE9F04F2DED028BBB
:10E4680085B080460293A84B01911C88009204F065
:10E478000204A4B294B1A54BB3F90240B3F9003039
:10E48800002CB8BF6442002BB8BF5B429C42B8BFA7
:10E498001C46B4F5007FA8BF4FF40074C24600259F
:10E4A8009A4B9B4833F815209A4B50F8256033F95E
:10E4B800153083EAE377A7EBE37711B2B7F5206F5E
:10E4C8004FEA450B4FEA41014FEA850911DC042761
:10E4D80093FBF7F3CB1A1E44B6F57A5FA8BF4FF447
:10E4E8007A568D4B9E42ACBF40F8256040F82530E7
:10E4F80002E0002340F8253050F809609AF80B3004
:10E508009AF80170F6115E437F4B1B884F439B07B7
:10E518004FEAA6164FEAA71756D0804B33F90B30AF
:10E52800022112FB0132009B5B429A4203DB009BF3
:10E538009342A8BF13467A4A3BF902209A1A029BD3
:10E5480033F91530D31808EE103AFFF7C5FD68B156
:10E55800B8EEC80A734BB2EE048A80EE080A585D1A
:10E5680002F06CFF20EE080ABDEEC08A6E4918EE74
:10E57800102A59F8013042F2107013448342A8BFA0
:10E5880003466A4898F808208342B8BF034649F80A
:10E59800013018EE101A4A4398F81C1001EB81015B
:10E5A800D2114842824203DB8A42A8BF0A4610467B
:10E5B80098F8122053431B13F61A3F1A6643674311
:10E5C80003EB662600EB6727524ADFF890C13BF859
:10E5D80002001CF805C003B24FF0040E93FBFEF1D5
:10E5E80001FB0CF1A7EBA11751493BF901C02BF82E
:10E5F800010098F85010CCEB030393FBFEF300EEF8
:10E60800103A69B14B4B4C48D3ED000A0392B8EE6F
:10E61800C00A00EBC500FEF707F9039ABDEEC00A71
:10E628004649474811F805E010EE103A0EFB03F38F
:10E63800B9195B11C91A2BF80010424949F8017041
:10E64800414F49F80760414E5B4249F806300AF1EC
:10E65800010A0DB9012523E72C4BB2F90420B3F9BF
:10E668000440019B9B790F335B0063435B11002BD4
:10E678004FF00405264C92FBF5F5A3EB0505B8BF52
:10E688005B42322BD4F808E098F80D200BDC304BB5
:10E6980002FB05E29342A8BF13462E4A9342ACBF41
:10E6A800A360A26001E00023A36098F8032002FBA6
:10E6B80005F3294A1278032A4FEAA3130CD9B8F8AC
:10E6C8004E20B2F5FA7F07D25542AB4203DB9342A4
:10E6D800A8BF134600E02B46A2688B6042F34F3276
:10E6E800B2F5807FA8BF4FF480726FF0FF04A2429A
:10E6F800B8BF22469C1800238480BA60B36005B076
:10E70800BDEC028BBDE8F08F681B0020B41200201E
:10E71800B41F0020F411002080C1FFFFB02D00209D
:10E7280090290020C47E0108D0250020F0D8FFFFE2
:10E73800DC250020AC1F0020CC1F00203820002042
:10E74800E41F0020EC1F0020F81F002004200020F8
:10E75800FEFFFF0F020000F0C42700202420002045
:10E768002DE9F04F2DED028B85B000260293A94BC1
:10E778000192B3F90270B3F900300090002FB8BFCE
:10E788007F42002BB8BF5B429F42B8BF1F46B7F518
:10E79800FA7F8146A8BF4FF4FA77B246B346B0462F
:10E7A80034469D4D2B8899075DD0022C5BD0994B40
:10E7B8009A4933F8143031F914104FF0020E13FB54
:10E7C8000E11019B5B4299424FEA440003DB019B17
:10E7D8008B42A8BF0B469249029A30F901B032F930
:10E7E8001410CBEB030303EB010BFFF775FC88B1A7
:10E7F80007EE90BA8B4BB8EEE70AB2EE048A185DC2
:10E8080080EE080A02F01AFE20EE080AFDEEC07A31
:10E8180017EE90BA99F80830642103FB0BF393FBC9
:10E82800F1F399F81C106FF0040808FB01F8434550
:10E8380004DB01EB81089845A8BF98467A4951F84E
:10E84800243042F210705B448342A8BF03467748E5
:10E8580099F812B08342B8BF03460BFB03FB41F89B
:10E8680024304FEA2B3B2B8803F00301012901D107
:10E87800022C42D16E4D674A35F9145032F914A072
:10E888006C48009A85EAE576A6EBE576B6F5206F42
:10E8980092F801E050F824204FEA840120DC022C91
:10E8A80018D00AEB8A00000190FBFEFE042095FBBD
:10E8B800F0F5C5EB0E0E02EB0E0CBCF57A5F5D4869
:10E8C8005D4DA8BF4FF47A5CAC45ACBF41F800C0C1
:10E8D8000D5007E08AEAEA76A6EBEA76642EE0DDD8
:10E8E800002545505348009A09587D2691FBF6F6B5
:10E8F800D17A7143402691FBF6F69A0712D5022C7D
:10E9080010D0C7F5FA7307FB06F507FB0AF103FBFE
:10E9180008114FF4FA7003FB0B5391FBF0F193FBD2
:10E92800F0F508E0DB0704D5022C02D05D4641462D
:10E9380001E0354651463E4B33F91400042390FB61
:10E94800F3F33E48205C022C03FB00F36FF04F000A
:10E9580093FBF0F30B444FEA440C08EE103A0ED147
:10E96800374B3848D3ED000ACDF80CC0B8EEC80ACA
:10E978001E21FDF759FFDDF80CC0BDEEC08A2C4BF7
:10E9880031493CF803003CF901302CF8010099F8B2
:10E9980050100FFA80FEC3EB0E034FF0040E93FBEA
:10E9A800FEF300EE103A79B1254B2848D3ED000A62
:10E9B800CDF80CC0B8EEC00A00EBC400FDF734FF78
:10E9C800DDF80CC0BDEEC00A214B22481B5D10EEDD
:10E9D800102A534318EE102A51194FF0200E93FBBA
:10E9E800FEF3C91A2CF800101B4941F824201B49D2
:10E9F80041F824501A495B4241F82430009B013405
:10EA08000133032C00937FF4CCAE05B0BDEC028B30
:10EA1800BDE8F08FB4120020681B0020B02D002044
:10EA280090290020C47E0108D0250020F0D8FFFFDF
:10EA3800F4110020B41F002080C1FFFF2420002013
:10EA4800AC1F0020A41F0020E0250020CC1F0020C0
:10EA580038200020E41F0020EC1F0020F81F0020B1
:10EA6800042000202DE9F04F2DED088B83B00AEE2D
:10EA7800102A0093D14B01931A8812F0020F054611
:10EA8800F7EE009A4CD0149BCD48DC89B0F90030E1
:10EA98001B1B03F2F31640F2E632964203D8002B12
:10EAA800B8BF5B4201E04FF4FA73B0F90220121BC1
:10EAB80002F2F31440F2E630844203D8002AB8BFC9
:10EAC800524201E04FF4FA7295F84C0058B3934261
:10EAD800B8BF1346C3F5FA7307EE903A9FEDB97ABB
:10EAE800F8EEE77A6423C7EE877A93FBF0F307EE34
:10EAF800103A77EEE97AB8EEC77AB0EE699AA7EEDF
:10EB0800879AF7EE006AB5EEC09AF1EE10FA0AD4C9
:10EB1800B4EE669AF1EE10FAC8BFB0EE669A04E059
:10EB2800B0EE699A01E09FEDA89AA84ECF1C2C463A
:10EB38004FF00008B8F1020F17F801BFDFF8DC92B8
:10EB48004FEA480AF2EE04AA0ED1B9F904109FED73
:10EB5800A07A0BF10A0B01FB0BF307EE903AF8EEE3
:10EB6800E77AC7EE877A68E0F8EE4A7A9FED956A09
:10EB780039F91830C7EE867A06EE903A954B33F994
:10EB8800183007EE103A1AEE103AF8EEE66AB8EEC8
:10EB9800C77A5B42A6EEA77A07EE903AF8EEE77AD4
:10EBA800B4EEE77AF1EE10FA08D4F8EECA7AB4EEC9
:10EBB800E77AF1EE10FAD8BFF0EE477A864B33F9D0
:10EBC8000A3008EE103A009BB8EEC88A33F91830BC
:10EBD80077EEC87A08EE103AB8EEC88A37EE888A17
:10EBE80088EE2A8AFFF778FA40B17C4B13F80800C0
:10EBF800B0EE480A02F022FCB0EE408A019B198868
:10EC0800CA0704D5D5ED117A68EE277A15E039F9E7
:10EC18000A309FED6F7A0BF1140B03FB0BF307EE31
:10EC2800903AF8EEE77A8B07C7EE877A42BF95ED00
:10EC3800127A28EE078AE8EE097A694BDFF8E0B124
:10EC480033F90A3094ED08BA9FED668ADFF8D4915B
:10EC580007EE103A644BB8EEC77AD3ED0A6A18F893
:10EC68000B30E7EE667AB8F1020FF0EE48BAF0EE34
:10EC7800678A67EE8B7A0BEE103AB8EECBBA27EEBE
:10EC88008BBA8BEE08BA09D1B0EE4B0A5748D9EDCA
:10EC9800000A1E21FDF7C8FDB0EE40BAD9ED000A02
:10ECA80094ED0B7A68EEA07A67EE877A96ED007A93
:10ECB800A7EEAA7ADFED4E7AB4EEE77AF1EE10FA13
:10ECC800F0EE47AA09D4DFED4B7AB4EE677AF1EE9D
:10ECD80010FAC8BFF0EE67AA01E0F0EE67AA89EE65
:10ECE800A08A45494FEA8809494491ED000AC6EDD2
:10ECF80000AAC1ED008A38EEC00A95F8501020EE3F
:10ED0800080A21B13D4800EBC800FDF78DFDD4EDA0
:10ED18000E7A1BF8083060EE277A00EE103AB8EE4B
:10ED2800C00A27EE800ADFED367A80EE2B8AB4EE31
:10ED3800E78AF1EE10FA09D4DFED327AB4EE678A89
:10ED4800F1EE10FAC8BFB0EE678A01E0B0EE678A4C
:10ED58003BEE2A0A08F1010830EE080A06F02CFEFC
:10ED68002949B0F57A7FA8BF4FF47A708842B8BFB6
:10ED78000846BDEECBBA25491BEE103A21F80A0029
:10ED8800FDEEEAAA2249BDEEC88A49F801302149B8
:10ED98001AEE903A49F801301F4918EE103AB8F1C6
:10EDA800030F49F8013004F1040406F104067FF466
:10EDB800C1AE03B0BDEC088BBDE8F08F681B002026
:10EDC800782C00200000FA430000000010200020EA
:10EDD80000004842B02D002090290020C47E010880
:10EDE800F41100200000C842D0250020A41F0020F4
:10EDF80000007AC300007A43FC250020CC1F0020C5
:10EE0800000096C30000964318FCFFFFE41F002093
:10EE1800EC1F0020F81F002004200020B41200205E
:10EE2800A01F0020AC1F0020044B00221A605A606B
:10EE3800034B00221A605A60704700BFD02500209B
:10EE48001C20002010B50B4C0123E3704FF48060A8
:10EE5800022384F82030FEF71FF8074A074B926B0D
:10EE68001B685178642212FB0133636123880133E4
:10EE7800238010BD582D0020D0250020BC2900205B
:10EE880010B54B88DC0641BF2F4B14791B6853F82B
:10EE9800244044BF2D4B43F820404B889B0641BF7C
:10EEA800294B54791B6853F8244044BF274B43F837
:10EEB80020404B881C070ED5254B0C781B78B3EBEC
:10EEC800141FA1BF204BD4781B6853F82440A4BF5B
:10EED8001E4B43F820404B889B070ED51D4B0C78E2
:10EEE8001B78B3EB141FDFBF174B54781B6853F81C
:10EEF8002440DCBF154B43F820404B88DC070FD576
:10EF0800154C0B78247803F00F03A342DFBF0E4B98
:10EF180014781B6853F82440DCBF0C4B43F820409E
:10EF28004B885B070FD50B780C49097803F00F0362
:10EF38008B42A1BF044B92781B6853F82220A4BFD0
:10EF4800024B43F8202010BD941F00207A0E0020A9
:10EF5800CF250020CD250020CC250020CE2500205F
:10EF6800254A264826490023F0B5156803700B701A
:10EF78001C461A462E1976884EB92F5D3FB9037084
:10EF880000230A704B7007781C461A460CE03605B9
:10EF980048BF013204F1040403F1010348BFD2B2AF
:10EFA800802CDBB2E6D1EAE7E0B2B8420CD215F821
:10EFB800240006099E4200F00F00A8BF731C90426F
:10EFC800A8BF421C0134EFE78A704B70C2F34701B7
:10EFD80002F001020A444C1E0A490B480A70C3F3A6
:10EFE800470203F00103134404700849501E084AFD
:10EFF80008701370F0BD00BF981F0020C4250020C2
:10F008000C260020CE250020CC250020CF2500206E
:10F01800CD2500202DE9F04FC24BDA682DED028B8B
:10F028001A61C14A1168D960C0490B6843F02003CE
:10F038000B60BF4B1978012990460CBF00220122B2
:10F048001A70BC4B1A78910789B040F13D83BA49D0
:10F058000978042940F23883B849097801F0040195
:10F0680001F0FF0011B922F001021A701B78DB07CA
:10F0780002D408B1F9F7D6F9B149CA78531C052268
:10F0880093FBF2F202EB82029A1AAE4BCA701B781B
:10F09800039392000023AC4CDFF8CCC2DFF8D8927F
:10F0A8005CF8231091FBF9F504F1080004F110064F
:10F0B80040F82350A54844F8231000FB051142F2FC
:10F0C800107091FBF0F080B226F813004FF0140E88
:10F0D80004F1140604F13C0A0EFB036E5AF823608F
:10F0E8005EF802704EF80210F61B314444344AF8B8
:10F0F8002310052691FBF6F109FB051144F82310AE
:10F10800039C012C4FEA830BE24605D10238B0F587
:10F11800797F98BF4BF80C100BB90123BBE7884CDB
:10F12800D8F80030226D9FED8A7A8A4E8A4D9B1A54
:10F1380007EE903AF8EE677AD8F800302365C7EE04
:10F14800877A7C4B1B78B7EE008AF4EEC87AF1EE2A
:10F1580010FA58BFF0EE487A13F00103C4ED157A9F
:10F1680012D005AA00927D4B06AA01920CCB9AE810
:10F178000300F9F755F86421059A069BB2FBF1F2F2
:10F1880093FBF1F3328000E033802B8094F8583001
:10F198006B48002B3BD0D0ED157AC26DDAF8003001
:10F1A800C8EE276A9B1A026E022507EE103AB8EEDF
:10F1B800C77ADAF8043027EE267A9B1AFDEEC77A6A
:10F1C800B0F9662017EE901A07EE903A644BB8EE45
:10F1D800E77AD3ED007A67EE277A67EEA67AFDEE36
:10F1E800E77A17EE903A02FA83F3B0F9642093FBBA
:10F1F800F5F302FA81F29BB292FBF5F292B2A0F813
:10F208006A30A0F86820A0F86630A0F864200123CE
:10F2180084F85830534BDAF804101B88DAF80000E9
:10F22800474D514E216603F03003E065002B00F096
:10F238004B8205F17403009305F178030193EA6E9C
:10F248002B6FF8F7EDFF72682B6F9B1A07EE903A59
:10F25800434B326893ED007AEB6EF8EEE77A9B1A2F
:10F26800EB67384B67EE877A1B78FDEEE77A012B60
:10F27800C5ED207A03D0022B00F0DF8024E2D5ED23
:10F28800287A3A4BD5ED215A95ED255A95ED156A10
:10F2980095ED264AD5ED274A35491D68B1EE677ABE
:10F2A800BDEEC77AFDEEE77A17EE10EA17EE90CAC0
:10F2B8000020304A91ED007A52F8207007EE907ADB
:10F2C800F8EEE77AA2F1140367EEA57A33F8106036
:10F2D800FDEEE77A283217EE903A9B1B9BB222F894
:10F2E80010301BB207EE903AF8EEE77A3B4467EE2F
:10F2F800857A4400FDEEE77ACDED037A07EE903A81
:10F30800F8EEE77ABDF80C8067EE847AA7EE867A85
:10F31800FDEEC77A17EE902A724531DB6245A8BF29
:10F3280062462EE010080020BC290020A01A002008
:10F338003A120020A41A0020AA1A0020B62D002094
:10F348000C260020FC0F002010260020806967FF93
:10F3580000007A441E1B0020201B00203C120020C5
:10F3680098000020681B0020AC1A00200010002024
:10F37800301000208826002080969800DB0FC940B6
:10F38800724607EE902AF8EEE77A5FED046AC1ED5F
:10F39800007AFDEEE77A313617EE903A43449AB296
:10F3A800AB78D1ED027A07EE103AB8EE477A4B689F
:10F3B8004F6027EE267AFB1A88EE077AB6B2622EDD
:10F3C80006EE903AF8EEE66A37EE067AC6EE866AF8
:10F3D80086EE077A76EEE76AE7EE267AC1ED047ADA
:10F3E800C1ED027A0FD964EEA77ABA4EFDEEE77A3C
:10F3F80017EE903AB3F5FA6FA8BF4FF4FA63B34229
:10F40800B8BF334600E0002313441BB240F6B832BD
:10F418009342A8BF1346B04A9342B8BF1346AF4AB7
:10F42800A352AF4A142303FB002351F8142B1A608C
:10F43800002840F0498101203BE7AA4BD5F87480A9
:10F448001F68D4F878903E89DFEDA78A4FEA580301
:10F458009E4228BF1E46B5F8A8301AB29642C3BFCE
:10F46800D5ED157A9FEDA17A67EE877AB6B2C1BF5E
:10F47800FDEEE77A17EE906AF618B6B2C8BFA5F89F
:10F48800A860D4F8AC50C5EB09052846F8F70CFF7E
:10F498000028D8BF404241F293129042CCBF0020CE
:10F4A800012088B307EE905AB8EEE70A20EE280A42
:10F4B800FDF77AFC07EE908AF8EE677A40F6B833E3
:10F4C80020EE270AFDEEC07ACDED037ABDF80C20B8
:10F4D800A4F8B02012B29A42A8BF1A467E4B9A42AC
:10F4E800ACBF09EB02034B4448F6A042934203DD4C
:10F4F800A3F50C43A03B04E0002BBCBF03F50C4371
:10F50800A033C4F8B43001E0C4F8B490D4F8B450CF
:10F51800C5F50C53283307EE903AF8EEE77A67EE14
:10F52800A88AB0EE680AFDF79FFC8DED070AB0EED9
:10F53800680AFDF739FCD4ED317AD4ED2E4AD4EDC2
:10F54800155A94ED2F4A94ED305A65498DED060A07
:10F55800B1EE677ABDEEC77AFDEEE77A0DF1180EC7
:10F5680017EE10AA17EE90BA0020614AFEEC016A65
:10F5780032F91030DFF88C9107EE903A07EE106AF6
:10F58800F8EEE77AB8EEC77A3C32D6EE877A4FEAD9
:10F59800400CFDEEE77ACDED037ABDF90C30B3F5FA
:10F5A8007A7FA8BF4FF47A734B45B8BF4B461FFA12
:10F5B80083F922F810900FFA89F207EE902AF8EEF4
:10F5C800E77A27EEA47ABDEEC77A8DED037A27EEA7
:10F5D800847AD1ED007ABDF80C90E7EE257AFDEE3D
:10F5E800E77A17EE902A524503DB5A45A8BF5A46D8
:10F5F80000E0524607EE902AF8EEE77A9FED3D6A62
:10F60800C1ED007ABA7891ED027A06EE902AF8EE0A
:10F61800666A4A684B6066EE866A9A1AC8EE266A77
:10F62800143106EE102AB8EEC66A76EEA56A86EEA2
:10F63800256AC5EEA66A36EE476AA6EE867A01ED19
:10F64800017A01ED037A25EE077ABDEEC77A17EE47
:10F65800103ABDEEE77A4B4417EE102A13441BB25A
:10F6680040F6B8329342A8BF13461B4A9342B8BF2C
:10F6780013461A4A2CF802301F4A142303FB0023AE
:10F68800C3ED007A08B901206FE73B7923B1642301
:10F6980095FBF3F5194B1D803B8898450DD9D4F897
:10F6A800AC30A06FC01AF8F7FFFD80EAE072A2EB59
:10F6B800E07242F210739A4206DD114B01221A7071
:10F6C8000E4BB4F8C8201A8009B0BDEC028BBDE817
:10F6D800F08F00BF30F8FFFF48F4FFFF84100020D0
:10F6E8005810002000100020D30237390000C8420B
:10F6F80074260020DB0FC94030100020F80F0020CE
:10F70800FC0F002018FCFFFF012380F845307047EC
:10F718002DE9F04390F84410002380F84430002984
:10F7280053D02E4C2268002A52D02268052A52D182
:10F738002B4C20290D4628BF20256E1C27687610E3
:10F74800DFF8A8E0DEF800309BBBDFF8A4C000F1CA
:10F758003203324613F8019C13F8028C013A48EA46
:10F7680009282CF8048C03F102030CF1040CF1D1E4
:10F778001C4B1A681C4B92B213445B002A46D3F800
:10F7880000C01D60DEF800302B44CEF80030DFF8F2
:10F7980064E0DEF8003023F4E04323F040039BB23A
:10F7A80083F0300343F4004343F08003CEF8003085
:10F7B80000E000228A4203D02368DB1B312BBFD92B
:10F7C800531A58425841BDE8F0830120BDE8F08340
:10F7D8001046BDE8F0831846BDE8F083982D002058
:10F7E800BC290020505C00400A300020D8260020A8
:10F7F80084610040045C0040002280F8452087E7CF
:10F8080090F84420531C0244DBB280F8443082F85C
:10F81800301090F845200AB1132B00D978E77047CB
:10F82800014B5868C0B27047D826002001207047A5
:10F838007047704720B9034B1B6808221A8270472B
:10F84800014870471C1D00209C00002020B9034B74
:10F858001B6808221A827047014870471C1D002047
:10F868009C00002021B901288CBF0220002070478D
:10F878000220704710B5094B1A68D378042B0BD8AF
:10F88800074C518ADB00234418B99B895B1A138201
:10F8980010BD9B68581810BD002010BD1C1D00200D
:10F8A8009C000020054B1968054B4A8A18B99B8DA6
:10F8B8009B1A0B827047986A104470471C1D0020E1
:10F8C8009C000020054B1968054B4A8A18B99B8E85
:10F8D8009B1A0B827047186B104470471C1D002040
:10F8E8009C000020074B1B681B7803F07F03212B2B
:10F8F80006D100F0DF00022814BF02200020704764
:10F90800022070471C1D0020212810B508D1114B7A
:10F918001B681B7803F07F03212B10D0022010BD39
:10F928002028FBD10B4B0C4A1B6810701B7803F086
:10F938007F03212B094B18BF00230BB9EEE7084BB7
:10F94800044A12680024936154822046984720464E
:10F9580010BD00BF1C1D0020BB2D00203DF8000875
:10F9680055F800087047034B1A78202A04BF002274
:10F978001A707047BB2D0020014B04221A60704793
:10F98800982D0020034B9B7A13B1034B05221A6074
:10F99800704700BF181F0020982D0020F7B51C4B9A
:10F9A8005A681D460AB95C6800E00124187A0021EB
:10F9B800CAB2A24201F1010107D202AE2F181644C1
:10F9C8003A44527A06F8042CF2E75A68121B5A6035
:10F9D8001A7A5D6822441A729DB903204021F9F70A
:10F9E80011F80C4A136823F4804323F070039BB288
:10F9F80083F4405343F4004343F080031360044B03
:10FA08001D72002CCBD09DF8040003B0F0BD00BFE0
:10FA1800D82600200C5C00402DE9F843664B674E61
:10FA28001B68DFF8B881664A00254FF0C0099D724F
:10FA380083F80990DD723560D8F8003023F4EC4380
:10FA480023F0700343F400739BB2C8F80030D8F871
:10FA5800003023F4E04323F040039BB248F28004D3
:10FA680083F010032343C8F80030336812FA83F395
:10FA78005B0040271A681F6033689BB203F100538C
:10FA880003F540535B0028461A6880221A60D8F8AC
:10FA9800003023F4F8731B051B0D2343C8F800300E
:10FAA800484B93F82C10F8F7ADFFD8F80030464AC9
:10FAB800464923F4804323F070039BB283F44053F8
:10FAC8002343C8F80030136823F4EC4323F0700391
:10FAD8009BB21360336811FA83F35B000320196843
:10FAE800C3F8009013683A4923F4E04323F0400335
:10FAF8009BB283F0200323431360136823F48043ED
:10FB080023F0700323439BB21360536823F4EC4340
:10FB180023F0700343F4C0639BB25360336811FA57
:10FB280083F35B0019684FF480711960536823F4FC
:10FB3800804323F0700323439BB25360536823F43C
:10FB4800E04323F040039BB283F020032343536038
:10FB5800D8F80C301F4A23F4EC4323F070039BB20F
:10FB6800C8F80C30336812FA83F35B0039461A6818
:10FB78004FF488721A60F8F745FFD8F80C3023F470
:10FB8800804323F070039BB283F440532343C8F8A7
:10FB98000C30D8F80C3023F4E04323F040031C4326
:10FBA800A4B2C8F80C402846F8F7A0FE0A4B012278
:10FBB8001A60BDE8F88300BF1C1D0020505C00409F
:10FBC800043000200C000020045C004008300020B5
:10FBD800103000201C300020982D0020005C0040D0
:10FBE800134A144B50681B68181810B5146808D0CD
:10FBF80011490822F7F753FC204610490422F7F769
:10FC08004EFC0F4B1A68002393720E4A01211160B3
:10FC18000D4913604FF4E0500B6010600B480B6007
:10FC28004FF43641A0F84A101160094A136010BD1C
:10FC3800B0F7FF1FACF7FF1FD6000020E60000203A
:10FC48001C1D0020405C0040445C0040D826002079
:10FC5800982D0020104B93F84C2013B51C46C2B9C0
:10FC68000E4B1B68ABB11A681AB10D4948690243BB
:10FC78004A619A88ADF8042002228DF80720986816
:10FC8800002201A98DF80620F5F736F8012384F83B
:10FC98004C3002B010BD00BFD8260020F002002072
:10FCA800001002400A4B10B519684FF6FB720A4063
:10FCB8001A60084A927A1C46074B0AB1052200E0EE
:10FCC80001221A6001F012FA4FF43643236010BD86
:10FCD800405C0040181F0020982D002007B5064BF7
:10FCE8000093064B01930649064A074B0748FCF761
:10FCF800BAFF03B05DF804FBC490010899900108AD
:10FD08002C9E0108369E0108B8900108099E01083A
:10FD180008B5037833B90C4B0C481978BDE808408E
:10FD2800FCF7A1BF05F0D4FC02280CD8064B1870CC
:10FD3800074B0C2202FB0030064B06301860FDF71B
:10FD480087F90548E5E708BD282700203D9E0108FA
:10FD58005C1A002034120020B793010808B5037814
:10FD68003BB90B4B0B4893F8A417BDE80840FCF7C8
:10FD78007ABF05F0ADFC022808D8054B83F8A40724
:10FD8800FDF7CCF8FDF788F90348E8E708BD00BFA0
:10FD9800BC120020419E0108B793010838B50378CA
:10FDA80003BB214B1B6801330F2B07D81F490C22BB
:10FDB80002FB03121C4695682DBB00E01C4601346B
:10FDC8000F2C01DD002400E005D818490C2202FBA5
:10FDD80004129568BDB99C42F1D11548BDE8384078
:10FDE800FCF741BF05F074FC0F28044605D80F4AFC
:10FDF8000C2303FB00239D682DB921460D48BDE85F
:10FE08003840FCF730BF084B1C6000F061FC21460D
:10FE18002A460948FCF727FF0C235C43034B185D6F
:10FE2800BDE8384000F068BCF0000020B87F010849
:10FE38004E9E0108649E01087C9E010873B50378F4
:10FE480013B9F9F7A3FA3DE01F4901AA05F0A1FC8F
:10FE5800002401462646254699B134B1012C08D123
:10FE6800084605F035FC064603E0084605F030FC78
:10FE780005461549002001AA05F08BFC013401460E
:10FE8800EAE70B2D02D911480C220BE0022C10D105
:10FE9800A6F57A73B3F57A7F07D90D484FF47A71CE
:10FEA8004FF4FA62F9F7EFF90CE00A4B03EB45035C
:10FEB8005E80084B084803EB45032946B3F9022046
:10FEC800FCF7D1FE02B070BD1E980108109601081B
:10FED800819B010828270020939E010838B50D4C06
:10FEE80023688342054606D1F9F71BFD2046002109
:10FEF8004C2205F052FBE36CAB4209D12846F9F7D6
:10FF080010FD054800214C22BDE8384005F045BBEE
:10FF180038BD00BF241D0020701D0020034B1A6847
:10FF2800D379591C1344D171187A7047481B0020A3
:10FF380010B5FFF7F3FF84B2FFF7F0FF04EB0020E2
:10FF480080B210BD10B5FFF7F3FF0446FFF7F0FFCE
:10FF580004EB004010BD064B10B504462146186856
:10FF680000F062FC034B1B6898796040987110BDE3
:10FF78004C1B0020481B002038B5044624200D46A1
:10FF8800FFF7E9FF4D20FFF7E6FF002C084C14BFF0
:10FF980021203E20FFF7DFFF2368002228469A71C0
:10FFA800FFF7D9FF236893F84900BDE83840D2E746
:10FFB800481B002001460020DEE710B50446C0B209
:10FFC800FFF7C9FF200ABDE81040C4E710B5044692
:10FFD80080B2FFF7F2FF200CBDE81040EDE737B51F
:10FFE80082888368044610060D4641BF2B4991F864
:08FFF800A4174FF4CC7000FBCC
:020000040801F1
:100000000133D10544BF2849097802F03F0244BFBB
:1000100001EB410103EB8103042A12D006D8012A27
:100020000DD0022A32D193F9001030E0102A0AD004
:10003000202A0AD0082A29D1B3F9001027E019781C
:1000400025E0198823E0196821E093ED000A68464D
:10005000FCF7A2FC01461548FCF709FE05B3D4EDF8
:10006000037A6846B8EEE70AFCF796FC01461048AA
:10007000FCF7FDFD94ED040A6846B8EEC00AFCF7F3
:100080008BFC01460A48FCF7F2FD09E00021094813
:10009000FCF7EDFD25B10848E1682269FCF7E7FDB2
:1000A00003B030BDBC12002028270020299701088A
:1000B00022970108A69E0108A29E0108024B014654
:1000C000D86900F0B5BB00BF2827002010B5441E3A
:1000D00014F8011F21B1034BD86900F0A9FBF7E721
:1000E00010BD00BF28270020F7B52B492B4B0878FF
:1000F0002B4D1C682B4B05EB80001A882A4BD0F83F
:10010000C0101B78294800914FF47A71B4FBF1F1CB
:10011000FCF7ADFD26484821FCF7A9FD254B1F68DB
:100120000026F3B205EB8302D2F8D010E9B1012426
:100130009C403C4217D0220715D01F4AD25C0B20AE
:1001400000FB0323164A1D4802EB8303D3F8F0207B
:10015000FCF78DFD022C06D1194B93F8281011B134
:100160001848FCF784FD0136DBE71748FFF7AEFFC0
:10017000164B17481A68174B9A420CBF164B174B71
:100180001A88174B198892B24FF4FA6303B0BDE88E
:10019000F040FCF76CBD00BFF01A0020BC29002025
:1001A000B87F0108901A0020F4000020A99E0108E1
:1001B000EC9E0108A01A0020FC000020FC9E010813
:1001C00028270020049F01084C9F0108CC11002023
:1001D000089F010800540040D0110020D2110020D7
:1001E000C81100202DE9F0410024804625460F4E1D
:1001F000A7594146384605F057FA58B139460C48D8
:10020000FCF735FD30190021FFF7EDFE0948FFF737
:100210005DFF0135143440F644439C42E7D11DB9DB
:100220000548BDE8F04151E7BDE8F081588101087B
:10023000A09701084C9F0108679601082DE9F04F2F
:100240002DED028B83B0054605F0EFF9064620B18F
:10025000012818D12B782A2B15D15C48FFF736FFDF
:1002600000245B4D5B486159FCF701FD28193146BC
:10027000FFF7B9FE5848FFF729FF143440F644430E
:100280009C42EED19CE028463D2105F0C0F90028B3
:1002900000F08F800346994613F8012D202AFAD0EA
:1002A000441C204605F018FA80462046FCF7EAFA7E
:1002B000C5EB0909B0EE408A0026DFF834A114220C
:1002C00002FB06F40AF5D07B54F80B70384605F0B3
:1002D000ACF903461A4628463946019305F0AEF9B3
:1002E000019B00285BD15FFA89F29A4257D10AEB51
:1002F0000402D2ED6B7AF8EEE77A0BEB0405B4EE6C
:10030000E78AF1EE10FA48DBD2ED6C7AF8EEE77A84
:10031000B4EEE78AF1EE10FA3FD8B2F8A431D2F881
:10032000A82113F0200F08BF08EE108A1C0641BF59
:100330002A4991F8A4174FF4CC7404FB0122D90583
:1003400044BF2749097803F03F0344BF01EB410153
:1003500002EB8102042B18EE100A0BD004D8013BEB
:10036000012B0ED810700CE0102B05D0202B06D0DE
:10037000082B06D1108004E082ED008A01E082EDB6
:10038000008A39461748FCF772FC2846002103B062
:10039000BDEC028BBDE8F04F25E6134803E00136C3
:1003A0009D2E8AD1114803B0BDEC028BBDE8F04F01
:1003B0008CE6284603B0BDEC028BBDE8F04F11E798
:1003C00003B0BDEC028BBDE8F08F00BF3A9F01087F
:1003D00058810108A09701084C9F0108BC12002019
:1003E000282700204F9F01085A9F0108679601089F
:1003F000B87F010870B50546284605F016F906468F
:1004000058B9194B19485A79194B03EB8203BDE8C7
:100410007040D3F8E01DFCF72ABC28461549324647
:1004200005F00CF960B91448144CFFF74FFE54F86E
:10043000041F19B11248FCF71AFCF8E7114805E04F
:100440000024114B53F8241019B91048BDE870402E
:100450003CE62846324605F0F1F801340028F0D198
:10046000014B0B4D5C71C7E7BC1200207A9F01085D
:10047000B87F010840970108869F0108988D010800
:100480003C9701084C9F01089C8D01086796010864
:10049000B793010808B50748FFF718FE064BD8695F
:1004A000F9F738FA00F02EFBFCF712FD034B044A73
:1004B000DA6008BD999F01082827002000ED00E0C0
:1004C0000400FA0508B50548FFF700FE00F0BEFB82
:1004D000FCF728FDBDE80840DCE700BFA59F010848
:1004E00008B50448FFF7F2FDFCF71CFDBDE8084025
:1004F000D0E700BFBB9F0108034B4FF4085208B17F
:100500009A6170471A85704700100048034B4FF4FA
:10051000085208B11A8570479A6170470010004868
:1005200010B544780078002202FB02F3193B6343C4
:1005300003F6C413534340F6C411434393FBF1F352
:10054000034921F812300132072AEDD110BD00BF56
:100550006C2700200430114B33F91000B0F5617F97
:1005600010B506DB40F6330398420246A8BF1A4690
:1005700001E04FF461720C78192340F2833013FBD1
:100580000404944207DA497813FB01039342B4BF91
:100590000020012010BD002010BD00BF782C0020DD
:1005A00010B500F1500302788A4203D18478C278F2
:1005B000944204D304309842F5D1002010BD0120AC
:1005C00010BD0B4B1B6813F4805F0A4BB3F9063068
:1005D00005D0C089421A934207DD084400E0008A32
:1005E0008342B4BF0020012070470120704700BF44
:1005F00098290020782C00201FB5094B1B681B038D
:100600000AD58DF8040001230D2001A98DED030A00
:100610008DF80530F9F798FD05B05DF804FB00BFD3
:10062000982900201FB5084B1B681B0309D58DF8BE
:100630000400029100230D2001A98DF80530F9F77F
:1006400083FD05B05DF804FB9829002010B50A4A27
:100650000A4B11689B6800BF12689142F7D1084AA3
:1006600014694FF47A7000FB04F2D31AB3FBF4F36D
:1006700000FB013010BD00BFBC29002010E000E0ED
:100680006C27002038B50446FFF7E0FF0546FFF76A
:10069000DDFF401BA042FAD338BD10B504462CB193
:1006A0004FF47A70FFF7EEFF013CF8E710BD024A05
:1006B0001368013313607047BC290020024B5B694B
:1006C00003B11847704700BF6C270020014B1B681F
:1006D000184700BF9C2D002010B50020FFF7F6FF43
:1006E000054B00241C7001F003FD044B1C76DC61FB
:1006F0001C845C6210BD00BF7C2D00206C27002094
:1007000010B510B9BDE81040E6E700230C225A43AB
:100710000A4C1119125D824203D00133102BF5D11E
:1007200010BD074B586A18B14A784078824203D20C
:10073000002259621A84DA6110BD00BFB87F010837
:100740006C27002010B540001428A8BF14200023F7
:10075000074A022199540B4499181424834201F842
:10076000014CF5DBFF21D1540F20BDE81040C7E755
:10077000542700202DE9F84380460B25013D3FD04A
:10078000224B4FF488429A614FF488521A8508F13F
:10079000010632274FF005091C4CA38A9BB283F453
:1007A0008843A382A38A9BB283F48853A382012047
:1007B000FFF78CFF3846FFF770FFA38A9BB283F4E4
:1007C0008843A382A38A9BB283F488530020A38228
:1007D000FFF77CFF3846FFF760FFB9F1000F08D044
:1007E000B9F10109D8D14FF4FA70FFF756FFFA2793
:1007F000D2E7013ED0D14FF47A70FFF74EFFBDE74C
:10080000034B044ADA60BDE8F88300BF00100048DB
:1008100000ED00E00400FA0503681B69184703684F
:10082000DB68184703689B68184703685B681847CC
:1008300003681B6818472DE9F84FB0F9023093425E
:1008400018BF00232DED048B18BF037005780446F4
:100850000E469146002D40F0978007EE902ADFED7E
:100860007D8AF8EEE77AB6EE009A67EEA88ADFEDA9
:100870007A7A68EEA78AA04668EE898A2746B0EEA3
:10088000680AFCF795FAB0EE408AB0EE680AFCF709
:10089000EFFA88EE000A40F2DC5363651023A4F8F7
:1008A00052301823A4F85030DFED6C6A60EE266AEF
:1008B000B7EE006AB0EE667AA0EE007AD0EE006A7B
:1008C00037EE067A76EE866AC6EE077A84ED046A1B
:1008D00027EE807AB0EE498A27EE007A77EE075A43
:1008E00084ED017AC4ED025A70EE005A84ED037A69
:1008F000B8EE007AA5EE807A27EE877A67EEA67AC0
:1009000084ED057AC4ED067ADFED557A98ED047A28
:1009100027EE277AF0EE678AB5EEC07AF1EE10FA8C
:100920004CBF77EE487A77EE087A013517EE900AD9
:1009300001F0C2FFD8ED017A67EEA87AC7E90E018F
:10094000F5EEC07AF1EE10FA4CBF77EEC87A77EE8A
:10095000887A08F1040817EE900A01F0ADFF032D24
:10096000C7E9080107F10807CED1A6F2DC531B0442
:100970002367E3676367C4F88030A367C4F88430F3
:100980000123A4F802902370D4F85490B4F9528053
:10099000636A276A206FE26FD4F840C0D4F88010F1
:1009A000C4F88020C9EB060606FA08F64FEAE67B93
:1009B000734307FB0B332667A7FB06671F44636C73
:1009C000656F60674FEAE27B53430CFB0B3EACFB69
:1009D00002237344B61A67EB0307E36AA26AC4F8FA
:1009E00084104FEAE07B434302FB0B3EA2FB002353
:1009F0007344B6185F41E36CA06CB4F95020A5674E
:100A00004FEAE17B4B4300FB0B33A0FB0101194490
:100A1000636B361A206B4FEAE57B05FB03F300FBA3
:100A20000B3367EB0107A0FB0501194480197941DD
:100A300001F010FD08F1FF3201239340E067C01878
:100A400041EBE371424601F005FDBDEC048B4844E7
:100A5000BDE8F88F6F12833ADB0F4940F404B53FCD
:100A60000000804B2DE9F8430024234B93F8586095
:100A7000E0B2B0420CD203EB8003204A9B6A32F80A
:100A800010101BB10B2801D8DB6898470134ECE744
:100A90001B4B1B685B032DD500242346E2B2B242F8
:100AA00028D2DFF8549009F128074FEA840857F854
:100AB000242055689D4215D02846FCF701FEEFF32F
:100AC0001283502282F3128828216A6A01FB009067
:100AD0000132C0F880206A6942F001026A61DBB22B
:100AE00083F3118857F808301B6800221A6001341C
:100AF0002B46D3E7BDE8F8836C27002014120020B2
:100B00009829002008B50E4B1B6813F4805F0D4B2D
:100B100014BFD3F89C21D3F8A02193F858109288E1
:100B20000023D8B2884204D2074820F813200133AA
:100B3000F7E7FFF797FF3220BDE80840ADE500BFBB
:100B4000982900206C270020141200200A4B1A68F4
:100B50000A4B30B502F48052D3F89C41D3F8A0512F
:100B600000230AB1A18800E0A988054820F81310E5
:100B700001330C2BF5D130BD982900206C270020C3
:100B80002A27002070B5124D0024214605F2A51039
:100B9000702285F8A44104F004FD2146D5F81832EE
:100BA0000B4A0B4493F9020080B102F2A5141E68AF
:100BB0000E5108199C8884809B79837192F8A43126
:100BC00007310133702982F8A431E7D170BD00BF2D
:100BD0006C270020094B1A680E2303FB0020437A80
:100BE000FF2B07D0064A12789A4203D9054A32F8F9
:100BF000130000E0808800B2704700BF9C1F0020F7
:100C0000C01D0020782C00200E4B1A786C2A16D1BB
:100C10005A88B2F5FA6F12D11A79BE2A0FD193F819
:100C2000CD27EF2A4FF000000BD113F8012B5040D5
:100C3000054A9342F9D1B0FA80F04009704700208C
:100C40007047704700F80308D0FF03082DE9F04F04
:100C50002DED028BEC4D00214FF4FA6285B0284651
:100C600004F09FFCE94B05F537721A60E84A00234F
:100C70001370E84A05F2A67111606C222A700322F3
:100C80006A714FF48072AA604FF41672A5F864215D
:100C9000FA22A5F866214FF4FA722021A5F86C21FA
:100CA000012285F85E2185F8681185F869216E2199
:100CB00085F86A2185F87C2185F88421052285F84C
:100CC0007A1185F81B220A2140F2DC5285F87B114B
:100CD000A5F896212B2140F24C4285F87D11A5F80C
:100CE0009821212140F26C7285F87E11A5F89A2195
:100CF000232140F2753285F87F11A5F89C214FF42D
:100D0000C87140F64302A5F89E21A5F880112A4635
:100D10002C46032BCCBF0121002103F1010382F8F3
:100D2000A01114BF1E217521122B82F8A11102F10E
:100D30000202EED14FF4FA63A4F8C631A4F8CA3126
:100D4000A4F8CE31A4F8D23140F27E40052340F21F
:100D50007E5684F8E031A4F84001C82340F23A708E
:100D6000A4F8486140F2EA5601274FF47A794FF02F
:100D7000320BA4F8E431A4F842014FF4C87340F2F6
:100D8000DC50A4F84A61DFF884A2A4F8E83140F20C
:100D9000B4561E211922A4F84601A4F84C61A4F807
:100DA000C491A4F8C891A4F8CC91A4F8D09184F887
:100DB000E27184F8E37184F8E671A4F84491A4F830
:100DC0004EB184F89311029184F8E12101920390CD
:100DD000A4F8503184F8DF7184F8EC71A4F852B1B2
:100DE00084F8EF71F7F78CFCDAF800300299019A79
:100DF000DFED897A9FED898A00262673D9721973EF
:100E00005521D9700F215971DA712221212299714E
:100E10005A740E2153221974DA7635215A224FF072
:100E2000780C4FF028084FF02D0E99761A720A218F
:100E3000642283F80AC0DFF800C283F80DE09974D9
:100E400002911A7783F814E01E7083F8018083F80A
:100E5000158083F8028083F81680DE7583F804B06D
:100E60009E731E76DE735E7683F809809F77C3F8E3
:100E700038C0C3F83CC0DFF8C4C1C3F828C0DFF8ED
:100E8000C0C1C3F834C04FF4FA7EDFF8B8C1A3F88C
:100E90004EE0C3ED0B7AC3ED0C7AC3F848C04FF0B7
:100EA000140EB7EE087AF1EE047A039883F850E056
:100EB0004FF04B0C83F84CC083ED087A83ED097A30
:100EC00083ED108AC3ED117A4FF0460CA4F8B007F9
:100ED000042084F8A62784F8A7C784F8AEE784F82E
:100EE000A8B784F8A96784F8AD6784F8AA6784F87E
:100EF000AB6784F8AC6783F85C0015200192A3F817
:100F00005860A3F85A60A3F85660C3ED187A83F8C6
:100F1000648083F8658083F868004148D86641485A
:100F200018674148586783F878704048F7F72EFCF7
:100F3000DAF80030029983F81161C8224FF4487042
:100F400083F8126183F8138183F8147183F81861B0
:100F5000A3F8160184F8D721019A84F8D611A4F8D1
:100F6000D89184F8DA61A4F8DC2119460E2202FB3C
:100F700006326FF0170082F81901032082F81A0177
:100F80006FF02F0082F81B01072082F81C016FF020
:100F9000230082F81D01052082F81E0101365A2027
:100FA00081F8200181F821016422FF20082E81F8B8
:100FB0001F2181F8220101F10E01D7D1002183F810
:100FC0008911C821A3F88A11142183F88C11A3F880
:100FD00090211E214FF4967283F88D11A3F892216F
:100FE0000121282283F88E11A3F89421104B18EECA
:100FF000102A45F8102F9D42F9D10E4800214022B9
:1010000004F0CFFA20E000BFBC1200201012002034
:101010002827002034120020CDCCCC3E0000000058
:101020009A99193FF6287C3F3D0A773F57AA010855
:101030007C130020581500208FC2F53C0000604052
:101040006666663F000040400023274D274C5959F3
:101050001A1904330868C2F89C02382BF5D104F53C
:1010600007700021802204F09CFA05F138017022FB
:1010700004F5077004F08AFAFDF776FFDAF80060ED
:1010800000230125314604F274404FF4CC7284F8F9
:10109000CC3784F8CA5784F8CB5704F077FA04F2B7
:1010A0000C6031464FF4CC7204F070FA104B1B68A0
:1010B0001A68C4F8B2275A68C4F8B6279A68C4F800
:1010C000BA271A68C4F8BE275A68C4F8C2279A68B3
:1010D000C4F8C627022384F8C85484F8603605B0E3
:1010E000BDEC028BBDE8F08F648E0108BC120020BD
:1010F000341200201549D1F8883043F47003C1F848
:101100008830134B1A6842F001021A605868114A7D
:1011100002405A601A6822F0847222F480321A6007
:101120001A6822F480221A605A6822F4FE025A6079
:10113000DA6A22F00F02DA62186B074A02401A6379
:1011400000229A604FF000638B60704700ED00E072
:10115000001002400CC07FF8CCFC00FF38B5094BF2
:1011600093F8CC5765B9084C2068F8F7DEFB074BBD
:1011700025601B78022B03D1BDE83840F7F77FBA12
:1011800038BD00BFBC120020DC290020D929002076
:10119000044B93F8CC371BB9034B1868FFF73CBBE3
:1011A00000207047BC120020DC29002038B505461D
:1011B0000446204614F8011B21B1034B1868FFF7C1
:1011C00037FBF6E7401B38BDDC2900200FB407B51C
:1011D00004AB064953F8042B01930020FBF75AFC9B
:1011E00003B05DF804EB04B0704700BF5B13010867
:1011F000024B01461868FFF71BBB00BFDC2900202B
:10120000F8B5011F06460023083051F8042F02F1FB
:1012100020043F2C3AD802F108040F2C06D80232E1
:10122000032A04D9002B08BF012300E002238142D6
:10123000EBD1012B30680ED0022B1AD0736803F06B
:1012400003039B0000F0030043EA0010B36803F0BF
:101250000303184317E000F00F0040F04000FFF7D1
:10126000C7FFB068736800F00F0040EA0310C0B217
:1012700009E000F03F0040F08000FFF7B9FF30794F
:10128000FFF7B6FF307ABDE8F840B1E706F10C078A
:1012900034463A46002552F8043D03F18001FF2907
:1012A0004FEA850510D903F50041B1F5803F02D220
:1012B00045F0010508E003F50003B3F1807F34BF7A
:1012C00045F0020545F00305B242E4D165F03F0068
:1012D000C0B2FFF78DFF05F00303022B207807D083
:1012E000032B0CD0012B13D1FFF782FF60780FE0A6
:1012F000FFF77EFF6078FFF77BFFA07808E0FFF73D
:1013000077FF6078FFF774FFA078FFF771FFE07850
:101310000434FFF76DFFBC424FEAA505DBD1F8BDF1
:1013200010B50446C0B2FFF763FFC4F30720BDE861
:1013300010405DE710B504467F2C06D964F07F00AD
:10134000C0B2FFF755FFE409F6E7E0B2BDE8104090
:101350004EE7430083EAE070ECE7084648E700BF49
:1013600040F2E9330F4A1289920704D4013B9BB241
:10137000002BF7D10BE00C4A40F2E9331070094919
:101380000989C9070AD4013B9BB2002BF7D1074A50
:10139000138801339BB21380FF2070471078C0B2CE
:1013A000704700BF003001400C3001408829002008
:1013B0000C4B0D49DA684378D243C2F30222C2F1E2
:1013C0000402934002781B010A44DBB282F8003326
:1013D00003780122580903F01F0302FA03F341F8CE
:1013E0002030704700ED00E000E100E073B50546F5
:1013F000002100680122FCF715F92A6813889BB2C6
:1014000043F001031380EB7A8DF8043001240026A9
:1014100001A88DF805408DF806608DF80740FFF7AC
:10142000C7FFEB7A1B2B0BD1192301A88DF80430D1
:101430008DF805408DF806608DF80740FFF7B8FF7E
:1014400002B070BDF0B5BE4CA3782DED028B013B10
:10145000012B85B000F26F81E578854240F06B8109
:101460002379022B00F06781B64B5B5D6371A37932
:101470006D00F2EE048A1BB16319B3F9083009E07C
:101480006319D4ED037AB3F90830F1EE677AC4ED4D
:10149000037A5B4208EE103A2369A94EB8EEC88A77
:1014A0001A0388EE288A35D5D6ED037AFDEEE77A61
:1014B00028EE280A17EE903AD6ED057A8DF80A3014
:1014C000FDEEE77A17EE903A8DF80B3004F0BEFA95
:1014D000FCEEC07A96ED060A17EE903A20EE280A46
:1014E000ADF8083004F0B2FAFCEEC07A96ED070AC7
:1014F00017EE903A20EE280AADF80C3004F0A6FA68
:10150000FCEEC07A0C2017EE903A02A9ADF80E302E
:10151000F8F71AFED4ED077A894BF5EE407AF1EE32
:1015200010FA60D1D3ED067AB4EEE78AF1EE10FA44
:1015300004DDDA6883ED068A5A61E8E0F5EEC07AE8
:10154000F1EE10FA40F3E38093F8202042B1022A32
:1015500000F2DD805A6B83ED078AFA329A63D6E097
:10156000D3ED037A38EE678AF7EE007AB4EEE78AB5
:10157000F1EE10FAACBF01210021D3ED0A7A69B176
:101580009FED717A27EE877ADFED707AB4EEE77A15
:10159000F1EE10FA58BFF0EE477A03E09FED6C7A57
:1015A00067EE877AC3ED0A7A2369654A1B0311D572
:1015B0008DF808105379116B0B440B205A788DF875
:1015C0000920DA7A8DF80A205B7D8DF80B3002A9AC
:1015D000F8F7BAFD0123226B84F8203063791344B5
:1015E0000022DA7291E0B4EEE78AF1EE10FA48BF19
:1015F00083ED078AA16B636B94ED067AD4ED076ADD
:10160000591AC943C90F77EE667A59B9B7EE006A1D
:10161000F4EEC67AF1EE10FA79DDB4EEE68AF1EE78
:1016200010FA74DDD4ED056A454BB4EEE67AF1EEBE
:1016300010FACCBF0126002666B1D3ED097A9FEDE2
:10164000427A67EE877A9FED427AC3ED097AD3ED4D
:101650000B7A0AE0B0EE007AF4EEC77AF1EE10FAF7
:1016600008DDD3ED0B7A9FED387A67EE877AC3ED0C
:101670000B7A07E0D3ED097A9FED357A67EE877A2A
:10168000C3ED097AD4ED097A206B627967EEA87A06
:101690001044FCEEE77ACDED017A9DF804304370FA
:1016A000D4ED0B7A2769FCEEE77A3F03CDED017AA2
:1016B0009DF8042042750ED546EA41018DF80810C8
:1016C0008DF80930C37A8DF80A300B2002A98DF805
:1016D0000B20F8F739FD94F82020194B022A11D17C
:1016E000D3ED0A7A9FED1B7A196B67EE877A002299
:1016F00083F82020FCEEE77A5A7917EE903A0A44F4
:10170000D37202E0022283F82020F6F7FBFEA279D2
:101710000B4B0AB1104A00E0104ADA602544D4EDC0
:10172000037AB5F9083000EE103AB8EEC00A80EE40
:10173000280A37EEC00A05B0BDEC028BF0BD00BF31
:10174000882900203C8F0108EC51783F6F12833AC2
:101750000AD7833F00007A440000A0410000A0C1E6
:101760002B4BF0B52B4D1E6805F110002F78F319A7
:101770002C46597801F00401013501F0FF0219B13E
:101780008542F3D10020F0BD224D631B022B0ADD00
:101790001AB102EB82025200D2B215F8013B303B83
:1017A0001A44D2B2F1E70021AC420AD919B101EBD7
:1017B00081014900C9B215F8013B303B1944C9B257
:1017C000F2E72E2F16D10134042000232578771953
:1017D00003EB83037F785B007F079BB244BF303D00
:1017E0005B1900F1FF3044BF01349BB210F0FF00E1
:1017F000ECD100E0002308484143642000FB0313C0
:101800000620B3FBF0F3054800FB0230F0BD00BF3B
:1018100004010020C429002040420F008096980057
:1018200030B500231A4610498C1894F83C40BCB1DE
:101830002E2C06D1013298B18C180444002584F86E
:101840003C5011440A2491F83C106343A1F1300448
:10185000092C9CBF303B5B180E2A03D80132E2E70B
:10186000184630BD002030BD882900200EB40FB5C9
:101870000749019006AB01A8064A0393FBF70AF952
:10188000019B00221A7004B05DF804EB03B07047AE
:10189000C5C70008349801082DE9F04FAB490B7813
:1018A00013F0010F87B003F0040200F07B81002ADF
:1018B00040F08581A648066816F0806640F07F817A
:1018C000980700F16F8143F004030B70A14BA24F06
:1018D0001A88A24B1A803B681B0340F11E81A04B63
:1018E00080201E70F6F7CAFF08B1FEF7FBFA9D4C88
:1018F0002578012D40F011819B4B93F8CA1721B137
:1019000093F8CB270AB1914203D3012283F8CA2767
:1019100011E096460846BEF1000F06D090FBFEFC93
:101920000EFB1C0C7046E646F5E791FBF0F183F8E0
:10193000CA1792FBF0F283F8CB2793F8CC271AB1A1
:10194000894A002182F8CC17884A93F8CC9712680C
:1019500041F6690102EBC2028A4284BF40F2E241D1
:10196000B2FBF1F282498CBFD2B204220A70B9F103
:10197000000F1FD18020F8F717FA8046D0B18021E0
:10198000F8F7ECF998F806207A4B607053F822309B
:1019900098F90000DFF8CC81B3F5613F0CBF02225B
:1019A000002202218DE8060080214A46F7F7D8FF81
:1019B000606008B90023AFE0494608F1080014222E
:1019C00003F0EFFD08F12803C8F81C3008F19C0370
:1019D000C8F8203008F58873C8F82430664B396899
:1019E0001B88A8F88431604B93F8922193F8CA873A
:1019F00093F884A1002A614A10685A7993F8CB378A
:101A0000A2F1190EC1F3C03C18BF4FF0010CDEF17A
:101A1000000747EB0E07012A14BF3A460122584F30
:101A200004929845574BD7F800E01B78039301F4D4
:101A30000069C0F3800BC1F34001C0F3C0002CBFAC
:101A40004FF000084FF0010805976A1ED2B2531EEE
:101A5000132B3DD8DFE803F00C0C0C0C0C0C0C0C19
:101A60000AADAF292B3F37121212393F049BA3E076
:101A7000039B9342B4BF0023012328E09EF800306B
:101A8000022B0BD10EEB820353ED027AF5EE407A76
:101A9000F1EE10FA14BF0123002318E00EEB02034D
:101AA0005B79003318BF012311E00B4684E0B9F1E4
:101AB000000F04D00AF1FF377B427B4100E04B4628
:101AC00003F0010378E0634676E0434674E013B127
:101AD000012393401E43142D02D80135EDB2B4E723
:101AE000059BC4F88861186819217930FEF758FD04
:101AF0000023C4F89031A4F89431A4F89631C4F8C6
:101B0000A031214BD4F89C211B68C4F8A43184F87F
:101B10008C01C4F89821022323701B4B124A1B68C6
:101B200092F8E0214FF47A7101FB0233174A1360F7
:101B3000094B1B681A062FD5154B1B789B072BD515
:101B4000144B1B78042B27D9062026E0B62D002045
:101B5000D4110020AC12002098290020FA0F002098
:101B6000C51D0020D8290020BC120020B01F002075
:101B700000010020E0750108381E0020A01A002096
:101B800010120020C4270020BC290020B40F002020
:101B9000A41A0020AA1A0020052007B0BDE8F04FC3
:101BA000FEF7AEBD5AB9012007B0BDE8F04FFEF711
:101BB000C9BD034600E05B46002B89D18DE707B025
:101BC000BDE8F08F10B5154A1378590725D523F0D5
:101BD00004031370124B1B681B0319D5114C237897
:101BE000A3F10802012A0BD8FF200021F8F7ACFA74
:101BF0000D4B1B68C4F8A431FFF7CAFA0A2306E0AC
